:020000040000FA
:040000006FD00400B9
:101000006F009044000000000000000090200020CD
:10101000A4220020A9BDF9F55C23002000000000F7
:10102000000000005C230020902000200000000051
:101030000000000090200020000000009020002010
:101040000000000090200020902000209020002030
:101050009020002090200020B82B0020902000201D
:10106000000000009020002090200020EC230020B1
:1010700090200020C22300209020002090200020FB
:101080009020002090200020902000209020002020
:101090009020002001A04111B7170040985F3AC688
:1010A000945F3247E39CE6FE3245410182800111A4
:1010B00013078008F337078093F787083EC20100C3
:1010C0000100B7170040930570052380B70413068D
:1010D00080FA2380C7040100010083C6B70493F699
:1010E000F60DA385D704238007049246F3A6068055
:1010F0000100010093760502D5CEF336078093F602
:10110000860836C4010001002380B7042380C70489
:1011100001000100B70614007D89558D88C70100C4
:1011200001000100010023800704A246F3A6068007
:101130000100010073370780137787083AC6010062
:1011400001002380B7042380C704010001000100CF
:1011500001003727004093061005A303D7802380A2
:101160000704B247F3A70780010001009307800836
:10117000F3B7078093F787083ECE01000100B71749
:101180000040130770052380E704130780FA2380CB
:10119000E7040100010003C7B70413670708A3852C
:1011A000E70423800704F247F3A70780010001004A
:1011B0000561828093760504BDC6F336078093F6F9
:1011C000860836C8010001002380B7042380C704C5
:1011D00001000100B7061400938606047D89558D31
:1011E00088C7010001000100010023800704C246F6
:1011F000F3A6068001000100733707801377870884
:101200003ACA010001002380B7042380C70401000B
:1012100001003727004093062005A303D7802380D1
:101220000704D24781B773370780137787083ACC12
:10123000010001002380B7042380C70401000100DE
:1012400098471367070C98C723800704E24719BF24
:101250000111814601468145114506CE6D24930753
:101260008008F3B7078093F787083EC601000100A6
:10127000B7170040130770052380E704130780FAAF
:101280002380E7040100010003C767041367170008
:101290002383E70423800704B247F3A707800100F4
:1012A0000100F2400561828041118146014681457D
:1012B0001145912C13078008F337078093F78708AF
:1012C0003EC401000100B7170040130670052380DB
:1012D000C704930680FA2380D70401000100FD555E
:1012E0002396B70223800704A245F3A505800100D9
:1012F000010073370780137787083AC601000100A1
:101300002380C7042380D7040100010003C76704BA
:10131000136717002383E70423800704B247F3A76A
:1013200007800100010001A0BD473305F50201005F
:101330007D1575FD8280411122C426C206C6AA848D
:10134000014463179400B2402244924441018280D8
:1013500005041305803E4204C13F4180DDB7000013
:101360009305000273A04580824573901534924026
:101370002242B2424243D2436244F2440255925561
:101380002256B2564257D2576258F25806499649E9
:10139000264AB64A464BD64B664CF64C065D965DE1
:1013A000265EB65E465FD65F09617300203041114C
:1013B000B7170040985F3AC6945F3247E39CE6FE59
:1013C000324541018280B71700401307000323888C
:1013D000E7028547171700002326F7F47300203033
:1013E000411122C406C6370400201C408297F5BF75
:1013F00037370040834747009146BD8B6389D7004C
:1014000099466394D700834757407300203097165E
:10141000000083C6F6F39387160017160000A30991
:10142000F6F203478700973700009387E75CB6978B
:101430002380E700B7E70400BC4F0946894517152C
:1014400000000345C5E98297C9B723030480154707
:101450002303E48001002302A48082808307648048
:10146000E3CE07FE23030480828083076480E3CEFB
:1014700007FE03454480828083076480E3CE07FE35
:101480002302A4808280411126C44AC24EC006C6EF
:101490001377F50BAD47AA892E8995446306F700AB
:1014A00019456537653F8D444E854537FD59FD1417
:1014B00063983401B240A2441249824941018280BA
:1014C000135509011375F50F453F2209CDB70111D9
:1014D00026CC06CEB704080051371545BD37713705
:1014E00069372AC6A53F32459377150089EB136506
:1014F00015001375F50FF240E24405618280FD147A
:10150000E9FC0145CDBF397126DC4ADA4ED852D606
:1015100056D45AD25ED006DE62CE66CCB7E700E083
:101520007D5783AA070022C603AA470023A0E71815
:1015300023A2E718B7170040130770052380E704BC
:10154000130780FA2380E70483C74704930B75FFD2
:10155000B684E20793FBFB0F8546AA892E8B32895E
:1015600037240040E187015763FA76016308D5000C
:101570008946130700026313D5000157D98F93F7EB
:10158000F70FB71C00402382FC0411472303E480BB
:101590001305F00F5D3D094CD135636D7C11B70526
:1015A0000700DA9537870700795563F2E504B387BA
:1015B0009500636EF702370B0800A94733EB65010E
:1015C0006399F90689E48144513D26850DA0DA85A9
:1015D0000945553D05090345F9FFFD14050B693D16
:1015E00081C49377FB0FFDF7DD3569FD7D55B71796
:1015F0000040130770052380E704130780FA238057
:10160000E70403C74704418B2382E704F250B7E79E
:1016100000E023A0571123A24711E254324452594B
:10162000C259325AA25A125B825B724CE24C21615F
:101630008280A5476395F90685691309F00FB30603
:101640009900B3742B01B6941349F9FFB374990050
:10165000856B33796901416B9387F9FFB3F72701F4
:1016600099E363FC340193D94900C147E3E637FFAE
:1016700099BF0569C1697D19D9B71305800D6388C4
:101680006901130500026384790113051008CA85F6
:10169000DD3B353D21DD4E99B3843441D9B7DA8540
:1016A0002D45D533CA94E30099F205097D3BA30F7C
:1016B000A9FED5BF9387F9FF93F7F70F6361FC0C81
:1016C00083C71C0413073008631FF704370708009B
:1016D000636BEB04B3079B00B706100063F5D704F8
:1016E000334BEB0089476393F9068980D549E38C36
:1016F00004ECDA850945413B11090327C9FF9147ED
:101700002320E48003076480E34E07FE2303348133
:10171000FD17EDFBFD14110B81C49377FB0FE9FF5F
:101720007D3371F5E1B5B717004003C75704B7071C
:1017300008001377070219E3B78707007955E378A4
:10174000FBEA33079B00E3FFE7F855B58547E382E3
:10175000F9F2DA852D45053B9389F4FFE38504E62C
:10176000293393F7390091EB83260480032709007E
:1017700093074900E39AE6E43E89CE84F1BFB5477A
:101780006396F9001305900BC93135BDB1471305B8
:10179000B00AE38BF9FE99476391F904B705080095
:1017A000B365BB002D45C53181448D4BA1497539C9
:1017B00063967401832704802320F9008504E3984D
:1017C00034FF8327048013172B016355070023126E
:1017D000F900D5BB2322F900FDB39D476399F902B7
:1017E00081451305B0044531BD442320090023225F
:1017F0000900FD599D3993F77400CA9703C7070084
:10180000FD14398D2380A700E39634FF6DBBA147FB
:101810006392F9046D398144630D0B008D47930485
:10182000C0036308FB009304000563048B01930469
:1018300040041375C507E30895D81945393139397E
:101840000545213126850D3909453D314931E31CD6
:1018500005D669BB91476399F90013056006F53613
:10186000F53E130590090DB7E38F09D4F154A9BBD8
:10187000BD660147173600001306C644938606A6C8
:1018800085458347060093F7F70F91C382800507CC
:10189000E3F9E6FE973700002386B742DDB77D16F1
:1018A0006206618693178601E18763D407000145CC
:1018B0008280931726003307F500AE9718439C43A8
:1018C00063E7E7007D16E37FF7FC7D5582800545E1
:1018D0008280FD15E205E18513978501618793F705
:1018E000F50F63480700FD15139725002A97584305
:1018F00065D7138517006205618582803308B502BC
:101900001C4283A80600B335B502C29733B5070160
:10191000AE98469585486367B5006394A50063E378
:10192000070181480C43C6950CC388C21CC2828043
:1019300081471397870161876343B70082801397BC
:1019400027002A97232007008507E5B7814701472D
:1019500093968701E18663C5B60013351700828030
:1019600093962700AA9694428507558FD5B793D7AB
:1019700055408A07AA979C4305453315B5007D8DD0
:10198000828017F3FFDFE702C33B2A84993705C53E
:10199000931725003E940327C4FF814711EB7D1563
:1019A00016053E954205418517F3FFDF6700A33B0F
:1019B00005838507E5B70145C5BF814713978701B3
:1019C00061876343C700828013972700B386E500D1
:1019D00094422A97850714C3D5B77D16620661869F
:1019E000014793178601E18763D507001335170078
:1019F000828093172600B306F500AE9794429C436D
:101A00007D16B58F5D8FF1BF8A05AA950147636387
:101A1000B500828083A6C5FFF11593D71600D98F34
:101A20009CC11397F601E5B72A8301480147014598
:101A30006343D7008280B387050183A80700B307FB
:101A400006019C43C697AA976384F80033B5170133
:101A50000507B3080301620723A0F8006187110896
:101A6000C1BF2A8301478147014563C3D7008280F4
:101A70003388E50083280800330EE600032E0E00AD
:101A80003388A8403308C8416384080133B508018E
:101A90008507B308E300E20723A00801E1871107E7
:101AA000E9B717F3FFDFE702C3290111B286B28459
:101AB0002E86AA850A8575372A84A6850A857935F2
:101AC00033348000060413351500018D056117F3CA
:101AD000FFDF6700432917F3FFDFE702032441110B
:101AE000AA89AE8A328BB68402C202C402C60144FD
:101AF000131C8401135C8C4163499C02939B14006A
:101B0000FD1B0549138CF4FFF15C33048901620469
:101B10006184634D740592478E04CE9423AEF4FE27
:101B2000410117F3FFDF6700C32213192400B30B31
:101B30002B01014A93172A00D69783A50B008843EF
:101B40007800340050005D3B050A93178A01E18755
:101B5000F11BE351FCFE92474E9905042320F90046
:101B6000A2473EC2B24702C63EC459B7131A890102
:101B7000135A8A41131D240093178A01E18763CF0A
:101B8000970092470A044E941CC0A2470509137996
:101B9000F90F3EC2B24702C63EC485BFB3079A03DF
:101BA00013152A0056950841780034005000050AA4
:101BB000EA97DA978C439933C1B70000197106C2CE
:101BC00012C416C61AC81ECA22CC26CE2AD02ED2BD
:101BD00032D436D63AD83EDA42DC46DECAC0CEC26D
:101BE000D2C4D6C6DAC8DECAE2CCE6CEEAD0EED29D
:101BF000F2D4F6D6FAD8FEDA97050000938505727E
:101C00008841E700050092402242B2424243D2435B
:101C10006244F244025592552256B2564257D25768
:101C20006258F25806499649264AB64A464BD64B60
:101C3000664CF64C065D965D265EB65E465FD65FE8
:101C40000961730020300000972100209381813BBF
:101C500017510020130101BB17F5FFFF1305C53A0B
:101C6000970500209385053A171600201306C6FD38
:101C700063FAC5008322050023A0550011059105D4
:101C8000E3EAC5FE17A501001305055097150020CE
:101C90009385C5FB171600201306C66563FAC500B9
:101CA0008322050023A0550011059105E3EAC5FE36
:101CB0001715002013050564974500209385854C72
:101CC0006377B500232005001105E36DB5FEFD42E5
:101CD000739002BC8D4273904280B72200009382C1
:101CE000828873900230970200209382A23193E29F
:101CF00032007390523097420000938242F1739009
:101D000012346FC0E42F73002030397101436EC666
:101D100019A0397141536AC866CA62CC5ECE19A057
:101D2000397101535AD056D252D44ED64AD826DAF7
:101D300022DC06DE33016140828241114AC026C2A4
:101D400022C406C68282B24D4101024D924C224C01
:101D5000B24B4101024B924A224AB2494101024927
:101D600092442244B240410182803D432A876373FA
:101D7000C3029377F700BDEFADE5937606FF3D8A8A
:101D8000BA960CC34CC30CC74CC74107E36BD7FED4
:101D900011E28280B306C3408A069702000096963D
:101DA0006780A6002307B700A306B7002306B70085
:101DB000A305B7002305B700A304B7002304B700A9
:101DC000A303B7002303B700A302B7002302B700A1
:101DD000A301B7002301B700A300B7002300B70099
:101DE000828093F5F50F93968500D58D9396050126
:101DF000D58D61B79396270097020000969686824C
:101E0000E78086FA9680C1171D8F3E96E374C3F86B
:101E1000A5B73367B500FD530D8B79E7B7877F7F93
:101E20009387F7F710419441B372F6003363F600DD
:101E3000BE92B3E262006397720C6318D6065041FB
:101E4000D441B372F6003363F600BE92B3E262008F
:101E50006398720A631BD60410459445B372F6006A
:101E60003363F600BE92B3E262006391720A631EAE
:101E7000D6025045D445B372F6003363F600BE92E5
:101E8000B3E26200639A72086311D6021049944962
:101E9000B372F6003363F600BE92B3E2620063935E
:101EA00072085105D105E30FD6F613170601939773
:101EB0000601631CF7001357060193D7060133058B
:101EC000F7409375F50F91E982804183C183330513
:101ED000F7409375F50F91E182801377F70F93F731
:101EE000F70F3305F74082800346050083C60500DF
:101EF000050585056313D60065FA3305D640828053
:101F000011059105E312D6FE014582802105A10548
:101F1000E31CD6FC014582803105B105E316D6FCF1
:101F2000014582804105C105E310D6FC0145828050
:101F3000B717004003C777051377E70FA38BE704B4
:101F4000130700F8A38DE7043D47238CE70413072C
:101F50005003A38CE70403C7A7051377D70F238D7E
:101F6000E7048280B717004003C7E7020D894111DB
:101F70001377C70F498F93068008F3B6068093F650
:101F8000860836C601000100930670052380D70439
:101F9000930680FA2380D704010001002387E7021B
:101FA00023800704B247F3A7078001000100410125
:101FB000828041112A83014E930E407E130F001937
:101FC000930F400663E56E12930800191303400651
:101FD000B3781503854E0D4FA14F337365020D89FC
:101FE0001335150063EFBE121308F6FF7946729899
:101FF0004208135808013307C70213D61700BE075B
:1020000032976146B3F6C60213068070B386C602E5
:102010003697A166F58F42075D8FB716004083C7DC
:10202000F60293F70708A303F1000346710083C784
:10203000F60293F70708E394C7FE83477100B716CB
:10204000004093F7F70F6388071293078008F3B7F0
:10205000078093F787083EC401000100B7170040CE
:10206000930670052380D704930680FA2380D70453
:102070000100010023AA070383C6170393E606089D
:10208000A388D70223800704A247F3A70780010093
:1020900001001166B71700407D16D45BC85F9385B9
:1020A0004703A98EF18EF5FA93068008F3B60680F1
:1020B00093F6860836C6010001009306700523805A
:1020C000D704930680FA2380D7040100010098C149
:1020D00003C7170313670704A388E70223800704D5
:1020E000B247F3A7078001000100410182807D1300
:1020F0003368E3039308E016630E08003368F303C4
:102100009308D016630808009378330093B818003A
:102110009388D81633081E01131E0801135E0E01A2
:1021200055B56393E50305486386080001486303DA
:1021300003002A8871087298FD15131E0801C20554
:10214000135E0E01C18179BD13F8150063F4BF0061
:102150007908D5B713381800E5BF83C7F60293F79F
:102160000708A303F1000346710083C7F60293F743
:102170000708E394C7FE8347710093F7F70FF1DF79
:10218000E9B531714AD966CB06DF22DD26DB4ED7B1
:1021900052D556D35AD15ECF62CD6AC96EC7AA8CCA
:1021A00002D8EF00901C2A8993078008F3B70780B4
:1021B00093F787083EDA01000100B71700401307C4
:1021C00070052380E704130780FA2380E7040100E9
:1021D000010003C7F7021377770FA387E70203C74E
:1021E000F70213678700A387E70223800704D2570B
:1021F000F3A70780010001000545AD33130780C137
:102200003347E902116A93070AE893065002BD6951
:10221000930BA004814A014B1304800893047005BA
:102220007D1AB347F9023307D7023EC0FD873ECC83
:10223000938709A69309803E3347F7023AC27D8708
:102240003AC4334739038549B399990193D9394041
:10225000B306D702B30B7703B3C6F602B3CBFB02C8
:1022600036C6FD8636C893D6FB4136CEB7460F003C
:10227000938606243349D9028566938606FAB39677
:102280009601B389E902130760553309D902930611
:102290000010B389E9023349D902B3C9F902931690
:1022A000390036CA37190040FD8636D0930D09042F
:1022B00093D7F9413ED2F336048093F6860836DC94
:1022C00001000100930770052380FD00930680FA4A
:1022D0002380DD00010001008346390593F6860F57
:1022E000A309D9048346390593E61600A309D90446
:1022F00023800D00E256F3A6068001000100130CB6
:1023000080FA116DF336048093F6860836DE0100FC
:102310000100930770052380FD0023808D010100DB
:10232000010083463905216693E60602A309D90414
:1023300083560905B3E6A6012318D9048356090577
:10234000D18E2318D90423800D00F256F3A60680FF
:10235000010001008346390593F60602638A0618D8
:1023600003463905218A6DDE0818EF001004733624
:10237000048013768608B2C20100010023809D000C
:1023800023808D0101000100B717004003C6370507
:102390001376F60DA389C70403C637051366060234
:1023A000A389C704835609052166B3E6A60123184D
:1023B000D90483560905D18E2318D90423800D0032
:1023C0009646F3A60680010001008346390593F680
:1023D00006026386061483463905A18AEDFE97003E
:1023E0000020E78040CBAA8636D497000020E78003
:1023F00080CAA256E30AD5FE835609054255B3E6C4
:10240000A6012318D904C12783463905A18AEDDE28
:10241000035609058346290582473376CA00B30669
:10242000DA0293D5F641B296B388F640E24733B864
:10243000C6002E983308F840A247B3B616013308F9
:10244000D84063C70701631DF800924763FA17017C
:10245000C247634DF80E63950701B24763E8F80E73
:10246000894663E7660FF2469315180013D3F80107
:102470005E8613951800B365B30042D646D4EF606C
:10248000C1363258050B137BFB0F63470001631203
:102490000838A258638F083613081500B336A80011
:1024A000B69513D6F5013298B336C800AE961358D8
:1024B0001800FE06B3E6060173360480137686081C
:1024C000B2C60100010023809D0023808D01010020
:1024D00001000356C902B296C206C1822316D90270
:1024E00023800D00B646F3A606800100010019BD49
:1024F000F336048093F68608B6C0010001002380FD
:102500009D0023808D01010001008346390593E67B
:102510000602A309D90423800D00864605BDF336C3
:10252000048093F68608B6C40100010023809D0054
:1025300023808D01010001008346390593E60602E0
:10254000A309D90423800D00A646A5BDE30D0BF019
:10255000F336048093F68608B6C80100010093069E
:1025600080FA23809D002380DD0001000100834666
:10257000390593F5FC0F93F6860FA309D90483461A
:102580003905CD8EA309D90423800D00C646F3A6D4
:10259000068001000100130580FA03463905930601
:1025A00039051D8A631496297336048013768608CC
:1025B000B2CC01000100130680FA23809D00238025
:1025C000CD000100010003C606001376F60D23803E
:1025D000C60003C60600136606022380C6008356A3
:1025E00009051166D18E2318D90483560905216681
:1025F000D18E2318D90423800D00E646F3A6068069
:1026000001000100130680FA8346390593F606029D
:102610006388062483463905130C3905A18AFDDA3F
:1026200008186123F336048093F68608B6D00100BB
:102630000100930680FA23809D002380DD000100C5
:10264000010083460C00116693F6F60D2300DC00B2
:1026500083460C0093E606022300DC00835609053E
:10266000D18E2318D904835609052166D18E2318EB
:10267000D90423800D008656F3A6068001000100D0
:10268000130680FA8346390593F606026385062011
:1026900083463905A18AEDFE97000020E780A09FC0
:1026A0002A8C97000020E780009FE30C85FF83566B
:1026B000090511664255D18E2318D9042923834672
:1026C000390513063905A18AFDDAF336048093F63D
:1026D0008608B6D401000100930680FA23809D008D
:1026E0002380DD00010001008346060093F6F60D0D
:1026F0002300D60023800D00A656F3A60680010015
:1027000001008356090503462905D247B376DA004E
:102710003306CA021305800C9355F6413696330DE5
:10272000F6408257333CD6002E9C3336A601330C3C
:10273000FC40330CCC403308850392564E86B335AB
:10274000A5033305A503C295EF60210A6346800106
:10275000631E0C16630C0D16130615003335A60008
:102760002E959356F5013696B335D600AA959396D5
:10277000F50105828585D18E6346B000639D051AFB
:10278000638B061A0356C90215823305D600333609
:10279000C500B2956348B000639105241306F00F9D
:1027A000637DA622894663F3561593078008F3B725
:1027B000078093F78708BED6010001003717004055
:1027C000930770052300F704930780FA2300F704AA
:1027D000010001008356C70289678117D58FC207A0
:1027E000C1832316F70223000704B657F3A7078017
:1027F00001000100FA506A54DA544A59BA592A5A67
:102800009A5A0A5BFA4B6A4CDA4C4A4DBA4D296126
:1028100082801308F5FF3335A800FD152E95135659
:10282000F5013298B336C800AA9651B1F336048048
:1028300093F68608B6CA0100010023809D0023801C
:10284000AD000100010083463905CD8EA309D904EE
:1028500023800D00D646F3A606800100010035BB9B
:10286000F336048093F68608B6CE0100010023807B
:102870009D002380CD00010001008346390593E6C9
:102880000602A309D90423800D00F646F3A60680AC
:102890000100010095BBF336048093F68608B6D29A
:1028A0000100010023809D002380CD000100010074
:1028B0008346390593E60602A309D90423800D0057
:1028C0009656F3A60680010001006DBB9306F5FF46
:1028D00033B5A600FD152E959355F501AE96B3B50B
:1028E000B600AA951396F501858269B5F336048082
:1028F00093F68608B6D801000100930680FA23807B
:102900009D002380DD00010001008356C902056699
:10291000011693F6F60FD18EC206C1822316D90294
:1029200023800D00C656F3A6068001000100850A2B
:1029300093FAFA0F49B233E6B60045C20356C9020C
:102940003305D0403338A000B305B040B38505410E
:1029500015826345B000D1E16371A608894663F032
:10296000560593078008F3B7078093F78708BEDA08
:1029700001000100B7170040130770052380E7042A
:10298000130780FA2380E7040100010003D7C70280
:102990007D8B2396E70223800704D65781BDF3364B
:1029A000048093F68608B6DC01000100930680FAE5
:1029B00023809D002380DD00010001008356C902B1
:1029C0000566011693F6F60FD18EC206C182231654
:1029D000D90223800D00E656B9B793078008F3B7F4
:1029E000078093F78708BEDE01000100371700401B
:1029F000930770052300F704930780FA2300F70478
:102A0000010001000356C70293975600B297C20710
:102A1000C1832316F70223000704F657C1BB914771
:102A200063EEB702178701001307C7AC8A05BA9592
:102A30009C41BA978287B717004003A7470B1345FD
:102A4000F5FF698F23AAE70A03A7070B698F23A85D
:102A5000E70A03A7070A798D23A0A70A8280B71780
:102A6000004083A6470B1347F5FFF98E23AAD70A28
:102A700083A6070B558D23A8A70A83A6070A758F7F
:102A800023A0E70A8280B717004003A7470B498FAE
:102A900023AAE70A03A7070B1345F5FF45BFB7179E
:102AA000004083A6470B1347F5FF758F23AAE70A5B
:102AB00003A7070A598D4DB7B717004003A7470B67
:102AC000498FEDB7914763EEB702178701001307EF
:102AD000A7A38A05BA959C41BA978287B717004089
:102AE00003A7470D1345F5FF698F23AAE70C03A73A
:102AF000070D698F23A8E70C03A7070C798D23A086
:102B0000A70C8280B717004083A6470D1347F5FF37
:102B1000F98E23AAD70C83A6070D558D23A8A70CE1
:102B200083A6070C758F23A0E70C8280B71700409F
:102B300003A7470D498F23AAE70C03A7070D1345E9
:102B4000F5FF45BFB717004083A6470D1347F5FFB4
:102B5000758F23AAE70C03A7070C598D4DB7B7173C
:102B6000004003A7470D498FEDB7B71700408847CE
:102B7000420541819377050491EB9377F501375531
:102B8000E801130505803345F50282809377050C33
:102B9000130700046397E7009377F50137459C1C02
:102BA000CDB72165130505D0828037E700E01C43CF
:102BB0005443A183E206D58F1CC1FD572320F7188B
:102BC0002322F718828013178500B7E700E023A0BF
:102BD000E710618123A2A7108280B7F700E0884741
:102BE000CC478280814737370040A14663C4C70085
:102BF000328582800345B740E38EA6FE3385F5001B
:102C00000345050085072304A740CDB7970700209B
:102C10009387476A9C43173700201307A7563E95B2
:102C2000636EE500174700201307C79D6368A70080
:102C3000170700202320A7683E858280FD57EDBF3F
:102C4000411122C406C62A840D372947B307E5027D
:102C5000B2408D83B3D7870222449507B3D7E702EA
:102C600037370040C207C1832316F7004101828035
:102C7000716541111305052006C6D937B7370040E5
:102C8000130770F82381E7000D47A381E7001307BE
:102C90000004A380E70005472387E700B240410115
:102CA000828037370040834727001A0593F7F703E0
:102CB000C98F93F7F70F2301F7008280B7370040E1
:102CC00003C7170019C9D98DA380B70003C7070030
:102CD000136787002380E700828093C5F5FFF98D95
:102CE000A380B7008280B73700402147B736004045
:102CF00091E1828003C6B700E30CC7FE05050346D9
:102D0000F5FFFD15C2052384C600C181D5B7411169
:102D100022C406C62A84913D2947B307E502B24082
:102D20008D83B3D7870222449507B3D7E70237379D
:102D30000040C207C1832316F740410182807165BC
:102D400041111305052006C6D937B73700401307D0
:102D500070F82381E7400D47A381E7401307000483
:102D6000A380E74005472387E740B24041018280C6
:102D7000CC41411106C6328503C6150083C5050046
:102D800022064D8E42068D654186138875A2630C1E
:102D90000611634BC804138845A26300060D634AFD
:102DA000C800938535A26301B60823900600294622
:102DB0004DA0138855A26305060D938565A2E31601
:102DC000B6FE8D451D4663E6E5081146198E63F390
:102DD000C7003E86B7E704002390C600FC479795DE
:102DE0000100938565349DA0138895A263030611A5
:102DF000634E060D1388A5A263000613938505A5EF
:102E0000E315B6FA99451D4663E5E504198E63F3AB
:102E1000C7003E86B7E704002390C600FC4797052D
:102E200000209385A5491DA09D451D4663E3E5024D
:102E30002146198E63F3C7003E86B7E70400FC47BE
:102E40002390C600970500209385C54ABA958297BE
:102E50000146B240328541018280AD451D46E3EA1C
:102E6000E5FE3146198E63F3C7003E86B7E70400DE
:102E70002390C600FC47977501009385E56BF9B771
:102E8000B1451D46E3E7E5FC3546198E63F3C700FF
:102E90003E86B7E704002390C600FC479775010003
:102EA0009385856A65B78D451D46E3E4E5FA1146CD
:102EB000198E63F3C7003E86B7E704002390C6006F
:102EC000FC47979501009385E52649B78D451D463A
:102ED000E3E1E5F81146198E63F3C7003E86B7E7D4
:102EE00004002390C600FC47979501009385452672
:102EF000B1BFA5451D46E3EEE5F42946198E63F3FF
:102F0000C7003E86B7E704002390C600FC479775CC
:102F100001009385A5611DBFB5451D46E3EBE5F2B4
:102F20003946198E63F3C7003E86B7E70400239045
:102F3000C600FC47977501009385455E01BFB7E762
:102F4000040003A3071397060020938626D9414661
:102F5000A54517050020130565CF02832D4559EFC0
:102F600003C5050009476317E50803A8450041119B
:102F700006C6034718003285034608002207416849
:102F8000518F930828FE6308170363E9E8000518CA
:102F9000630307052390060029451DA8130648FE74
:102FA000630BC7021518E31707FF15463E87637BBF
:102FB000F602154705A83E8691C30546B7E704000B
:102FC000FC472390C6004206CC45418282970145CA
:102FD000B240410182801306700F3E876374F60091
:102FE0001307700FB7E704002390E600FC471316A1
:102FF0000701D9BF23900600054582808280416782
:1030000079176304E504411122C406C685472A8462
:10301000639FF500B7E7040022852244B24003A372
:103020008713970500209385A52D410102838947C9
:103030006399F500B7E7040083A7070B85458297DE
:1030400071D9B2402244410182808280797122D4B8
:1030500052CC2E842A8A97750100938525511775C5
:1030600001001305655206D63AC626D24AD0B68468
:1030700032894ECEEF50B142A68517750100130577
:10308000A551EF50D1412945EF50B1458347840008
:1030900093F70702E1E78349040089470545324772
:1030A0006396F908544083C7160083C60600A2073A
:1030B000D58FC166138616FE638CC7028D16638F8B
:1030C000D7068D669386269029456391D706B7E784
:1030D0000400A285225403A34714B250F249A686E5
:1030E0004A86925402595285624A85474561028355
:1030F0002D450DEF9307700F354563E99702B7E74C
:103100000400FC4748441306700FCA858297814922
:10311000970700209387871F9C43014581CB9C43E1
:1031200091C74E852686CA8582970145B2502254A2
:1031300092540259F249624A456182802D457DF7D9
:103140009307700F3545E3E397FEB7E70400FC47AC
:1031500048441306700FCA8582975DBF2145F9B7B1
:10316000411122C437E404008327841326C2AA84B1
:10317000416506C697050020938585187D158297C1
:103180008327C40A170500001305A5E785888297E1
:1031900095C0032304132244B240924497060020B2
:1031A000938686C54146C545170500201305C5B35E
:1031B00041010283B2402244924401454101828090
:1031C00019C59707002023A3A71401458280454510
:1031D00082801147636AA70A977601009386C637F3
:1031E0000A0536951841411106C63697AE87B28555
:1031F00002871307700F6145639DE700B7E704007E
:10320000FC471306700F170500201305E51682977B
:103210000145B2404101828005476145E39BE7FEDD
:10322000B7E70400FC470546170500201305050D08
:10323000F9BF1307700F6145E39DE7FCB7E7040092
:10324000FC471306700F1705002013056522C1B750
:103250001307700F6145E39EE7FAB7E70400FC47E8
:103260001306700F17050020130505304DB71547DD
:103270006145E390E7FAB7E70400FC4715461705F8
:1032800000201305250861B709458280411126C237
:10329000B7E4040083A7C41322C44AC006C62E8420
:1032A000970500209385C5052A898297058905C55C
:1032B00097070020938747A383D7A70BA28503A373
:1032C000440D2310F4002244B24092444A8502493E
:1032D000014641010283B2402244924402494945D9
:1032E000410182809707002023840702970700206E
:1032F00023A20702B717004003A7070CB706C0FFB9
:10330000FD16758F23A0E70C03A7070DB706400035
:10331000558F23A8E70C03A7070C3D9B23A0E70CC0
:1033200003A7070D1367070123A8E70C8280B717CF
:10333000004003A5470C83A7470C5981134515008E
:10334000C18B058999E3136525009707002083C782
:1033500027FC6380A70297070020238BA7FA11C9D7
:1033600097070020938707FB03A30700630303006D
:103370000283828011456FE0DFE0411193962500C2
:10338000AA852D4506C697F0FF1FE780C017B240FB
:10339000014541018280011122CC06CE3714004044
:1033A00026CA4AC84EC652C483447405034AB405AB
:1033B0008349840503499405EFE09FB78347A4053B
:1033C00093F4F40F137AFA0F93E71700230DF40424
:1033D00093F9F90F1379F90FB717004003C7A70541
:1033E000058B6DFF03D5C705A38D4705238C3705D6
:1033F000A38C2705A38B9704F2406244D244424930
:10340000B249224A0561828041119397050122C485
:1034100006C626C2C1872E8463DC0700B7E4040019
:10342000FC54829719C1BC5482972165218D3DA01F
:1034300093F7150013C5150095E393F7250085C78D
:10344000FD35B7E70400BC4F1306000A8945170590
:1034500000200345A5EC829713452400B240224486
:103460009244410182809397250163D50702B7E416
:10347000040083A7C41E8297F53DBC4C37F60200BA
:10348000130606E0896517050020034525E98297A4
:10349000096569BF939715010145E3D107FC1775CD
:1034A000010013052516EF505114B7E70400BC4F77
:1034B00013060064916517050020034525E68297F1
:1034C0001165ADB72D71232A9110FD74E98C232C61
:1034D000811023282111232631112A84AE893289B3
:1034E000930600100A86A6852D45232E111097F00D
:1034F000FF1FE780400113154401B7E70400FC47B4
:1035000051810A0513962900CA850A958297A685D6
:1035100085660146254597F0FF1FE780C0FE0A86B5
:10352000A68593060010294597F0FF1FE780A0FDB0
:103530008320C11103248111832441110329011126
:103540008329C11015618280B7F7070003C70701FF
:10355000411106C622C426C24AC0A547631AF70015
:103560009537B2402244924402490145410182808C
:1035700013942500AA843289A286AA85014625458E
:1035800097F0FF1FE78020F8A2864A86A685294586
:1035900097F0FF1FE78020F7E9B71D71A2CC37E451
:1035A00004005C5C485886CE4946977501009385B7
:1035B000E500829701E91775010013056501EF50D9
:1035C000D10201A0B7F600E0795798CAFD57DCCACE
:1035D0000567B7E700E023A0E7101306F00290C2EA
:1035E00023A0E71801000100370700201847130641
:1035F000000481459706002023A0E6D24157A38A04
:10360000E7403C440808829797170020938787DE9D
:103610003EC8856713870760231AE1001D673ACC0F
:1036200037070105130707103ACE9387B7D313075F
:10363000B00F2310E1022312F102054797F7FFFFB5
:103640009387E7592301E1023ED8170700001307CB
:1036500007D397070000938747D4B7F50700BAC28E
:103660003EDC17070000130767EE970700009387FB
:10367000A7D081463000E1051945BAC43EDE97F077
:10368000FF1FE78040E818088147994630003E96C2
:103690000346060085070507A30BC700E398D7FE7E
:1036A000C24791C70357410185676373F70001A0C3
:1036B000B7E7040083A7470A08088297AA8501C9CB
:1036C00017750100130505F2EF50615D01A0F6408A
:1036D000664425618280411126C2B7E4040083A7B5
:1036E000040806C622C417050000130525D28297D8
:1036F00017040020130484C22300A4003128DD36FF
:1037000003450400224403A38405B24092441306F7
:103710000032896541010283797106D622D41307EC
:103720008008F337078093F787083EC20100010045
:10373000B7170040930570052380B704130680FA7D
:103740002380C7040100010083C6F70293F6A60F89
:10375000A387D702238007049246F3A606800100C0
:10376000010073370780137787083AC4010001000E
:103770002380B7042380C7040100010003C7F702B8
:1037800013672700A387E70223800704A247F3A754
:103790000780010001000545EFE0CFFCE13E014755
:1037A00081468147054685451305407EEFE07F80D1
:1037B00037E404003C446800514681458297B707CE
:1037C000C0A83EC8B787E803938707D03ECA97F7DB
:1037D000FF1F9387C7BD3EC67C5868008297B250D2
:1037E00022544561828041119775010093854551AE
:1037F00017750100130545D906C6EF50414A1775E4
:1038000001001305656AEF508149B2402945410125
:103810006F50214D4111977501009385A54F177584
:103820000100130565D606C6EF5061471775010004
:1038300013054566EF50A146B240294541016F503E
:10384000414A411122C406C6834705002A849DC30C
:10385000977501009385C551177501001305C5D2F1
:10386000EF50E1434C401775010013052578EF50E8
:1038700001431DA058411DE7977501009385454FF1
:1038800017750100130545D0EF5061411775010010
:1038900013054577EF50A1402244B240294541012C
:1038A0006F502144A1679386D7036311D7029775A0
:1038B00001009385E54B177501001305E5CCEF502A
:1038C000013E177501001305E574E9B7ED0797751B
:1038D00001009385E549177501001305E5CA6319D1
:1038E000F700EF50C13B177501001305E5735DB795
:1038F000EF50E13A4C40177501001305E57485BFA0
:103900004111977501009385254217750100130534
:10391000A5C706C6EF50A138B240294541016F50F6
:10392000413C797122D426D24AD02E842A898145FD
:10393000B2844800714606D6EFE02FC397F7FF1F09
:103940009387076BDC4783D70700231421012313D8
:10395000F100EF20D0029547A305F1009307401F27
:103960003EC6FD572305A100230AF100EF20701386
:103970002686A2854800EF207003B250225492544C
:10398000025945618280970700202392079C970780
:103990000020238D079AB7E70400BC47411106C6F3
:1039A000414681451385413D8297EF10B067EF1086
:1039B00010450145EF30601503C7C1259307F00A94
:1039C000631BF7009307F00889451385C125239EE3
:1039D000F124EF30E03FEF30C04F81453705040060
:1039E0009707002023A0079697070020239A0794A3
:1039F000970700202387079497070020239F0792AB
:103A000097070020239A079297070020239907928F
:103A100097070020239A0792EF20E0370145EF3007
:103A2000E041977501009385A532177501001305D4
:103A3000A5B5EF50C1261775010013052567EF5096
:103A40000126B240294541016F50A129411122C4EC
:103A500006C626C293F715002E84638D070C814697
:103A600017F6FF1F13064656854517050020035518
:103A7000658CEF80900A05C5977501009385052E2A
:103A800017750100130545B0EF506121177501004E
:103A9000130585CFEF50A1202945EF50812497755C
:103AA00001009385A52B177501001305E5ADEF50B7
:103AB000011F17750100130565CEEF50411E294502
:103AC000EF50212217F5FF1F130585525C4505476E
:103AD0002390E700EFF0C01A977501009385052841
:103AE00017750100130545AAEF50611B17750100FA
:103AF000130505CCEF50A11A2945EF50811E9307FD
:103B000010F8238EF1249707002083D76782A38EB5
:103B1000F1241385C125A1839145238FF124A38F1F
:103B20000124EF30E02A13451400B24022449244AD
:103B30004101828093F72500D1CB1707002003575E
:103B4000278051C397F6FF1F9386C67F94429777CD
:103B500001009387A75717F6FF1F0346867E81450E
:103B60001385413DEF40B008AA8431CD977501001F
:103B70009385852517750100130505A1EF502112C6
:103B8000A68517750100130525C4EF50411129457D
:103B9000EF50211597F7FF1F2394077A930710F82A
:103BA000238EF12497F7FF1F83D78778A38EF12404
:103BB000A183238FF12491458D471385C125A38FC0
:103BC000F124EF30E0201345240085B793F745003A
:103BD000B1CF977501009385251F17750100130557
:103BE000A59AEF50C10B177501001305A5BFEF5043
:103BF000010B2945EF50E10E930720F8238EF124A5
:103C000097F7FF1F83D76773A38EF124A183238FB8
:103C1000F1248547A38FF124EF20A0681385C125E7
:103C20009145EF30E01A1345440001B793F7850042
:103C30008DCF977501009385251917750100130520
:103C4000A594EF50C105177501001305E5BAEF50B3
:103C500001052945EF50E10897F7FF1F2392076EF2
:103C6000EF40D00513458400C9B593F70501A5C3FE
:103C7000854517F5FF1F0355456CEF00914F97756C
:103C8000010093856514177501001305E58FEF504A
:103C9000010117750100130565B7EF504100294573
:103CA000EF502104930730F8238EF12497F7FF1F7C
:103CB00083D7A768A38EF1241385C125A1838D45E1
:103CC000238FF124EF30C01013450401B9BD93F7E1
:103CD0000502B5C3977501009385050F177501009F
:103CE0001305858AEF40B17B17750100130545B4B4
:103CF000EF40F17A2945EF40D17E930740F8238EBB
:103D0000F12497F7FF1F83D72763A38EF124A183A4
:103D1000238FF1248547A38FF12497F7FF1F239D5D
:103D20000760EF2000581385C1259145EF30400A08
:103D300013450402DDBB93F70504CDC79775010059
:103D4000938585081775010013050584EF403175CB
:103D500017750100130545AFEF4071742945EF4019
:103D6000517883C7C1251307700A6388E7041307D6
:103D7000800A6386E7061307600A6397E7029307E2
:103D800060F8238EF12497F7FF1F83D7475BA38E3C
:103D9000F124A183238FF1248547A383F126B14524
:103DA0001385C125EF30C002EF20A04F1345040456
:103DB00097F7FF1F239507588DBB930770F8238E45
:103DC000F12497F7FF1F83D78757A38EF124A18390
:103DD000238FF1248547A380F1269945D1B7930716
:103DE00080F8F1BF93F705080145E38007D4977584
:103DF0000100938565FD176501001305E578EF4027
:103E0000116A177501001305A5A5EF4051692945F1
:103E1000EF40316D9307A0F8238EF12497F7FF1F31
:103E200083D78752A38EF124A183238FF124854762
:103E3000A38FF12497F7FF1F23980750EF206046C8
:103E40001385C1259145EF20B07813450408F1B9D9
:103E5000411122C4977501009385C5F22A84176524
:103E600001001305657206C6EF4071634C4017757B
:103E7000010013052515EF4091622945EF40716659
:103E8000034704009307F00F6319F70297750100C9
:103E9000938545EF176501001305056FEF4031600D
:103EA0004C40177501001305E512EF40515F2244A5
:103EB000B240294541016F40D162B24022444101E4
:103EC000828085CD411122C4176501001305C56BA1
:103ED0002E84977501009385E5E506C6EF40315CB9
:103EE000A285177501001305251AEF40515B224486
:103EF000B240294541016F40D15E8280411122C408
:103F000026C22E84AA8497750100938565E3176500
:103F100001001305656706C6EF407158177501006B
:103F200013054517EF40B1572945EF40915B977551
:103F300001009385E5E097F7FF1F239D973E1765E6
:103F4000010013056564854497F7FF1F2392873EA0
:103F500097F7FF1F239F973C97F7FF1F2399873EF3
:103F6000EF40F15397F5FF1F83D5653E17750100AC
:103F70001305C512EF40B1522945EF40915697F70E
:103F8000FF1F2385973CEF1080672285EF20F037D5
:103F90000545EF20B06A97F7FF1F93876705DC4759
:103FA00003D70700C167FD176312F7022244B7E782
:103FB0000400B240924403A3870517F5FF1F034591
:103FC00065361306000A854541010283B24022444A
:103FD000924441018280011122CC37E404005C5CF0
:103FE00006CE26CA354697750100938525ED1775CF
:103FF000010013056579829701E917650100130532
:10400000255DEF40915E01A097F7FF1F93874765FD
:104010003EC4B7F507008567938707C0814617F64A
:10402000FF1F13066630E10519453EC697E0FF1FE6
:10403000E780604D7C44194697F5FF1F9385C52E98
:10404000138581368297340017F6FF1F1306C62D9D
:104050009775010093850531177501001305053229
:10406000EF406011AA8415C9977501009385C5D4E6
:104070001765010013054551EF407142A68517757C
:1040800001001305A5E4EF4091412945EF4071453A
:10409000F2406244D24405618280EFA04028177547
:1040A00001001305A5D9EF30A02CEF708016EF00AA
:1040B000113517F5FF1F130565F0EF00F121177596
:1040C00001001305A5D8EF005135AA84EF30500741
:1040D000EFC0605AEF20B154EF407023EF3090668C
:1040E000EFE0503797750100938505CD1765010006
:1040F0001305854989C8EF40913AA68517750100D7
:10410000130505DF49B7EF40913917750100130515
:1041100065E0EF40D1382945EF40B13CEFE0F019C0
:10412000EFB020446305050E854537050400EF1008
:10413000904697750100938525C817650100130502
:10414000A544EF40D13517750100130525DEEF407A
:1041500011352945EF40F13897F7FF1F938787D92D
:1041600083D7070017F7FF1F2313F71E854717F79D
:10417000FF1F230DF71CEF10E065EF10404817F507
:10418000FF1F0355C51CEF20501897F7FF1F83C76B
:10419000D71BB9EFA303010083274417130671004F
:1041A0008545130550308297977501009385C5C0EA
:1041B000176501001305453DEF40712E177501008D
:1041C000130505D9EF40B12D2945EF409131977581
:1041D0000100938565BE176501001305E53AEF40C0
:1041E000112C177501001305A5DCEF40512B71BD93
:1041F00097750100938545BC176501001305C53807
:10420000EF40F12917750100130505D865BF9775B3
:104210000100938565BA176501001305E536EF4087
:10422000112817750100130565E8EF40512729454E
:10423000EF40312B0145EF20704051BF411122C4A6
:1042400037E404008327041A06C68297EF20B014CF
:104250008327040817F5FFFF1305857F829797F7DB
:10426000FF1F2381A70C17F5FF1F130565D8EF204B
:1042700020302244B2404101B9BB411122C49146D1
:104280002A84138601349D652D4506C697E0FF1FDD
:10429000E7806027B7F7070003C70701A547631347
:1042A000F70001A09306001001469D65254597E0A3
:1042B000FF1FE7804025238081342244B24091468D
:1042C000138601349D652945410117E3FF1F6700EF
:1042D0008323B7E704001171FC47CED79389C1252A
:1042E000A2DDCAD986DFA6DB2E8432892E86AA8576
:1042F0004E85829783C70900130780029387E707DB
:1043000093F7F70F636AF774176701001307C72F56
:104310008A07BA979C43BA9782878D4797750100A1
:104320009385C5AB1765010013050526630BF400E3
:10433000EF40F1161765010013050569EF403116CE
:10434000FDA2EF40D1151765010013056569EF4027
:1043500011152945EF40F118930720F81146938570
:10436000C1254A85238EF124A38F0124EFF06FDB52
:104370002A840DC597750100938545A61765010030
:1043800013058520EF40B111A285176501001305C3
:10439000E568EF40D1102945EF40B1149775010051
:1043A0009385C5A3176501001305051EEF40310F66
:1043B000176501001305C567EF40710E2945EF40F1
:1043C00051124165930730FA05469385C1257D1545
:1043D000238EF124EFF0EFD42A840DC597750100E8
:1043E0009385C59F176501001305051AEF40310B32
:1043F000A2851765010013056562EF40510A294542
:10440000EF40310EB7E70400BC4F0566130606C83F
:10441000A14517F5FF1F0345E5F08297FE506E5446
:10442000DE544E59BE591161828091476301F402F6
:10443000977501009385859A176501001305C514CA
:10444000EF40F105176501001305C561C5BDB7E76C
:104450000400FC4F914517F5FF1F0345A5EC82971B
:104460009775010093858597176501001305C511A0
:10447000EF40F1021765010013058560EF4031023E
:104480002945EF401106EF10D0619145E1A2854723
:104490006301F40297750100938545941765010047
:1044A0001305850EEF40A17F176501001305C55E5A
:1044B00071B597F7FF1F239227E9B7E70400056658
:1044C000BC4F130606C8C145A9B78D476301F40266
:1044D0009775010093858590176501001305C50A3E
:1044E000EF40E17B176501001305C55C81BD9307B3
:1044F00040F811469385C1254A85238EF124A38F68
:104500000124EFF00FC22A84E30A05F09775010039
:104510009385C58C1765010013050507EF402178C9
:10452000A285176501001305654FEF4041772945C6
:10453000EF40217BE5B59147E31CF4F8B7E70400B1
:10454000FC4F9305000217F5FF1F0345A5DD829779
:104550009775010093858588176501001305C502CD
:10456000EF40E173176501001305455601BF894708
:1045700063E1870297750100938545861765010001
:1045800013058500EF40A17117650100130545551E
:1045900075B383C4E12583C7D12597750100938541
:1045A000E583A20417650100130505FEDD8CEF40CD
:1045B000016FA285176501001305C553EF40216EF9
:1045C000C2042945EF40E171C1849305D4FF93965D
:1045D0000401C1824A8693F5F50F1385F125EF108A
:1045E000007FE35D90E2930750F8238EF12483C7A8
:1045F000390022869385C12585074A85A38FF1243A
:10460000EFF02FB22A84E30B05E097650100938554
:10461000E57C17650100130525F7EF404168A28589
:1046200017750100130545A509B7894763E187029E
:10463000976501009385857A176501001305C5F418
:10464000EF40E165176501001305854CC5B9EF1012
:104650005045A2851385C125EF208077C1B38D47D2
:104660006301F402976501009385457717650100A2
:10467000130585F1EF40A162176501001305054B95
:1046800075B9B76602000146B7750200054597E0A7
:10469000FF1FE78040E7930760F8238EF124A38F84
:1046A00001249307002623A0F126E57793870721AD
:1046B0002392F1263146A383A1269385C1254A85FD
:1046C00023830126EFF0EFA52A84E30905D497653B
:1046D00001009385A570176501001305E5EAEF4019
:1046E000015CA285176501001305C5453DBDB147B5
:1046F0006301F402976501009385456E176501001B
:10470000130585E8EF40A1591765010013054545DC
:1047100035B1B7E70400FC4F9305000417F5FF1F00
:10472000034545C08297EF10D037B14525B7914773
:1047300063E18702976501009385456A176501006B
:10474000130585E4EF40A1551765010013050543E6
:10475000F5B683C4012683C7F125A204DD8C8E043F
:10476000B77702006D14BE942286A68517650100F6
:1047700013050542EF40A152B7E70400FC4722862B
:10478000938511262800829793160401C182300078
:10479000A685094597E0FF1FE780E0D62A8419C562
:1047A0001765010013058540EF402164930770F8F9
:1047B00019469385C1254A85238EF124A38081263D
:1047C000EFF02F962A84E30B05C4976501009385CB
:1047D000E56017650100130525DBEF40414CA2851C
:1047E000176501001305853D89B399476301F410EE
:1047F000976501009385855E176501001305C5D88F
:10480000EF40E149176501001305C53C05BE91471E
:1048100063E18702976501009385455C1765010098
:10482000130585D6EF40A147176501001305053C28
:1048300031B683C4012683C7F125A204DD8C8E0422
:10484000B77702006D14BE942286A6851765010015
:104850001305053BEF40A144B7E70400FC4722865F
:10486000938511262800829793160401C182300097
:10487000A6850D4597E0FF1FE780E0C82A8419C58B
:104880001765010013058539EF402156930780F81D
:1048900019469385C1254A85238EF124A38081265C
:1048A000EFF02F882A84E30B05B697650100938506
:1048B000E55217650100130525CDEF40413EA28565
:1048C000176501001305C5368DB199476301F402E0
:1048D0009765010093858550176501001305C5CACA
:1048E000EF40E13B176501001305053681BCB7E7D2
:1048F0000400FC4F9305000417F5FF1F034585A234
:104900008297EF10101A9945B1B38D476301F402F5
:10491000976501009385854C176501001305C5C691
:10492000EF40E137176501001305853301BC1765BA
:1049300001001305E533EF40414B1305C01297E02A
:10494000FF1FE780409F0145EFE02FA60D45EFF0E8
:10495000DF92294597E0FF1FE780E09D97E0FF1F6A
:10496000E780008F65BC99476301F40297650100F9
:104970009385C54617650100130505C1EF40213237
:10498000176501001305852F55BA03C7112683C784
:10499000012622075D8F9166BA96C2061166C18212
:1049A0001306F6EF8D476363D60297E7FF1F9387E1
:1049B00027649C4B03C6F1259386C70039C603D6EE
:1049C00007005DCA8907E39CD7FE89471307A0F853
:1049D00011469385C1254A85238EE124A38FF124B6
:1049E000EFE03FF42A84E30B05A29765010093856D
:1049F000E53E17650100130525B9EF40412AA28560
:104A0000176501001305C5280DB603D6070063021C
:104A1000E60A8907E39BF6FE8D474DBF9147630287
:104A2000F402976501009385653B17650100130546
:104A3000A5B5EF40C126176501001305E5266FF007
:104A4000FF8FB7E70400FC4F9305000817F5FF1F21
:104A50000345458D829705BC976501009385053810
:104A600017650100130545B2EF406123176501008A
:104A7000130505256FF09F8C2390E70017E5FF1FB6
:104A800013050557EFE06021976501009385053513
:104A900017650100130545AFEF4061201765010060
:104AA00013050523EF40A11F2945EF4081238147CE
:104AB00031BF2390070017E5FF1F13056553EFE093
:104AC000C01D9765010093856531176501001305C9
:104AD000A5ABEF40C11C176501001305E520D9B750
:104AE000411122C406C6834705002A849DC39765E9
:104AF00001009385652A176501001305E5A8EF40BD
:104B0000011A4C40176501001305455DEF4021195E
:104B100075A05841B707CF009387777D6313F706D9
:104B20009765010093854527176501001305C5A505
:104B3000EF40E1161C448356E4008355C40003C6CD
:104B40000700176501001305E55AEF404115294597
:104B5000EF4021190357E40097E7FF1F83D7277F12
:104B60006307F7008355C4000844EFE0CF9703566E
:104B7000E4008355C40008442244B24041016FF070
:104B80004FF5B707CC009387777D631FF7029765D2
:104B9000010093856520176501001305E59EEF4030
:104BA00001101C448356E4008355C40003C607006B
:104BB0001765010013050554EF40610E2244B24011
:104BC000294541016F40E111B707CE009387777DFA
:104BD0006302F702976501009385051C17650100C4
:104BE0001305859AEF40A10B4C4017650100130592
:104BF000A54529BFB2402244410182805171CAD1EA
:104C000037E904008327C904A2D52E8686D7A6D308
:104C10002E84AA851385C125829783C7C1251307D2
:104C2000700A638DE70C636CF7001307600A6382F8
:104C3000E704BE502E549E540E596D6182801307B6
:104C4000800A6382E7121307900AE394E7FE8D4718
:104C5000630BF416976501009385051A176501002B
:104C600013058592EF40A10317650100130505AFF9
:104C700015A08D476306F402976501009385C5175B
:104C80001765010013054590EF40610117650100AC
:104C9000130505A6EF40A1002945EF40810451BF4F
:104CA000854717650100130565A617E7FF1F230752
:104CB000F768EF408113B7750200B766020001463E
:104CC000054597E0FF1FE7800084930760F8238E77
:104CD000F124A38F01249307002623A0F126E57772
:104CE000938707212392F126B14523830126A383CD
:104CF000A1261385C125EF20A00D25BF914763E1B3
:104D00008702976501009385250F1765010013053C
:104D1000A587EF30D17817650100130525A19DBF48
:104D200083C4012683C7F125A204DD8C8327C9042F
:104D30006D14228693851126280082978E0493167F
:104D40000401B7750200C1823000A695094597D0CD
:104D5000FF1FE780407B930770F8238EF12499456D
:104D6000A380A12679B7914763E187029765010087
:104D7000938585081765010013050581EF303172B1
:104D8000176501001305059C31B783C4012683C74D
:104D9000F125A204DD8C8327C9046D142286938536
:104DA0001126280082978E0493160401B77502001D
:104DB000C1823000A6950D4597D0FF1FE780A074F3
:104DC000930780F859BF176501001305659AEF40F6
:104DD000C1011305C01297D0FF1FE780C0550145E0
:104DE000EFD0BFDC0D45EFF04FC9294597D0FF1F2D
:104DF000E780605497D0FF1FE78080451DBDB7E76F
:104E000004004111FC4726C29384C1252E8606C6A4
:104E100022C44AC02E842A89AA852685829797654E
:104E20000100938525FF175501001305E575EF3047
:104E3000116783C5C125176501001305E5A3EF3090
:104E400011662945EF30F16983C704004147938714
:104E5000070693F7F70F6365F74817670100130715
:104E6000E7848A07BA979C43BA9782879D47630372
:104E7000F402976501009385E5F9175501001305C4
:104E8000A570EF30D161176501001305659FEF3004
:104E90001161D1A283C7D125ADCF83D7012603D716
:104EA000E125C207D98F17E7FF1F232DF74883C7D6
:104EB0006400976501009385E5F51755010013051A
:104EC000A56C17E7FF1F230EF746EF30515D97E7FC
:104ED000FF1F938727478C4317E6FF1F034666464D
:104EE000176501001305859BEF30715B2945EF3095
:104EF000515FA38E01242244B24092440249930799
:104F000000F8238EF1249D451385C12541016F10C2
:104F1000306CEF304066239FA124935705012A840B
:104F20002380F126935785010145A380F126EF30B8
:104F300040652381A126976501009385A5ED17554E
:104F4000010013056564EF30915503C62126A28543
:104F5000176501001305059641BFCD476301F402B3
:104F600097650100938505EB175501001305C56191
:104F7000EF30F152176501001305459509BF37E47D
:104F800004007C4441469385D1251385413D829799
:104F90001385413DEF00607D9D2583C7E12603C752
:104FA000D126A20703238405D98F17E7FF1F2319F2
:104FB000F7381306000A89452244B2409244024958
:104FC00017E5FF1F03450536410102838D47630145
:104FD000F402976501009385E5E317550100130579
:104FE000A55AEF30D14B176501001305E59D45B576
:104FF00003C4E12583C7D12597650100938585E129
:10500000220417550100130525585D8CEF303149F6
:10501000A285176501001305E58CEF30514829453D
:10502000EF30314C0D469385C1252285EFE07F8F0F
:10503000AA8415C9976501009385C5DD1755010040
:1050400013058554EF30B145A6851765010013059A
:10505000A58AEF30D1442244B24092440249294506
:1050600041016F30114897E7FF1F2398872CB7E75E
:105070000400116603A38705130606E891452DBFBA
:105080008D476301F402976501009385A5D81755F4
:1050900001001305654FEF309140176501001305BE
:1050A00065A1F5B303C4E12583C7D1259765010048
:1050B000938545D62204175501001305E54C5D8CF8
:1050C000EF30F13DA2851765010013052584EF300F
:1050D000113D2945EF30F1400D469385C1252285CC
:1050E000EFE03F84AA840DC197650100938585D2C6
:1050F0001755010013054549EF30713AA68517652C
:1051000001001305E581B1B797E7FF1F23968722BA
:10511000B7E70400116603A38705130606E89305A5
:10512000000259BD894763E18702976501009385B5
:1051300065CE1755010013052545EF30513617652B
:1051400001001305E599A1B383C4E12583C7D125E7
:1051500097650100938505CCA2041755010013053E
:10516000A542DD8CEF30B133A6851755010013053C
:10517000A57CEF30D1322945EF30B13622869385B8
:10518000C1252685EFE0EFF92A84630A05169765A5
:105190000100938525C8175501001305E53EEF3042
:1051A0001130A285175501001305457A5DB5854775
:1051B00063F78714834519002244B24092440249A0
:1051C000B335B00097E7FF1F238AB71617550100C4
:1051D0001305057941016F30912CA2852244B2401C
:1051E00092444A85024941016FF05FA199476301EA
:1051F000F402976501009385E5C117550100130579
:10520000A538EF30D12917650100130525A741B155
:1052100003C4E12583C7D12597650100938585BF28
:10522000220417550100130525365D8CEF30312718
:10523000A2851755010013052574EF305126294525
:10524000EF30312A19469385C1252285EFE06FEDB5
:10525000AA840DC1976501009385C5BB1755010050
:1052600013058532EF30B123A685175501001305CC
:10527000A571C5B397E7FF1F2398870CB7E7040014
:10528000116603A38705130606E8930500082DB3EE
:105290008547976501009385E5B71755010013050C
:1052A000A52E6309F400EF30911F17550100130577
:1052B000E56EF1BEEF30B11E175501001305856F85
:1052C000EF30F11D2945EF30D1212244B240924404
:1052D000024997E7FF1F2395070641016F30001E23
:1052E00097650100938505B3175501001305C5297E
:1052F000EF30F11A176501001305859C49BEB240D5
:1053000022449244024941018280411106C622C4CE
:10531000EFE02FE19377F50F95CB2A849765010095
:105320009385C5B01755010013050526EF303117D9
:105330009375F40F17650100130505D4EF3031168E
:105340002244B240294541016F30B119B240224494
:105350004101828001114EC697E6FF1F83D626FFCA
:10536000B28917E6FF1F035666F726CA4AC806CE5B
:1053700022CCAA842E89252397E7FF1F83C707FD28
:10538000A9CB03C4440083C734001765010013058B
:10539000A5DA22045D8CEF3091104A86A68522851D
:1053A000AD37638F090297E7FF1F83C707FA8DCBDD
:1053B0006308090297E7FF1F83C747F895E3624434
:1053C000F240B249CA8526854249D24405616F1030
:1053D0003020176501001305A5D6EF301121D1B794
:1053E000F2406244D2444249B24905618280834717
:1053F000550083454500176501001305A5D2A20796
:10540000DD8D6F30D109176501001305A5D06F3010
:10541000D11D8D4763F2B70A011126CA06CE22CCF0
:105420000344350097E4FF1F83C434F297650100FD
:105430009385C5D1B337800017E7FF1FA307F7F0A7
:1054400009C497650100938525D1176501001305EF
:1054500025D1EF30D10497E7FF1F83C717EF638390
:105460009700252C97E7FF1F83C737EE9DC385471D
:105470002306F100B7E7040083A7471770008545AE
:1054800013055030829717650100130565CEEF3084
:10549000D1159967938757EE2316F1006800854769
:1054A0009145A30781002307F100EF107012F2402D
:1054B0006244D244056182808280894763F2B708E2
:1054C000011122CC06CE26CA8344250085472A84B2
:1054D0006398F404914763F0B7040345450083479C
:1054E000340022055D8D97E7FF1F2399A7DE25294C
:1054F0009967938767EE2314F100834734002305EF
:105500009100A305F1008347440095452800230638
:10551000F100EF10F00BF2406244D244056182804A
:10552000FDF89967938767EE2314F10097E7FF1F53
:1055300083D7C7DAA305F10023050100A183F1B7E2
:1055400082800111996722CCD51717E4FF1F13043D
:10555000E4DF2314F1008347040026CA97E4FF1F09
:105560009384E4DE2305F10083D7040028009545E9
:10557000A305F100A18306CE2306F100EF1050052C
:1055800003D6040083450400176501001305C5BF59
:10559000EF30E170F2406244D244056182809D6741
:1055A0007971D9172316F10097E7FF1F83C707DA30
:1055B00006D62307F1009DCBB7E70400FC47414620
:1055C0009385413D1305F10082976800CD45EF10AA
:1055D000300097E5FF1F83C565D7176501001305E8
:1055E000A5BDEF30C16BB25045618280B7E70400C2
:1055F000BC47414681451305F1008297F9B7B7676B
:1056000002036971938757AA3EC48567938717D0B1
:105610002316F10097E7FF1F938747D383C707003F
:1056200023248112A30701002307F10097E7FF1F3E
:105630009387E7D183D7070037E4040023261112AC
:105640002318F10097E7FF1F938747C983D7070007
:10565000414648082319F1007C449385413D8297D7
:10566000F1452800ED2A2312A1027C442C002810C9
:10567000794682973C44130561041306900D8145D9
:10568000829730109305700F0145EFD09FB48320AF
:10569000C1120324811255618280B7C7A55A011136
:1056A0009387C7333EC497E7FF1F83C717CA3EC619
:1056B000B7F7070003C7070106CE22CCA54763133F
:1056C000F70001A01164930504F093060010014651
:1056D000254597D0FF1FE78000E33000930504F0D5
:1056E000A146294597D0FF1FE780E0E197E5FF1F1E
:1056F00083C5B5C5176501001305C5BCEF30215A38
:10570000F24062440561828001119165A14630003A
:10571000938505F02D4506CE97D0FF1FE780A0DECC
:105720002247B7C7A55A9387C7336312F702B2451A
:1057300017650100130545ACB335B00097E7FF1FAF
:10574000A385B7C0EF30A155F2400561828085473F
:10575000854517650100130565AC17E7FF1FA30614
:10576000F7BEEF30C153153FC5B7B7C7A55A79711A
:105770009387F7353EC6B7E70400FC47AA8506D6EF
:1057800022D4414608088297B7F7070003C70701EC
:10579000A5476313F70001A01164930504E893067D
:1057A00000100146254597D0FF1FE780C0D5700047
:1057B000930504E8D146294597D0FF1FE780A0D480
:1057C000176501001305C5B3EF302162B2502254B2
:1057D0004561828079719165D1467000938505E8B5
:1057E0002D4506D697D0FF1FE780E0D13247B7C7D7
:1057F000A55A9387F73517650100130525AA631E7F
:10580000F700B7E70400FC471385413D41460C080B
:10581000829717650100130565A6EF30015DB25050
:1058200045618280B7F7070003C70701A5476313E7
:10583000F70001A091654111930600100146938580
:1058400005E8254506C697D0FF1FE780C0CBB240CC
:10585000176501001305859841016F300159C16733
:1058600069768146FD170506139706014183636437
:10587000B7003E8582803307D50003470700B98F04
:10588000214713F81700858363050800B18FC2070D
:10589000C1837D171377F70F6DF78506F1B749C1FF
:1058A000A547054763FFB706834715000347050073
:1058B0003168A207D98F13978700A183D98FC207B8
:1058C000C1831308C8550547639D0705411106C6E6
:1058D00022C426C203442500914763FD8702930733
:1058E00054006399F502A301C50021822302C5007B
:1058F0009304340091C6A302D500A1822303D500EE
:105900002A84A685A93F26942300A4002181A30010
:10591000A4000147B240224492443A85410182806A
:1059200005473A858280B7C7A55A01119387E734A6
:105930003EC42AC6B7F7070003C7070106CE22CC2C
:1059400026CAA5476313F70001A091642A849385B2
:1059500004EE930600100146254597D0FF1FE7800F
:1059600080BA3000A146938504EE294597D0FF1FE9
:10597000E78060B9A285176501001305A596EF3091
:105980000132EFF0DFC7F2406244D2440561828009
:1059900001119165A1463000938505EE2D4506CE97
:1059A00097D0FF1FE78020B62247B7C7A55A938735
:1059B000E7346314F702B245176501001305058843
:1059C00097E7FF1F239CB790C205C181EF30212DBF
:1059D000EFF0FFC2F24005618280D147D1451765E3
:1059E00001001305A58717E7FF1F2319F78EEF3076
:1059F000012B17E5FF1F0355658E3537E1BF0111F8
:105A000026CA06CE22CC93F71500AE848DCBAD67A7
:105A1000371700409387A7AA1CC3B7E70400BC4F01
:105A200013060019854517E5FF1F0345058B82976F
:105A300013C51400F2406244D2440561828093F79A
:105A4000250063830712976501009385658F2D46B6
:105A50004800EF30611997E5FF1F83C5358F8547F3
:105A600093C4240063E1B70489CD97E7FF1F83C780
:105A7000C78D85C38545170500201305A5F7EF10D1
:105A800020351395040197E7FF1FA381078C4181FF
:105A900055B741650546970500209385A5F57D1509
:105AA000EFF0BF86F9BF170400200344A4F4970762
:105AB000002083C737F422045D8CAD679387B75508
:105AC0006306F40863E68702A9679387A755630610
:105AD000F40897E7FF1F83C747878DE741652E8648
:105AE0007D15970500209385E5F0EFF01F82B9A0A2
:105AF000B1679387C755630EF400B5679387D75591
:105B0000E319F4FC170500201305C5EEEF10402C37
:105B100035A00546170500201305C5EDEFF09F835E
:105B200097E7FF1F83C7878291EB4800EF3021344E
:105B300093150501C1814800EFD0EF9AA285175552
:105B400001001305E57DEF30811525BF1705002005
:105B5000130545EAEFF0BF89D5B7170500201305F7
:105B600065E9EFF05F8AD9BF93F745000145E3830C
:105B700007EC175501001305E57BEF300127EF1007
:105B8000003713C544007DB5411122C437E4040039
:105B90005C5C06C63546975501009385253217652E
:105BA0000100130565BE829701E917550100130531
:105BB000E579EF30812301A08327041C82972A8492
:105BC0000545EF802075EF10C168EF100147EF70B9
:105BD000B0292285B2402244410182801567B7175F
:105BE00000401307575598C3D8439D66558FD8C3B7
:105BF000D843FD76758FD8C3D8431367F70FD8C342
:105C000035671307C7CC98C3828041111305800400
:105C100006C622C426C24AC097C0FF1FE78020499B
:105C200085457D55EFC0BFDF85457D55EFC09FE9B8
:105C3000371400408327840A8D451305002093E71D
:105C400007202324F40AEFC09FDDB7E40400EFD05F
:105C50000F8FC8581309840C1304C40CEF30E118DB
:105C600017650100130545B2EF3021188327C4FFE3
:105C70008545414593E70708232EF4FEEFC09FE4D6
:105C80008D4513050008EFC0FFE3EFC07FFE01451F
:105C9000EFD02F8185450545894717D7FF1F230979
:105CA000F76AEFD0AF8137070004B7E700E023A021
:105CB000E710EFD09F8EEFD01FA2F935EFF0DFA4F1
:105CC000EFF01FCDEFE08FD78D450D65EFC09FDF63
:105CD00017050020130505E285671CC58967232089
:105CE000250140C12326250100C95CC983A7841E64
:105CF000829783A7040817050000130585D08297B3
:105D000097D7FF1F238BA75CBC4C13060064854507
:105D10008297E93597C0FF1FE780806C014582803C
:105D2000B7F7070003C70701A547AE866316F7005C
:105D30009397450191C301A0AA850146254517C344
:105D4000FF1F6700437C4111B2862E86AA852D4530
:105D500006C697C0FF1FE780007BB24001454101A6
:105D600082809307000463E6C7021D71A2CC2A84D7
:105D7000080886CE32C6EF203167B2461008A285E9
:105D8000294597C0FF1FE7800078F64066442561EB
:105D9000828039558280411126C2AE848D4522C44D
:105DA00006C62A84EFC01FD2B717004099C803A5C2
:105DB000C70C418D23A6A70CB24022449244410156
:105DC000828003A5870C418D23A4A70CF5B78347D8
:105DD000050003471500A207D98FC2076177C18765
:105DE000130727206397E700834525003705040044
:105DF0005DB7828097D7FF1F9387C75518429C4392
:105E000083D645000345070083C5C70003564600F7
:105E10006396A50083D5E700638DD502011106CEF8
:105E20002386A7002397D700B705CF00DC4B9385C7
:105E3000757D05077D162EC2230001003AC4231686
:105E4000C1002317D10099C30A858297F2400561EA
:105E500082808280DC4DDC4B81CFB7E70400904527
:105E600003A38705914517D5FF1F0345E54E028320
:105E700082806D713C083EC6B707E5002322911071
:105E80003EC8AA843C083285232611103ECA23242A
:105E90008110232021112E89EF2090672A849755A5
:105EA00001009385E552174501001305E56DEF20CC
:105EB000115FA2851755010013058561EF20315E42
:105EC0002945EF201162B705CB009385757D6800E9
:105ED000EF10A043A2856800EF20305901478146AA
:105EE0007000CA852685EF10C06215C52A849755B3
:105EF00001009385E54D174501001305E568EF2086
:105F0000115AA285175501001305455DEF2031593F
:105F10002945EF20115D8320C110032481108324C3
:105F20004110032901105161828097D7FF1F938789
:105F3000674218429C43797122D406D60348070071
:105F400083C807012A8483D645000355460063961B
:105F5000080183D82701638DD8022388070105072C
:105F60002399D7003708CC00DC4B1308787D3ACC56
:105F70001307F5FF42CA23080100231EE100231F77
:105F8000D10099C7080832C62EC482973246A2456E
:105F90002285C535B2502254456182806D713C081E
:105FA0003EC0B707E5003EC23C083EC423261110A0
:105FB00023248110232291102317010023180100AC
:105FC00023190100231A0100231B010097D7FF1F8B
:105FD00083D7070699E3C167FD172316F10097D70A
:105FE000FF1F83D7070591EB97D7FF1F938787364E
:105FF0009C439C43DC4783D7070017D4FF1F13043F
:106000002403584C2317F10083574400484B2318AE
:10601000F10005ED97550100938585421745010074
:1060200013058556EF20B14717550100130585422A
:10603000EF20F1462945EF20D14A8320C1100324E7
:106040008110832441105161828097D7FF1F83C73D
:1060500097FE89EBB7E70400BC5782975C4C23AAF4
:106060000700E1BFFD1797D6FF1FA386F6FC035676
:106070000701834704014C470A85230BF100EF20F9
:10608000F03C97D7FF1F9387E72C9C43014781463D
:1060900088430A866C00EF10C047AA841DC9975533
:1060A00001009385E539174501001305E54DEF2003
:1060B000113FA685175501001305853AEF20313EA3
:1060C0002945EF201142584CB7E70400BC57484B14
:1060D00069B797D7FF1F83C717F6F5D7B7E704004F
:1060E000BC4F1044854517D5FF1F0345E526829711
:1060F000A9B75C4EDC4BA9CBA1C9411122C41745FD
:106100000100130565482E8497550100938585315C
:1061100006C6EF20D138A285175501001305853634
:10612000EF20F1372945EF20D13BB7E704002244A7
:10613000B24003A3870517D5FF1F0345E5211306CA
:1061400040069145410102838280411122C417D447
:10615000FF1F1304E4EB1C4C06C689C7DC4399C33C
:106160004C488297584CB7E70400BC57484B82977D
:106170005C4CB240224423AA07004101828017D719
:10618000FF1F1307C715834707009306F00B85070A
:1061900093F7F70F63E9F60097D6FF1F2381F614F4
:1061A000034507008280930700F8FDB78357450039
:1061B0006386070E01114AC817D9FF1F130949E763
:1061C00052C4032AC90106CE22CC03274A0126CA9B
:1061D0004EC656C2F15721EF1307D00DFD57636825
:1061E000C704B7E9040083A709072A8413058600BA
:1061F00042054181B284AE8A8297232AAA000325F0
:10620000C9015C499DEF975501009385A51F17456E
:10621000010013056537EF2091281755010013057C
:10622000A52EEF20D1272945EF20B12BDD57F240D5
:106230006244D2444249B249224A924A3E850561AB
:10624000828093874400B705CF002319F50093851A
:10625000757D3105EF10600B0325C901834564008E
:106260003105EF2090200325C9012686D68531050A
:10627000EF20D01D7146A2854A85EF20F1165044CB
:1062800019CA83A78905854517D5FF1F0345C50C86
:106290008297814769BFEFF07FD0E5BFFD573E850C
:1062A0008280411126C297D4FF1F938464D8D84CB2
:1062B00022C437E404003C54484B06C68297DC4CA9
:1062C0000323C4052244B240924423AA070017D5F1
:1062D000FF1F03456508854541010283411126C220
:1062E00097D4FF1F938404079C4006C622C44AC06B
:1062F000C9CBDC43D9C75CC12300B5002A849755BC
:1063000001009385650B174501001305E527EF2074
:1063100011192945EF20F11C9C4023A4070023A25A
:10632000070097D7FF1F9387A7CEDC4FDC4B81C7B1
:106330002955EFF09FE197D7FF1F938767CFDC4F79
:10634000DC4B91C3B93F37E904008327C905894570
:1063500017D5FF1F0345450082978327C90591453F
:1063600017D5FF1F034545FF82979C4003A34701B4
:106370006309030022852244B2409244024941014C
:106380000283B240224492440249410182800111B9
:10639000328506CE22CC26CA2E84EF207017AA841E
:1063A0009755010093858504174501001305C51D08
:1063B000EF20F10E03078400035664008355440068
:1063C000A686175501001305E50DEF20510D29454F
:1063D000EF20311197D7FF1F83C7E7C3639897005A
:1063E0000145EFF09FD681450A85CD3DF2406244DC
:1063F000D244056182806D712324811023261110FF
:106400002322911093F745002E84638507123C08E0
:106410003EC0B707E5003EC23C083EC4231701005A
:106420002318010023190100231A0100231B010076
:1064300097D7FF1F83D7C7BD99E3C167FD17231601
:10644000F10097D7FF1F83D7C7BC91EB97D7FF1FEA
:10645000938747F09C439C43DC4783D7070017D7BB
:10646000FF1F1307E7BA2317F100544F8357470064
:106470002318F100DC4A95EF97550100938545FB01
:106480001745010013054510EF2071011755010054
:10649000130545FCEF20B1002945EF209104134579
:1064A00044008320C11003248110832441105161D2
:1064B000828097D7FF1F83C717B62555ADCBFD1731
:1064C00017D6FF1FA309F6B403D6060183470701B9
:1064D000CC460A85230BF100EF20407797D7FF1FAA
:1064E000938747E79C4317D7FF1F130767B2976649
:1064F00001009386A6C888430A866C00EF106001ED
:10650000AA8451DD97550100938585F21745010056
:1065100013058507EF20A178A685175501001305FF
:1065200025F4EF20C1772945EF20A17B2685EFF0E8
:10653000DFC1B5B793F725009DC3B7E70400BC479B
:1065400041468145280882972555EFF01FC028084D
:106550009305F00FEFF09FD81345240099B793F7F8
:10656000150001459DDFEFF07FA31345140015BF13
:106570005C4D411106C688C317D7FF1F232CF7DCDB
:10658000B7E7040083A70708170500001305E5E631
:106590008297B24097D7FF1F2380A7DC01454101B6
:1065A000828001119307700F2316F10006CE97D752
:1065B000FF1F83C737DB8DE7B7E7040083A7870D8D
:1065C00017D6FF1F034606D26C0017D5FF1F0355D1
:1065D000A5D982973335A00097D7FF1FA384A7D8EA
:1065E000F2400561828041119397050122C406C6DD
:1065F00026C2C1872E8463D40702B7E40400FC548A
:1066000017D5FF1F034505CE829719C1BC54829749
:106610002165218DB240224492444101828093F74A
:1066200015008DC7B7E7040083A7471A17D6FF1FC9
:10663000130606A297F5FF1F9385C55017D5FF1FB8
:10664000034545CA829713451400E9B793F725001F
:1066500099CFB7E70400BC4F13060064894517D5EE
:10666000FF1F034525C882971345240065B793F79C
:1066700085009DC7B7E7040003A8871A1307401FCA
:1066800097D7FF1F83C707C6814613064006994563
:1066900017D5FF1F035545CD0298134584009DBFB4
:1066A00093F745000145BDD7B7E4040083A704185C
:1066B00017D5FF1F035545CB8297BC4C13060064CA
:1066C000914517D5FF1F0345E5C182971345440047
:1066D00091B797D7FF1F83D727C96396A70217D70C
:1066E000FF1F2314B7C817D7FF1F2311C7C817D719
:1066F000FF1F231ED7C62E8617550100130585F6EA
:10670000BE856F20C15917550100130525F76F206D
:10671000C16D03574500011106CE22CC97D7FF1F4C
:1067200083D787C417550100130545F56310F70695
:10673000C167F91717D7FF1F2328F7C237E40400F2
:1067400097D7FF1F23A407C27C4C894517D5FF1F8D
:10675000034545B982977C4C914517D5FF1F0345EA
:1067600065B8829797D7FF1F83C737BE95C7854700
:10677000A307F100832744171306F100854513058D
:1067800050308297175501001305C5E4EF20E165ED
:10679000F24062440561828097D7FF1F83C707BB21
:1067A000175501001305C5E7F5F38547A307F10069
:1067B000832744171306F10085451305503082974F
:1067C00017550100130545E3D1B77D15954763E0E3
:1067D000A71A175701001307A7DC0A053A951C41B1
:1067E000011122CC06CE26CABA972E84828717556D
:1067F0000100130525E9EF20415F0DA203C7250025
:106800009947631DF7002E85EFF0BFF083456400C4
:1068100017550100130505E8EF20614897D7FF1FC2
:10682000238507B217550100130585E8E9B703C7AB
:10683000250095476317F702C16717D7FF1F035756
:10684000A7B2F91703D5A5006307F702B7E704005D
:1068500083A7C717829717550100130565E6EF2038
:10686000C158854717D7FF1F2301F7AE1755010001
:10687000130585E749B797D7FF1F2397A7AE83D79F
:10688000E500B7E40400096617D7FF1F231FF7AC24
:1068900083D705011306069017D5FF1F034585A46E
:1068A00017D7FF1F2314F7AC83D72501A14517D7AE
:1068B000FF1F231EF7AABC4C8297BC4C1306006432
:1068C000914517D5FF1F0345E5A182970356E400C4
:1068D0008355A400175501001305C5DFEF20213CA7
:1068E00049B7175501001305E5E031B783C5250009
:1068F0009147639AF502854717550100130505E195
:10690000A307F100EF20614EB7E7040083A7471704
:106910001306F1008545130550308297F24062441A
:10692000D244056182809947639EF5002285EFF08D
:106930005FDE83456400175501001305A5D5EF20E0
:106940000136E9BF9547639FF5008347140017554B
:1069500001001305A5DBE39007EA175501001305B5
:10696000A5DC51BD17550100130585DCC9BF828028
:106970006D7123248110232611102322911032845B
:1069800001CD89476306F5028320C11003248110DD
:10699000832441105161828017550100130505DAE7
:1069A000AE84EF208144A2852685EFE04FC5E9BF84
:1069B000B7E70400FC47280082971755010013052C
:1069C000A5D8EF2081428347810039C01307000B0F
:1069D000638EE7001387A7051377F70F8D4663E9EA
:1069E000E602A2852800EFE06FA179BF8547E3FDAD
:1069F00087F88345910017450100130565F6B33507
:106A0000B00097D7FF1F238BB792EF204129ADBF6E
:106A100003479100A207D98F35671307D755638DB8
:106A2000E7066366F7022D671307B7556381E7062C
:106A300031671307C7556386E70429671307A7550E
:106A40006392E702A2852800EFE0FF9B35BF39671C
:106A50009306E7656383D70663E9F6001307E755F6
:106A60006388E704A285280089B73D679306F75538
:106A7000638AD7041307F766E396E7FEEFE03FB2B9
:106A800021B70146A2852800EFE0DF8CF5BDA28585
:106A90002800EFE0DF95CDBD8947E3F787EE93054A
:106AA000E4FFC205C1811305A100EFC0CFA3E9BD7A
:106AB000A2852800EFE0FF95C1BDA2852800EFE088
:106AC000DF9FD9B5EFE0FFA7C1B5411122C417C4BC
:106AD000FF1F1304A459AA86175601001306C6AD5A
:106AE0002285C14506C6EF2041310357440097C7B0
:106AF000FF1F9387A7582393E7000357640023944D
:106B0000E700B240224441018280011106CE22CC2E
:106B10006D3F37E404008327841417C6FF1F130654
:106B2000E654D54501458297832784179305F100E4
:106B30001305503082978347F100A1C7A3070100D6
:106B4000832744171306F1008545130550308297BB
:106B50008327441717C6FF1F13064652CD4513055A
:106B6000703082978547A307F100832744171306E7
:106B7000F1008545130550308297F240624405616B
:106B800082808327441717C6FF1F1306264FCD4563
:106B900013057030D5B7130101DE232C812037E4B3
:106BA000040083270408232E1120232A9120232860
:106BB00021212326312117050000130505A3829703
:106BC00017C9FF1F13090972994785442300A900BB
:106BD0002318F10097550100938505A793074006F8
:106BE000174501001305459A2314F1102304910061
:106BF00097C9FF1F9389A975EF20610A83D5090002
:106C0000175501001305059CEF2061092945EF2068
:106C1000410D03D50900EFF05FEB832744173000E7
:106C200085451305503082978327441717C6FF1FE9
:106C30001306C644CD451305703082978327441749
:106C400017C6FF1F13068641B545130560308297AE
:106C5000832744171008894513051031829783272D
:106C60004417300289451305203182978327441544
:106C7000930500050D45829783274415930500056C
:106C800011458297A30191002302910023049100F2
:106C90002324011023080100832784163002914524
:106CA00013057040829783278416130631008545AB
:106CB00013050040829783278416500085451305ED
:106CC00010408297832784161008854513052040BD
:106CD000829783278416300085451305504082979C
:106CE000832704157D558297832744137D5582970A
:106CF0007D55EFC0EFC68327440C8297EFC02FA4C9
:106D00008327841417C6FF1F13064636D545014551
:106D1000829789471306700F814508082302F10006
:106D2000EFB0AF848D471306700F8145280223080A
:106D3000F100EFB08F8391472304F11097C7FF1F35
:106D40009387C75A984383C747003AC42306F10084
:106D5000EFE0FF8A500085450545EFC08FC710085A
:106D60009305700F0945EFC0CFC630029305700F31
:106D70000D45EFC00FC6300095451145EFC06FC5FA
:106D8000C16717C7FF1F1307275EF9171CC323220C
:106D9000070017C5FF1F1305A554EFC06FC2832757
:106DA000C41D17C5FF1F1305655B82973C4803454B
:106DB0000900854582978320C121032481218324F2
:106DC0004121032901218329C1201301012282804D
:106DD0000111C16726CA06CEAA8422CC17C5FF1F9F
:106DE00003558558F9176306F50437E40400832733
:106DF00084122E862315B10001478146ED45829706
:106E00007C440356A1002AC6A68582972C0017C58C
:106E1000FF1F03556555EFC06FC701CD1755010022
:106E200013058583EF10717C8327C412ED4528007C
:106E30008297F2406244D24405618280011106CEFD
:106E400022CC2DC9854717C7FF1FA30EF72097C770
:106E5000FF1F238B072037E4040083278417930543
:106E6000F1001305503082978347F100A9CBA307A7
:106E70000100832744171306F100854513055030A0
:106E800082978327441717C6FF1F1306261DB54593
:106E90001305603082978547A307F10083274417C5
:106EA0001306F1008545130550308297F240624485
:106EB0000561828097C7FF1FA387071A49BF8327F1
:106EC000441717C6FF1F13066619B5451305603032
:106ED000E9BFC16717C5FF1F03550549F9176307C8
:106EE000F500B7E7040003A3C717028382800111EE
:106EF0008547A307010017C7FF1F2305F746B7E71C
:106F0000040083A7471706CE1306F1008545130535
:106F100050308297F24005618280EFA27FE02A84A0
:106F200008452E89B28909C900C1970500009385DB
:106F3000C5746105EF00810181447D5AEF10C009DD
:106F400063C3A4048144EF10200A63C6A40497F726
:106F5000FF1F9387E7BF9C43DC47B307F940918746
:106F60002302F400638109048327C900B307F440B6
:106F70009587A302F4001C4C89C79C4799C32285BE
:106F800082976FA03FDD5C44139714008504BA9785
:106F90002390470165B71C48139714008504BA97DE
:106FA000239007004DB7832789000547B307F440B6
:106FB0009587A302F40083570400638EE7028DC314
:106FC00009476384E7040D47E397E7FA9757010001
:106FD000938747CA1CCC975701009387A7CA11A86B
:106FE00097570100938787901CCC97570100938790
:106FF000E7905CC849B7974701009387277C1CCC72
:10700000974701009387877CEDB7975701009387D7
:1070100027CB1CCC97570100938787CBD9BF85E13D
:10702000EFA2BFD1004618448347940075839D8B1F
:107030006315F700EF00501C48C46FA05FD2828038
:10704000EFA21FCE13893500C16442094111AA89FC
:107050000144F11413590901054A2EC6EF00D077F7
:10706000B2456346A400014541016FA0BFCE83A78E
:10707000090013171400BA9783D707006388B70075
:107080006394970063742A010504C1BF0545E9BFF5
:10709000EFA23FC8AA892E89328BB6843A8ABE8A6B
:1070A000EF80204C55C12685EF1030368D4763E5C3
:1070B000A7007D556FA07FC983DB4400EF00D07728
:1070C0002A84EF00B07893077400314433058502B9
:1070D00063C5A702EF005076EF0010762A84EF0018
:1070E000F0769307740031443305850263CDA7021F
:1070F000EF0090749307450019A8EF003075330531
:1071000085021307F0179307C017E357A7FC2D5507
:10711000E3C277FB63000B02D6865286A6854A85BA
:10712000EFE0106341BFEF007072330585029307F3
:10713000C5FFF1BF832749001385C90083D5270008
:10714000EFF01FF071F9B5B76955ADB797F7FF1FAD
:107150002392A7A097F7FF1F9387879F90438147AC
:107160000C463307F500420741836393B7008280E2
:107170005446139847008507C2962390E600D5B77A
:1071800097F7FF1F9387C79C9C4303C587008280A6
:1071900017F5FF1F0355059C8280EFA21FBAC16738
:1071A0001387D7FF6307E5026368A700F117630E33
:1071B000F50001456FA0BFBA1387E7FF630EE50036
:1071C000FD171D8D13351500F5B7EF40003D7D15FA
:1071D000D5BFEF40801AE5BFEF40E018CDBFEFA26A
:1071E000DFB54111AA8401442EC6EF00F05FB2451D
:1071F0006346A400014541016FA07FB69C4813156A
:1072000014003E9583570500E387B7FE0504E9BFE8
:1072100003485500814693F7F60F63E50701814760
:107220003E858280584593975600BA9703D727002A
:107230006316B70003D70700E304C7FE8506E1BF66
:107240008346450001479377F70F63E4D7008147F2
:1072500011A81C45131657000507B29703D607005F
:10726000E313B6FE3E858280EFA29FAB9317050124
:10727000C18797FAFF1F938AAA8D6355F00883A7E9
:107280000A00C0479C4703570400198D42054181FD
:107290006366F500014422856FA0DFAB12052A94D6
:1072A000DDBFDC4713944900014A3E948347440004
:1072B0006341FA02014A834754006347FA02850991
:1072C000C20993D9090183A70A009847E3EBE9FCB7
:1072D000D1B71C4413195A00A6853E994A85EFF090
:1072E0001FF011ED050AD9B75C4413195A00A685A1
:1072F0003E994A85EFF0BFEE19E1050A6DBFE30044
:1073000009FC51BFAA8481497DBFEFA21FA31C4580
:107310002A8481E79307C5001CC51C44231204007E
:107320001CC09307F00F63E9B70093F5F50F2285B2
:10733000EF10B0136FA0BFA293940501C167C18085
:1073400063F7F500A6852285EF10D015E5B7C1815A
:1073500093F5F50F2285EF105011A6852285EF10C9
:107360001012C9BF97E7FF1F9387877E88438280EB
:107370001C4599C797E7FF1F23ACA77C0145828076
:107380007D55828097E7FF1F9387877C98438347CB
:107390004500484792073E958280EFA21F9A61718F
:1073A00000451C183EC6B70780013EC81C183ECADF
:1073B0008357440002CE02D002CC231EF100834743
:1073C00084002A8902D22301F1023C083ED402D66D
:1073D000EFF05FFB835705002316F102EF30706B6F
:1073E0002307A1025C4003556400F18313F71700E3
:1073F0008347F10252055181F99BD98FA307F1020E
:10740000EFE0702639C5AA8403550500EF804016C9
:1074100083D704002AD26800231CF10083D72400FC
:10742000231DF1001C4803D647008C43EF101002C7
:107430008347B400CA86174601001306A631811798
:10744000A305F4006C004810EFE090305D616FA080
:107450001F912155E5BF1C45B1CF03C5A700894643
:1074600013576500630BD7028D46630ED70285461E
:107470006300D702130740063305E50203C7B700D0
:10748000418B15CB83C7B700BD8B3355F540828048
:107490001375F5031307803EC5B709671375F50328
:1074A00013070771D1BF372709001375F5031307B9
:1074B000077CD9B701458280EFA23F8803A98500E8
:1074C000630509048347B900AE8493F7070E91CF93
:1074D00003459900930520030D810505B305B50209
:1074E00088446105EFF0B0320DA02E85EFF0BFF6B5
:1074F0002A8401CD11238325C900B307B54063F861
:1075000087002E94B305A440E1FD6FA05F858545FB
:10751000C1BFEFA29F822A8403D50500011132C6A4
:1075200036C43AC22EC002CA02CC02CEEF8040045A
:1075300082452ACA22852ECCEFF0DFE403570500EE
:10754000231EE100EF30F054A24632469247230F4B
:10755000A10036874C08B28622850146EFF05FB362
:1075600005616FA0CFFFEFA24FFD61711C183EC6F1
:10757000B70780013EC81C183ECA3C0800453ED4EF
:10758000AA8402CC02CE02D002D202D6EFF09FDF54
:107590008357050035592316F102EF30904F23072A
:1075A000A10209C48357440091E721594A855D61CE
:1075B0006FA0EFFA0355640052055181EFE0B00A65
:1075C0002A8965D58347B40093F7070E89C7130549
:1075D0008401EFF0502583574400231EF1008347B8
:1075E00084002301F1025C4003550900D98313F79D
:1075F000070883471102231CA10093F7F707D98FCF
:10760000A300F10283572900231DF1005C40F183A0
:1076100013F717008347F102F99BD98FA307F102F3
:10762000EF7010752AD251D18347940068001397E8
:1076300057008347B400FD8BD98FA305F4001C4885
:1076400003D647008C43EF106060A6871747010000
:1076500013074710740005464C102685EFF05FA312
:107660002A8929D58347B400A685FD8BA305F4009C
:10767000EFF09FE425BFEFA24FEC832485FE2A8420
:1076800041112685EFF03FDD834734FF93F7070E66
:107690009DC32AC62685EFF05FD019C9834734FF02
:1076A000B245FD8BA309F4FE81C52285EFF03016AB
:1076B00041016FA0CFEA6DDD8327C4FF2685829745
:1076C00065F9834734FF93F7070E81C72285EFF0F2
:1076D0009015032584FEEFF01FE9D9BFEFA2EFE27A
:1076E0009C4141112A8903C7070089472E8493567C
:1076F0006700638CF6020D466382C6049307F007A9
:107700006302F7022E85EF10A060AA848149C16B45
:10771000130C490097E7FF1F938787439C439847C3
:1077200063ECE90241016FA00FE203D745008547F2
:10773000E3FAE7FE2E85EF108061C1BF03D7450055
:10774000E3F2E7FE2E85EF10A05CAA842285EF10FD
:10775000805DC204C98C5DBFDC470355A900139A44
:1077600049003E9A93170501C187635DF000835776
:107770000A006395A70263E574038327CA00034DDB
:107780005A001DA0A1672167A98F1307F7EFE374C3
:10779000F7FE63950900EFF05FA071FD85099DBFBD
:1077A00083278A00034D4A00835DA90003576900BF
:1077B000216A138BC7003AC6814A33CA4D01631E42
:1077C0005D0197E7FF1F938727399C43E1DBA28682
:1077D0006286814526858297D1B7A1679387F7EFA7
:1077E000930C4BFF63F04703B2455A85EFF05F857A
:1077F00019CD03278B00104719CA10436380C402B8
:107800003107D5BFEE856685EFF07F9D71FD9386CC
:107810001A0093FAF60F130B0B0255B78356440068
:107820005C43E3EDF6F622853AC6EF10603DA167B2
:107830009387D7042A8A035D4400324763E89700A0
:107840008347D90093E707F8A306F9001C4766852C
:107850002286E2858297C1670844FD17337AFA00D1
:10786000529508C02312A40115BF97E7FF1F938705
:10787000272E9843814715C31447814763FFD500DE
:10788000939745004C47BE9519C903C755008147DA
:107890006375E600DC451606B2973E85828003C715
:1078A00045008147E37BE6FE16069C45F5B7EFA24F
:1078B0002FC7AA892E8A814497EAFF1F938A4A29F3
:1078C00083A70A00984763E4E4006FA0AFC8DC47D1
:1078D0001394440001493E9413BB140083474400B1
:1078E000634BF900014913BB140083475400634FF5
:1078F000F9008504F1B70844931759005287DA86D6
:107900000146A2853E9582990509C9BF484493174F
:1079100059005287DA860546A2853E958299050967
:10792000E9B7EFA28FC1814517F5FFFF1305255F6A
:1079300097E7FF1F23900722EFF07FF76FA02FC27A
:1079400097E7FF1F9387C7209C4381CFEFA2EFBE2D
:10795000814517F5FFFF1305855CEFF05FF56FA01C
:107960000FC08280EFA2CFBB37E4040083278412CC
:1079700041112315E100AE893289368A3A86814663
:107980000147ED45AA8482972AC621C50356A10066
:10799000D285EF1061258327C413CE852685829773
:1079A000058915C58327440D2314210101462C00A8
:1079B000268582972A8401C9B7E7040083A7C712E6
:1079C000ED4528008297228541016FA0AFB8494458
:1079D000E5B76554CDBF5C41FD175CC18280EFA265
:1079E000CFB5B7E70400FC5F829795473305F502F2
:1079F00081450D816FA0AFB6EFA22FB4B7E70400A9
:107A0000FC5F829795473305F5020D816FA02FB576
:107A1000EFA2AFB2B7E7040083A7870B03550500B9
:107A200082976FA0CFB3EFA24FB103550500328705
:107A3000AE8617B6FF1F0356866A97E5FF1F93852C
:107A4000E511EFF03FF26FA08FB1EFA20FAFB7E7F4
:107A5000040083A7C71782976FA06FB0EFA2EFADA6
:107A6000B7E7040083A7871397E5FF1F9385050FEA
:107A7000829701456FA0AFAEEFA22FACB7E704002D
:107A800083A7C71F814517B5FF1F0355456182971F
:107A90006FA0EFACEFA26FAAB7E7040083A787132C
:107AA00097E5FF1F9385850C829701456FA02FAB4B
:107AB000EFA2AFA8B7E7040083A7C71F814517B59A
:107AC000FF1F0355C56382976FA06FA9EFA2EFA6B2
:107AD0002E85EF600055EF60900D6FA04FA8EFA2CC
:107AE000CFA5EF60D0176FA08FA75C49E1175CC9E5
:107AF0005CC583572501A1072319F50083570501AC
:107B0000A1072318F5008280F1473305F50297E7B6
:107B1000FF1F9387A7079C433E9582808D4763177D
:107B2000F60603D74600854763F2E706EFA2EFA00B
:107B3000368536842E89EF10A01D39C18357440045
:107B400093140501C18063ED97022285EF10401C5C
:107B5000FD14231294009307A002630EF50093070F
:107B6000B0026301F50293079002631BF5002285C2
:107B7000EFC0B07E31A00146CA852285EF80000F9C
:107B80006FA0EF9D2285EF001059DDBF828097E640
:107B9000FF1F9386E6FF9C42014599CF9843D4424C
:107BA00017E6FF1F2326E6FE6396D70097E6FF1F22
:107BB00023A2E6FE1385C7FE8280EFA20F98E92676
:107BC0007144330585029145EF70606201E56555AA
:107BD0006FA0EF9897E7FF1F23A8A7FA7526330534
:107BE00085029145EF70A0607DD197E7FF1F23AF1D
:107BF000A7F8592E97E7FF1F2392A7F8712697E75A
:107C0000FF1F239EA7F6974701009387E7B917E761
:107C1000FF1F2329F7F697070000938747ED17E723
:107C2000FF1F232FF7F4014565B7EFA20F91AA8537
:107C300017E5FF1F130585F4EF1060216FA02F9249
:107C4000EFA2AF8FEFF07FFEEF10E02197E7FF1F6D
:107C5000938707F49C4381CF1387C7FE09CB83D555
:107C6000C7FF17E5FF1F130525F3EFF0403A6FA09C
:107C70000F8FEFA28F8CEFF09FF119C9834785001A
:107C80002A8493F7070499E70355E500EFF05FFBBB
:107C90006FA0EF8C8347C5009304450117E9FF1FD0
:107CA000130909EF85E3832709005CC997E7FF1FE4
:107CB00023A097EE83274900E1FF97E7FF1F23AB3F
:107CC00097ECF9B7FD172306F5006105EF60E07E3C
:107CD0008307840063CB07048347840093E707F896
:107CE0002304F400B7E704009C5F82974205A9478C
:107CF00041813375F5028347840093F707FCC98FF0
:107D00002304F4008347D4003E951C402318A400AC
:107D100089CF984319CB8347C400504081458507DC
:107D20003305F502420541810297832709005CC8AB
:107D300097E7FF1F23AE97E48327490089E797E77A
:107D4000FF1F23A997E48347C400B9D383550401D7
:107D500017E5FF1F130545E4EFF0602B15BFEF9209
:107D6000DFFD97E7FF1F938767089C4701448583E2
:107D7000858B81EFAE84B2853A86EF1020142A8479
:107D800009C5EF10200B829408CC22856F903FFD2F
:107D9000EF921FF941112E8932C6AA89712C324700
:107DA00013060502CA8697050000938525D617E5B8
:107DB000FF1F1305A5DCEFF09FFA2A8429CD930459
:107DC000C50065261946AA852685EF0030688545D9
:107DD0002685EF001065174501001305A59A4E95FD
:107DE000834505002685EF0050685C483146814593
:107DF000A1075CC85CC483572401E1172319F40070
:107E000083570401E1172318F4001C4C3E85EF90C2
:107E1000DFF5A3042501228541016F90BFF3EF92A6
:107E2000DFF14111AA842EC632C4EF100003004DC9
:107E3000B2452246834784000CC050C093F7F70335
:107E400093E707042304F400231804002685EF00B9
:107E5000707E83479400A9462317A40013D73700E8
:107E600005073307D7029D8B85072306F400A30679
:107E7000E40083C70401D8488507230FF7FE17E7FE
:107E8000FF1F1307E7D05843232A04009307440138
:107E90001DEB17E7FF1F232FF7CE17E7FF1F23293F
:107EA000F7CE17E4FF1F130424CF2285EFF0A00BB9
:107EB0001C44858B5D8D09E581452285EFF02015F9
:107EC00041016F90DFE91CC317E7FF1F2324F7CCA4
:107ED000C9BFEF929FE697050000938565C40145F1
:107EE000EFF0DFBE01456F909FE7EF921FE5EFF0E7
:107EF0001FBF6F90DFE68347C500A1E7EF92FFE366
:107F00002A840355E500EFF05FD215C9834784004A
:107F100093F7F7FB2304F4001C4091C7DC4381C7AF
:107F20004C4001458297EFF09FC617E5FF1F1305F0
:107F3000A5C6EFF0400F0355E400EFF07FD06F903F
:107F40001FE28280EF927FDF97E7FF1F938747C48E
:107F500097050000938525D217E5FF1F1305C5C3BC
:107F600023A0070023A20700EFE0507E6F903FDFC1
:107F70001C4D91CBDC4381CBEF923FDC8345070066
:107F800082976F90DFDD828097E7FF1F938707C39B
:107F90009C4303C50700828097E7FF1F938707C2B2
:107FA0009C4303C51700828097E7FF1F938707C193
:107FB0009C4303C52700828097E7FF1F938707C074
:107FC0009C4303C54700828097E7FF1F938707BF45
:107FD0009C4303C53700828097E7FF1F938707BE46
:107FE0009C4303C55700828097E7FF1F938707BD17
:107FF0009C4303C56700828097E7FF1F938707BCF8
:108000009C4303C57700828097E7FF1F938707BBD8
:108010009C4303C58700828097E7FF1F938707BAB9
:108020009C4303C59700828097E7FF1F938707B99A
:108030009C4303C5A700828097E7FF1F938707B87B
:108040009C4303C5B70011E11D45828097E7FF1FE0
:108050009387C7B69C4303C5C700828097E7FF1F7D
:108060009387C7B59C4303C5D700828097E7FF1F5E
:108070009387C7B49C4303C5E700828097E7FF1F3F
:108080009387C7B39C4303D50701828097E7FF1FFF
:108090009387C7B29C4303C52701828097E7FF1FE0
:1080A0009387C7B19C4303D54701828097E7FF1FA1
:1080B0009387C7B09C4303D56701828097E7FF1F72
:1080C0009387C7AF9C4303D58701828097E7FF1F43
:1080D0009387C7AE9C4303C5A701828097E7FF1F24
:1080E0009387C7AD9C4303C5B701828097E7FF1F05
:1080F0009387C7AC9C4303C5C701828097E7FF1FE6
:108100009387C7AB9C4303C5D701828097E7FF1FC6
:108110009387C7AA9C438857828097E7FF1F93875E
:10812000E7A99C4303D5C702828097E7FF1F938787
:10813000E7A89C4303D5E70219E11305800C828070
:1081400097E7FF1F938787A79C4303C50703828098
:1081500097E7FF1F938787A69C43C85B828097E7BA
:10816000FF1F938727A58843828097E7FF1F938788
:10817000A7A48843828019E17D558280F5DE98426C
:1081800065DFFDD917E7FF1F130747C61847AA8702
:108190007155058B6319072203C507001547E37D59
:1081A000A7FC03C737001305F0057D171377F70FFA
:1081B000E364E5FC03C35700E30003FC83C86700E6
:1081C000E38C08FA03C77700494579171377F70F4F
:1081D000E364E5FA03C7A70011481305F7FF137519
:1081E000F50FE36BA8F803CE97000D481305FEFFCB
:1081F0001375F50FE362A8F803C8B7006309080018
:1082000065181378F80F1305600DE36705F703C5CC
:10821000C700794879151375F50FE36FA8F403C803
:10822000D7000D457D181378F80FE36705F503D8DF
:108230000701930E40175118420813580801E3ED47
:108240000EF303C8E7007D181378F80FE36605F313
:1082500003C827017D181378F80FE36F05F103C8F1
:108260008700C54E75181378F80FE3E70EF103D8B1
:108270006701856E938EBEE06D18420813580801A1
:10828000E3EC0EEF03D847016D18420813580801BC
:10829000E3E40EEF03D88701791842081358080168
:1082A000E36C05ED03C8A7017D181378F80FE365AB
:1082B00005ED03C5B7011D487D151375F50FE36D79
:1082C000A8EA03C5D701714879151375F50FE36561
:1082D000A8EA03D5E7011308E00F7D1542054181A7
:1082E000E36CA8E803C50702494879151375F50F33
:1082F000E364A8E8C85301C937C834005915130806
:1083000058BFE36BA8E603A8870237C534001305FE
:1083100055BF5918E36205E717E5FF1F232EC588EF
:1083200003C6050117E5FF1F232AF5880545E375F8
:10833000C5E403D82501D04933760603E31E06E2DF
:1083400003C61501E30A06E217E6FF1F2324B686DB
:1083500083C5270001466387A50003C61700F145C2
:108360003306B60283C707039305C00272971A0744
:108370001307C70516031A9796084697B387B702DF
:1083800041553E97329742074183636EE802EF9270
:10839000DF9A3685EF60D06FEFD0B0212A84EF806E
:1083A000B01D2A94EFC090252A94EF7040072A94BC
:1083B000EFF0BF802A94EF2050632A94EF5040667C
:1083C00022956F90DF998280EF923F974111A3072A
:1083D000A100EF80801E9305F10017050000130532
:1083E00065B9EFF0CFCC014541016F905F97EF92F7
:1083F0005F9217E4FF1F1304649F032884007959D8
:108400009368180097E4FF1F23A6149F13781800A1
:10841000631E0800BA84BE89368B328A2E89AA8AE6
:10842000EFE01FD67D15269509E531594A856F90F5
:10843000DF91EFE0FFD47D152695A167E357F5FEA8
:1084400097E7FF1F938787D198433E8C814B11C7D5
:108450000145EFC0B03E933B15004A85DA8656864B
:10846000D285EF7070372A8911CD1C44F99B17E72C
:10847000FF1F2321F79883270C00CDDBE3880BFA3D
:1084800082976DB7268597E7FF1F23A30796EFE036
:10849000FFCB4146CE8517E5FF1F1305A59EEF00D4
:1084A000A174EFA070080325040BEFA0700A054526
:1084B000EFA070100545EFF03FF18DBF97E7FF1F6C
:1084C0009387C7929C47858BD5C7EF921F8717E587
:1084D000FF1F1305659997E7FF1F23A9079097E7EB
:1084E000FF1F23A7079097E7FF1F23A50790EFE043
:1084F0009033EF40C002EFE0F00AEFE0700F97E733
:10850000FF1F9387278D9C4381C70545EF60B033DC
:1085100097D7FF1F9387C7759C4389C741657D1512
:10852000EF50A06BEFC0703AEFA0F00097E7FF1F8D
:108530009387C7A09C431397170163540700EFC0AC
:10854000A04597E7FF1F23AF079297E7FF1F23ADD3
:10855000079297E7FF1F23AB079297E7FF1F23A917
:108560000792EFF09F984923EFF0AFBBEFC0806711
:108570006F90EFFE828097E7FF1F938727878843DE
:108580008280EF928FFBEF60B07EEF7080006F9083
:108590000FFDEF92EFF82A849304140201112E8547
:1085A000B289A685214636C63A89EF0081611DE170
:1085B000B24638082686CE8513059404EF40604302
:1085C00021462C084A85EF00C15F1335150005616F
:1085D0006F904FF80145E5BFEF922FF693054506E2
:1085E00017D5FF1F1305C55DEFE070226F902FF7C1
:1085F000EF92AFF441112EC6EFF00FC0B24588C123
:1086000041016F90CFF5EF92AFF1AA842E84EF6015
:108610005078AA8985452285892D83C7E40113896D
:10862000940899E313890403CE8522853D2D2146C4
:10863000930519022285192D97D7FF1F9387077B72
:108640008C432285EF00E0682146938584022285D1
:10865000F52B6F902FF0EF92CFEB3971EFC0E04E1A
:108660009305400645EDEF60D06F630E051097D778
:10867000FF1F83C7A75613B7170097D6FF1F238F77
:10868000E654014489CFC16417D9FF1F1309097645
:108690009309400EFD14EFF03F986348A408EFF0F3
:1086A000AFB54169B7290900096AFD7A2A8B81446F
:1086B0007D199389F97B130A0A71938A8AC7EFF0AF
:1086C000BF9563D5A4041304400EB387840217D763
:1086D000FF1F1307A7710324070B3E948357C401A0
:1086E0006386270918403307EB4063EAE9008347B4
:1086F00044008507B3874703D6976369F7060146A9
:1087000081450945EFF0CFE8AA8B29E1EF20105A07
:108710008547631FF50489659385057117D5FF1F8C
:108720001305054AEFE0B00EA1A8B30734030327F1
:10873000090BBA9703D7C7016308970003C757000F
:10874000A38207002382E7000504B1B79305C500A3
:108750002285EFF05FEB5E852286973501009385D9
:10876000A503EFF0CFEB5E85EF00E06F850481BFDE
:1087700097D7FF1F938787679C478D83858BC1FFA2
:1087800021616F908FDC01468545094502D002D2F8
:1087900002D402D6EFF0CFDFAA847DD1EFC0203A19
:1087A0001389C4002A8481454A85C1210C40414671
:1087B0004A85692983294400638809084E8502D8BF
:1087C00002DA02DC02DEEF00816A2ACE14100546CE
:1087D0002C0808184ECCEF4060191375F50F2DE5E5
:1087E0008355840093E525004A856D2911460C10B8
:1087F0004A85A929014697350100938565FA2685A2
:10880000EFF0EFE12685EF0000665C40B5DB014646
:1088100085450D45EFF0CFD7AA843DD14840138957
:10882000C400EF00C1642AC64A85C5263246636A81
:10883000C5004C404A851929014681452685EFF03F
:108840000FDE26850D252DBF8355840071BFEF9265
:10885000CFCE97D7FF1F938767599C4719CD93E7D2
:10886000870017D5FF1F1305A53517D7FF1F232333
:10887000F758EFE060786F908FCEDD9B17D7FF1F22
:10888000232AF756EF2090427DF517D5FF1F1305D9
:108890002533EFE04079C5B7EF92AFC74169AA89A8
:1088A0002E8AB28A368BBA8B814417DCFF1F130CD9
:1088B000EC53930C400E7D19EFF00FF663C4A40047
:1088C00001442DA03384940383270C0B3E948357DB
:1088D000C401638027055A87D6865286CE85130544
:1088E0000403EFF01FCB11C523800B0022856F908E
:1088F000CFC58347F40191CF5A87D6865286CE855D
:1089000013059408EFF0FFC809C585472380FB00D5
:10891000F1BF850455B783574500638D0716EF9265
:108920002FC001112A84ED2619C58547630AF50475
:1089300005616F902FC2EFC040217DF9835744003D
:108940004947ED9BE396E7FEC14522854524AA846D
:108950002285F52E0357440002CE91472A896317DA
:10896000F700228539293C082ACC3ECEEFC0201DD5
:108970005C55DDDF74084A86A685054582974DBFA4
:1089800003574400D147E3F5E7FA032A0400C1691D
:10899000014997DAFF1F938A6A45130B400EFD19B0
:1089A000EFF08FE76344A90C2285032A04008D268B
:1089B000A1452A8922851D2CAA842285D926144006
:1089C0002A86AA8978082685CA85EFF0FFECAA8452
:1089D00025D103C7F40189476315F7008347C10117
:1089E000A1DB5546D28513856400EF00E11F0145E8
:1089F000EF60103801C583D7C401B1EB97D7FF1FD3
:108A00009387C73E9C4793551900858913D7370034
:108A1000058B11CB8983858B6397B70001452EC6E3
:108A2000EFF0FFE2B2454E85EF60703C0346C101B6
:108A30002A84937519002685EF70703131C9268517
:108A4000EF607037268511C00145EF60D061EF20DF
:108A5000F0258547E31EF5EC83C754001307F00F9C
:108A6000E388E7EC8507A382F400D9B5B304690372
:108A700083A70A0BBE9483D7C40163893701554687
:108A8000D28513856400EF00C11371D1050909BFB8
:108A90005DDC5DBF8280EF92AFA8EF60902C11CDBE
:108AA000C164014417D9FF1F130949349309400ECB
:108AB000FD14EFF06FD6634AA40017D5FF1F13050E
:108AC0002510EFE060536F90EFA833053403832740
:108AD000090B3E958357C501638697002312050055
:108AE000EF60702D0504F1B797D7FF1F938707300C
:108AF0009C478D83858B99EBEF922FA417D5FF1F91
:108B00001305050CEFE020526F906FA58280EF9265
:108B1000CFA297050000938545B417D5FF1F130515
:108B2000250AEFE0A0426F908FA3EF920FA188413A
:108B3000B7E70400BC5B050542054181829709C582
:108B400085472300F50005056F906FA183C7F5FFEA
:108B50002E858507A38FF5FE828083C7F5FFFD175D
:108B600093F7F70FA38FF5FE99EBEF920F9DB7E701
:108B70000400BC571385F5FF82976F904F9E82804B
:108B80001C41035745008D8FBA951CC12312B500B7
:108B90003E85828093D78500A2051441DD8D8357E1
:108BA00045001387E6FF18C189072312F50013D685
:108BB00085004111238FB6FEA38FC6FE410182803E
:108BC00018419307F7FF1CC18357450085072312FF
:108BD000F500A30FB7FE8280835745008D8F2312C7
:108BE000F5001C41BE950CC12E858280AA8703D753
:108BF000470008410D8FAA952392E7008CC382801D
:108C0000184108453305A740828083574500035724
:108C100065001D8F1C4108453385A7403305A740DB
:108C20008280EF928F9141112EC62A84EFF0FFFDD2
:108C3000B2456373B50001A0835744000840BE9558
:108C40002312B4003E9541016F906F91EF92EF8E29
:108C500041112E84B28532C6EFF0BFFC3246A285A8
:108C6000EFF0907841016F908F8FEF920F8D2E84EF
:108C70008545EFF01FFB230085006F904F8EEF922C
:108C8000CF8B41112317B1008945EFF09FF983473E
:108C9000E1002300F5008347F100A300F500410146
:108CA0006F90EF8BEF926F8993D78500A2054111EA
:108CB000DD8D2317B1008945EFF0BFF68347E10052
:108CC0002300F5008347F100A300F50041016F90F8
:108CD0000F89EF928F861397850193D78501C1661F
:108CE000938606F0D98F13D78500758FD98FA2058B
:108CF0003707FF00F98D4111DD8D2EC69145EFF04C
:108D00005FF26C001146EFF0306E41016F902F85DD
:108D1000EF92AF821C41854503C40700EFF0DFEB03
:108D200022856F90CF83EF924F811C41411189457D
:108D300003C7070083C717002307E100A307F1005B
:108D4000EFF09FE90355E10041016F904F81EF8201
:108D5000DFFE1C414111894503C7070083C7170087
:108D60002307E100A307F100EFF01FE78357E100BD
:108D7000410113D58700A2075D8D420541816F80B7
:108D80001FFEEF829FFB0C4141112A8411466800AF
:108D9000EFF0906591452285EFF01FE4B247C16680
:108DA000938606F01397870113D58701598D13D742
:108DB0008700758F598DA2073707FF00F98F5D8DEA
:108DC00041016F80DFF91C45BE950CC18280AE87E2
:108DD000944391E6584101EF0CC15CC1828003C706
:108DE000570013671700A382E700B687D5B70CC3F7
:108DF000EDB7AA87084119CD1841D44398C363132E
:108E0000D500D8C32A87034657009376160081E61B
:108E1000232007008280944381CA8C4203A8470024
:108E20008CC363930601CCC3799A14C3A302C70011
:108E30003687D1BF1C45DC471D8DB777DBB69387DE
:108E400077DB09853305F502420541818280F147D0
:108E5000B385F50248452E958280834745008507F6
:108E60002302F5008280EF825FED2A8419E06F8093
:108E70001FEF83474400E5DFFD1793F7F70F230249
:108E8000F400F5F71C4403D7270005072391E700FA
:108E9000DC4399C3228582974C4889CD834754008F
:108EA000898B99E71C4422859C479C439C47829769
:108EB000232A04000040232004004DBFEF82FFE777
:108EC0008357250041112EC691E7014422854101B7
:108ED0006F80FFE8035705008147F146E307F7FE7F
:108EE000B385D702404585072E948345440008C4C6
:108EF000F5F5B247AA8481E7232A040009A81C4596
:108F00006C0022859C439C43829748C85DDD854761
:108F10002312F400B247232004002318040023196D
:108F2000F4005C485CC483D72400FD172391F4004F
:108F300071BFEF829FE097D7FF1F938767CA88436F
:108F400023260500232405004105EFE0C00D6F80B6
:108F50001FE1EF829FDE17D4FF1F130464C81C407B
:108F6000411189CF9C472300B5002AC65CC1EFF0B0
:108F70005FFC1C40DC4399C33245829741016F80FE
:108F80001FDE034745001DEB584DAA877D550DCBCD
:108F9000EF82BFDA1CC3DC4797D6FF1F23A2E6C4CB
:108FA000F156130507012390D7009705000093851C
:108FB0008501EFD0B07901456F807FDA7D558280E1
:108FC0008280EF829FD70111614681452800EF80A2
:108FD000DFD997D7FF1F9387A7C09C43280093052D
:108FE000F00FDC473EC6EFF0DFF605616F803FD73C
:108FF00097D7FF1F9387C7BE9C43D847A167938726
:10900000C7026312F70A397106DE22DC26DA800015
:109010004AD84ED652D456D23285B284EFF05FCFC2
:10902000AA892685EFF03FD02318A4FC2685EFF00F
:109030009FCF2319A4FC2685EFF0FFCE83D74400F1
:109040000A8A231AA4FC858393F7F70F230EF4FCF6
:109050008607BD0793F7073F3301F1408A8A01492C
:109060008347C4FD6365F902CE85130584FC232C78
:1090700054FDEFF01FEE5281130104FCF2506254D4
:10908000D2544259B259225A925A2161828026857D
:10909000EFF07FC993171900D69705092390A70011
:1090A0001379F90F75BF828097D7FF1F938747B356
:1090B0009C43D847A1679387A7026310F70A3971C9
:1090C00006DE22DC26DA80004AD84ED652D456D2AA
:1090D0003285B284EFF0DFC3AA892685EFF0BFC4E2
:1090E000FD572318A4FC26852319F4FCEFF0BFC319
:1090F00083D744000A8A231AA4FC858393F7F70FC9
:10910000230EF4FC8607BD0793F7073F3301F140B8
:109110008A8A01498347C4FD6365F902CE85130538
:1091200084FC232C54FDEFF0DFE25281130104FC98
:10913000F2506254D2544259B259225A925A216181
:1091400082802685EFF03FBE93171900D697050958
:109150002390A7001379F90F75BF828097D7FF1F5F
:10916000938707A89C43D847A16789076318F70826
:10917000397106DE22DC26DA80004AD84ED652D477
:1091800056D232853289EFF0BFB8AA894A85EFF00E
:109190009FB9835749000A8A2318A4FC858393F753
:1091A000F70F230CF4FC8607BD0793F7073F330145
:1091B000F1408A8A8144834784FD63E5F402CE85C9
:1091C000130584FC232A54FDEFF0BFD8528113010C
:1091D00004FCF2506254D2544259B259225A925A63
:1091E000216182804A85EFF01FB493971400D697CF
:1091F00085042390A70093F4F40F75BF828097D75E
:10920000FF1F9387E79D9C43D847A1679387E70497
:109210006312F70A397106DE22DC26DA80004AD8AA
:109220004ED652D456D23285B284EFF07FAEAA89A0
:109230002685EFF05FAF2318A4FC2685EFF0BFAEC4
:10924000231AA4FC2685EFF01FAE83D744000A8AB8
:109250002319A4FC858393F7F70F230EF4FC8607EC
:10926000BD0793F7073F3301F1408A8A01498347DD
:10927000C4FD6365F902CE85130584FC232C54FDDF
:10928000EFF03FCD5281130104FCF2506254D254EE
:109290004259B259225A925A216182802685EFF0B2
:1092A0009FA893171900D69705092390A700137953
:1092B000F90F75BF828097D7FF1F938767929C43F2
:1092C000D847A1679387C7046310F70A397106DE90
:1092D00022DC26DA80004AD84ED652D456D23285C5
:1092E000B284EFF0FFA2AA892685EFF0DFA3FD5735
:1092F0002318A4FC2685231AF4FCEFF0DFA283D701
:1093000044000A8A2319A4FC858393F7F70F230EE0
:10931000F4FC8607BD0793F7073F3301F1408A8AC3
:1093200001498347C4FD6365F902CE85130584FCBA
:10933000232C54FDEFF0FFC15281130104FCF250C5
:109340006254D2544259B259225A925A21618280AF
:109350002685EFF05F9D93171900D6970509239096
:10936000A7001379F90F75BF828097D7FF1F9387E6
:1093700027879C43D847A167DD07631BF702EF826D
:10938000DF9B797132853284EFF09F982AC622855F
:10939000EFF07F992311A1022285EFF07F97B2456C
:1093A0002300A1022808EFF0DFBA45616F803F9BE0
:1093B000828097D7FF1F9387A7829C43D847A167D6
:1093C00093878704631BF702EF823F977971328599
:1093D0003284EFF0FF932AC62285EFF0DF94231149
:1093E000A1022285EFF0DF92B2452300A1022808F6
:1093F000EFF03FB645616F809F96828097C7FF1F51
:109400009387077E9C43D847A1679387A704631C73
:10941000F700EF829F92011128008145EFF07FB3A2
:1094200005616F80DF93828097C7FF1F9387477B1B
:109430009C43D847A167938757026311F702EF82D5
:10944000DF8F01113285EFF0BF8C2308A100814529
:109450002800EFF01FB005616F807F90828097C772
:10946000FF1F9387E7779C43D847A1679387E7025D
:10947000631FF702EF827F8C011132853284EFF097
:109480009F8AAA842285EFF01F8A854719E52285E5
:10949000EFF01F884205B337A0002800814523184C
:1094A00091003ECAEFF0FFAA05616F805F8B82805A
:1094B00097C7FF1F9387C7729C43D8479947631F7D
:1094C000F704EF829F87797132853284EFF05F84F1
:1094D0002AC62285EFF03F852310A1022285EFF0F6
:1094E0003F832301A1022285EFF09F82A301A10205
:1094F0002285EFF0FF812302A1022285EFF05F8138
:109500002313A1022285EFF0BF80B2452314A102EC
:109510002808EFF01FA445616F807F84828097C781
:10952000FF1F9387E76B9C43D847A1679387C703C7
:10953000631FF704EF827F80797132853284EFF008
:109540002FFD2AC62285EFF00FFE2310A1022285EF
:10955000EFF06FFD2311A1022285EFF06FFB2302D4
:10956000A1022285EFF0CFFAA302A1022285EFF03B
:109570002FFA2303A1022285EFF08FF9B245A3034E
:10958000A1022808EFF0FF9C45616F804FFD8280AB
:10959000EF82AFFA01112A84EFF08FF7AA842285B7
:1095A000EFF06FF82285EFF00FF8035744008D4776
:1095B00063F5E7002285EFF00FF72285EFF0AFF6B5
:1095C0002800A685EFF0FF9805616F804FF997C7D7
:1095D000FF1F9387E7609C43D847A167FD07631986
:1095E000F700EF828FF53285EFF09FFA6F802FF74B
:1095F000828097C7FF1F9387A75E9C43D847A167C8
:10960000E5076311F706EF824FF3797132853284F3
:10961000EFF00FF02AC62285EFF0EFF02285EFF091
:109620008FF02310A1022285EFF0EFEF5205518158
:109630002311A102228523020102EFF06FEDA302A4
:10964000A1022285EFF0CFEC2303A1022285EFF0E7
:109650002FECB245A303A1022808EFF09F8F4561CC
:109660006F80EFEF828097C7FF1F938767579C43F8
:10967000D847A1679387E7036319F700EF82EFEB01
:109680003285EFF0FFF06F808FED828097C7FF1F6C
:10969000938707559C43D847A16793874704631472
:1096A000F702EF828FE9797132853284EFF04FE66D
:1096B0002AC62285EFF02FE7B2452808EFF07F8910
:1096C00045616F80CFE9828097C7FF1F938747511D
:1096D0009C43D847A167938787026316F702EF82FE
:1096E000CFE5797132853284EFF08FE22AC6228588
:1096F000EFF00FE2B2452300A1022808EFF07F85CA
:1097000045616F80CFE58280EF822FE30111EFF09A
:109710002FE0AA852800EFF0DF8305616F802FE43A
:1097200097C7FF1F9387C74B9C43D847A167D107B3
:109730006319F700EF826FE03285EFF0FFFC6F8076
:109740000FE2828097C7FF1F938787499C43D847C2
:10975000A167C5076319F700EF822FDE3285EFF0AE
:10976000BFFA6F80CFDF828097C7FF1F938747477D
:109770009C43D847A167B9076319F700EF82EFDB75
:109780003285EFF07FF86F808FDD828097C7FF1FF3
:10979000938707459C43D847A167AD076319F70036
:1097A000EF82AFD93285EFF03FF66F804FDB8280DA
:1097B00097C7FF1F9387C7429C43D84789476310C9
:1097C000F702EF828FD70111328532C8EFF04FD404
:1097D000AA852800EFF0EFF705616F804FD88280EF
:1097E00097C7FF1F9387C73F9C43D847A1678D0743
:1097F0006317F702EF826FD4011132853284EFF0E4
:109800002FD113066100AA844C002285EF20D00CD2
:109810002800A685EFF0EFF305616F804FD48280BA
:1098200097C7FF1F9387073C9C4381CBDC4391C7BD
:10983000EF82AFD082976F808FD28280EF82EFCF9E
:1098400079713C08AE843ED2A165B7070A002A842C
:109850003ED448103C08DD053ED636C432C63AC276
:10986000EFD0BFAA12474810BA85EFF00FC03246BA
:109870004810B285EFF0AFC0A2464810B685EFF0B1
:10988000CFBE501001478146A6852285EFD07FC804
:1098900045616F80CFCCEF824FCA01117C00032954
:1098A000C501AE843ECAA165B70707002A843ECC35
:1098B00048087C00C5053ECEEFD03FA58345D900C2
:1098C0004808EFF08FBA500801478146A6852285E7
:1098D000EFD03FC405616F808FC8EF820FC683C78A
:1098E000950093F7F707A384F500EFF0DFFA6F8098
:1098F0000FC7EF828FC479713C08AE843ED2A16558
:10990000B70709002A843ED448103C0893854504D3
:109910003ED632C636C4EFD05F9FA2464810B68509
:10992000EFF0AFB432464810B285EFF04FB55010AB
:1099300001478146A6852285EFD0BFBD45616F8076
:109940000FC2EF828FBF83C7950041112A8493F71E
:10995000F707A384F50032852EC6EFF0CFBC8567EC
:109960002AC4637CF500EF50B0402246B24509E9B5
:10997000114781462285EFF07FEC41016F802FBEB9
:1099800001478346F501FDB7EF828FB901113C0015
:109990003ECAB7070A003ECC3C003ECE83C79500C6
:1099A000AA89328593F7F707A384F5002E84EFF098
:1099B0008FB785676371F504A165AA8493858504D3
:1099C0004808EFD09F942685EF50903A2A891DE5EC
:1099D00091454808EFF06FA9A6854808EFF02FAA37
:1099E000CA854808EFF06FA8014781465008A28554
:1099F0004E85EFD01FB205616F80CFB58145480815
:109A0000EFF0AFA603490902C1BFEF826FB17971D0
:109A10001C103ECAB7070F003ECC404D1C10AA8454
:109A2000AE894808994532C636893ECEEFD0FF8DC3
:109A300032464808B285EFF04FA363040902A545FA
:109A40004808EFF00F9E2546CA85EFF0E019500850
:109A500001478146CE852685EFD0BFAB45616F803B
:109A60006FAF8355C4024808EFF06FA10355E402BD
:109A7000814515C185478545630FF500C167FD1711
:109A80009305F00F6309F5007D15EF5020749305E1
:109A9000150093F5F50F4808EFF02F9D834504035B
:109AA0004808EFF08F9C834514034808EFF0EF9BC4
:109AB000835524034808EFF08F9C835544034808DE
:109AC000EFF0EF9B69B7EF824FA783C79500814600
:109AD000014693F7F707A384F500EFF01FF36F80BB
:109AE0000FA8EF828FA579713E841C103ECA2E8983
:109AF000B7070F00A1653ECCFD051C10AA844808DD
:109B000042C03AC23ECE36C432C6EFD01F80324683
:109B10004808B285EFF06F95A2464808B685EFF089
:109B20000F9612474808BA85EFF06F950248630414
:109B3000080291454808EFF0CF8E1146A285EFF05C
:109B4000A00A500801478146CA852685EFD07F9C30
:109B500045616F80CFA089454808EFF08F8C83471F
:109B600004002300F50083471400A300F500D1BFD3
:109B7000EF820F9B83C7950001112A8A93F7F7079D
:109B8000A384F5003285AE8432C6EFF0CF99324619
:109B90002A893285EFF0CF978567637FF900AA891C
:109BA0004A85EF50F01C2A8419E9114781464A86FC
:109BB000A6855285EFF09FC805616F80AF999387A6
:109BC000E9FF93F7F70F0547E368F7FE8347F501D1
:109BD00095E78947E382F9FE8346F4015285014700
:109BE0004A86A685EFF09FC5A167D90748083ECCF5
:109BF000230A010002CEEFF0BFC27DBF639CE700E5
:109C00008947639CF90093071020231FF500EF504C
:109C1000901AD9B70947E391E7FC8D47E39EF9FA1B
:109C20002285EF50D03B97C7FF1F9387A71A9C430D
:109C300099E797C7FF1F9387A7039C4389C703D55D
:109C40000400EF60300C231F04002285C9B7EF82A7
:109C5000CF8E01113C003ECAB7070B003ECC3C0042
:109C60003ECE83C795002A89328593F7F707A384F0
:109C7000F500AE84EFF02F8B93170501C187635E6B
:109C8000F004A1652A849385E5024808EFD0EFE748
:109C9000A2854808EFE0BFFE97C7FF1F938747FDE7
:109CA0009C439DEF01449375F40F4808EFE0FFFBE0
:109CB0009355844093F5F50F4808EFE01FFB93554B
:109CC000044193F5F50F4808EFE03FFA014781465C
:109CD0005008A6854A85EFD0DF8305616F802F8805
:109CE000416585460546A2857D15EF3070675DD9D3
:109CF0005105EFD04027130440063344850265B771
:109D0000EF82AF830111B70706003EC683C79500F7
:109D100021642A8993F7F707A384F500AE8428000D
:109D20009305A4040AC40AC8EFD02FDE300001470F
:109D30008146A6854A85EFD0CFFDEFE02FF81304CA
:109D40009404480822CC230A010002CEEFF05FAD54
:109D500005616F80CF80EF72BFFCC1642A89014426
:109D600097C9FF1F93898908130A8002FD14EFE049
:109D7000AFAB6345A40001456F70DFFDB30744033B
:109D800003A7C90ABA9703D707006306970083D7CA
:109D90002700638427010504D9BF0545F1BFEF7291
:109DA0003FF82A8A2E8999C123A005008149814460
:109DB00097CAFF1F938A4AE3614BEFE02FAD63C55B
:109DC000A4004E856F701FF93384640383A70A00D3
:109DD0003E948357040099E7630409002320890017
:109DE0008504E1BF4146D28513054400EFE0705D74
:109DF00065F9A289F5B7EF72BFF239717C083ED4DC
:109E0000B7070A003ED67C083ED883C795002A8A49
:109E1000328593F7F707A384F5002E8932C6EFE069
:109E20009FF085676373F5063246AA843285EFE0BA
:109E30003FEE8547AA8963EAA704A1659385850457
:109E40002810EFD08FCC2685EF5080722A8429E12C
:109E500091452810EFE07FE1A6852810EFE03FE272
:109E6000CE852810EFE07FE0014781463010CA859B
:109E70005285EFD00FEAA1679387770448183EDC3C
:109E8000230A010202DEEFF0BF9921616F709FEC9F
:109E900081452810EFE07FDDA6852810EFE03FDE4A
:109EA00097C7FF1F9387472B9C4391C722856387E2
:109EB0000900EFB0600C8345040265B7EFB0200BDA
:109EC000DDBFEF72FFE583C795004111AA8993F7C3
:109ED000F707A384F5003285AE84328AEFE0BFE451
:109EE0008567637BF5022A89EF5080682A84914652
:109EF00021C18347F50105476383E70291C70D47F9
:109F0000636EF702AD462DA09305050303250A00F5
:109F10004146EFE0104B1DE141016F70BFE3930537
:109F2000950803250A004146EFE0B049814679F9DA
:109F30004A86A6854E85EFF0DF9BF9BF83250A0090
:109F400013059408EF60600119C1C146D5B797C7E2
:109F5000FF1F938727E89C4399E797C7FF1F9387C5
:109F600027D19C4389C72285EF60A05479FD85479E
:109F7000A30FF4002285EF80B05D2285EF50A0632F
:109F80004E8581464A86A685EFF0BF96A1679387E6
:109F9000570448003EC42302010002C6EFF05F8868
:109FA000A5BFEF721FD783C795004111AA8993F708
:109FB000F707A384F50032852E89B28AEFE0BFD679
:109FC00085676370F50CAA84EF50805A2A841DE9D6
:109FD000416B014A97CBFF1F938B4BE1130C400E53
:109FE0007D1B19A833048A0383A70B0B3E94835768
:109FF000C401638D6703050AEFE00F82E344AAFE04
:10A00000954639A88357C5016392970293050503C6
:10A0100003A50A004146EFE0D03A994611E1814696
:10A020002686CA854E85EFF0DF8CA1A883A50A009D
:10A0300013050403EF507072C1467DF12285231E83
:10A040009400EF80F0502285EF50E05697C7FF1F35
:10A05000938787109C438DCB230004022285EFA0B9
:10A0600090614E8581462686CA85EFF09F88A1675C
:10A070009387070448003EC42302010002C6EFF0A4
:10A080002FFA41016F707FCC89472300F402D1BFC2
:10A09000397106DE22DC4AD8800052D456D25AD01A
:10A0A00026DA4ED65ECE2E8A32892A8BEFD0DFF3A7
:10A0B0000605710541998A8A3301A140232224FCB7
:10A0C000231404FCEFD05FF283479A0006053505A0
:10A0D00093F7F7072315A4FCA304FA004A85232667
:10A0E00024FCEFE05FC493170501C1876340F002D1
:10A0F0005681130104FCF2506254D2544259B259B1
:10A10000225A925A025BF24B21618280AA844A85CC
:10A11000EFE07FC1AA894A85EFE0FFC0A165938582
:10A12000C5022A89130544FCEFD02F9E2685EFD067
:10A13000AF93854501C94A86CE85EFD06F8DAA8B36
:10A1400015ED8945130544FCEFE03FB2A6851305E4
:10A1500044FCEFE0DFB2CE85130544FCEFE03FB2F4
:10A16000CA85130544FCEFE09FB101478146130601
:10A1700044FCD2855A85EFD0CFB99DBF81451305E8
:10A1800044FCEFE09FAEA685130544FCEFE03FAF33
:10A19000CE85130544FCEFE09FAECA85130544FC51
:10A1A000EFE0FFAD8144EFD03FE4E3D0A4FC83A710
:10A1B0000B0113971400BA9783D5070089C51305BF
:10A1C00044FCEFE0DFAB8504F9BF797106D622D4F9
:10A1D0004AD000184ECE52CC56CA26D25AC8AE89A2
:10A1E0003289AA8AEFD05FE00605690541990A8A9B
:10A1F0003301A140232A24FC231C04FCEFD0DFDE22
:10A2000083C7990006052D0593F7F707231DA4FCC6
:10A21000A384F9004A85232E24FCEFE0DFB09317D6
:10A220000501C187634FF0005281130104FDB25054
:10A23000225492540259F249624AD24A424B456131
:10A240008280AA844A85EFE01FAEA1659385A502AE
:10A250002A89130544FDEFD04F8B2685EFD0CF80A0
:10A26000854519C5CA85EFC0BFFD2A8B0DE9894513
:10A27000130544FDEFE07F9FA685130544FDEFE045
:10A280001FA0CA85130544FDEFE07F9F014781466B
:10A29000130644FDCE855685EFD0AFA771B7814533
:10A2A000130544FDEFE07F9CA685130544FDEFE018
:10A2B0001F9DCA85130544FDEFE07F9C8144EFD0CC
:10A2C000BFD2E3D5A4FC83270B0113971400BA97E0
:10A2D00083D5070089C5130544FDEFE05F9A850427
:10A2E000F9BFEF729FA583474500404DD5E7FD5765
:10A2F0004DC0834694000947636DD7080346B400F8
:10A30000854663E8C6088306E40063C406085C4526
:10A31000F9562390D70097C7FF1F83C7278D99E36E
:10A32000A304E40097C7FF1F938787949C4381E7AA
:10A330008947A306F40097C7FF1F9387E7E19C4373
:10A3400081E789472306F4009705000093854505BA
:10A35000AA8413050401EFC0703FFD57231AF402CD
:10A3600081471CDC014897C7FF1F23AD878697C72D
:10A37000FF1F93876787232E040304C08043EFD019
:10A38000FFD061463306C50281452285EF70FF9DEF
:10A3900081473E856F70BF9CFD57E5BFEF72FF9907
:10A3A0002A8403554502EF50A01C09E5231E040032
:10A3B0006F70FF9A8357E401E5DF930504FF1715DB
:10A3C00001001305A577EFB01063DDB7EF72FF96BC
:10A3D0002E89A16541119385E5032A8436C432C6CE
:10A3E000BE843AC2EFC07FF212472285BA85EFE001
:10A3F000DF8732462285B285EFE07F88A24622853C
:10A40000B685EFE0DF87630D090091452285EFE017
:10A410005F811146A685EFE0207D41016F703F947A
:10A4200089452285EFE0EFFF83C704002300F50094
:10A4300083C71400A300F500CDB7EF721F9083C748
:10A440009500444D054793F7F707A384F5001C4298
:10A45000411183C70700636DF7042E842A8985CCD8
:10A4600003C7D4006309F70217C7FF1F130747800C
:10A47000184301CFA386F400EF80902B83C7D4004C
:10A4800089E741657D15EF30407583D72403918BB3
:10A4900099C3EFB0B0624A85A285EFF0CFBFA16744
:10A4A000C10748003EC42302010002C6EFF04FB7C7
:10A4B00041016F70DF8AEF725F8803D745008D47D7
:10A4C000AA8441112E8432892E8563EDE700EFE0E6
:10A4D0009F85AA85230009002685EFC07FD641010C
:10A4E0006F70FF87EFE03F842AC62285EFE0BF83CD
:10A4F000B24585472A862300F9002685EFC05FD143
:10A50000F9BF397106DE22DC26DA80004ED652D43D
:10A5100056D24AD85AD05ECEAE89B284AA8AEFD03B
:10A52000BFAB06051305250241990A8A3301A140F4
:10A53000232224FC231404FCEFD01FAA83C7990014
:10A5400006054D0593F7F7072315A4FCA384F9002E
:10A550002685232624FCEFE00FFD93170501C18714
:10A560006340F0025281130104FCF2506254D25451
:10A570004259B259225A925A025BF24B21618280AF
:10A58000AA8B03AB0400EFC03FCE35E983D744006C
:10A5900001498544F11793B71700A301F4FC8347E1
:10A5A00034FCA165BDC79385E504130544FCEFC0E9
:10A5B000DFD5A685130544FCEFE02FEBDE85130500
:10A5C00044FCEFE0CFEB834734FC114691E30946AE
:10A5D000DA85130544FCEFE06FE781446308090066
:10A5E000416B7D1BEFD05F9F63C8A402014781468A
:10A5F000130644FCCE855685EFC0BFF1A5B7A685EE
:10A60000130634FCEFF03FEB933415002A898604DF
:10A6100079B79385C50451BF8327C90013971400E8
:10A62000BA9783D5070063866501130544FCEFE004
:10A630000FE5850445BFEF72CFED79711C103EC464
:10A64000B7070F003EC61C103EC883C79500AA8AF4
:10A65000328593F7F707A384F500AE893284EFE0E3
:10A660008FEC93170501C1876350F0062A8A228573
:10A67000EFE06FEB2A895285032B0400EFC0DFBEA9
:10A6800039E58357440081440544F11793B7170017
:10A69000A303F10083457100DA872287CA865286B8
:10A6A0002800EFF0BFD2014781463000CE855685A5
:10A6B000EFC03FE6A1679387D70348083ECC230A43
:10A6C000810026CEEFF0CF9545616F700FE8A2852F
:10A6D00013067100EFF03FDEAA84094445DD3544DE
:10A6E000E30A55FB4A85EFF00FE70D4445D50144D9
:10A6F000EFD09F8E634BA400C16B0144FD1BEFD0D4
:10A70000BF8D634EA400154471B7DC4413171400C9
:10A71000BA9783D70700638127030504D1BFD844C4
:10A7200093171400BA9703D7070063197701239092
:10A7300027012685EF80C0540144A9BF0504C1B795
:10A74000EF720FDE83C7950041112A8A93F7F7074E
:10A75000A384F50032852E893284EFE0CFDC931795
:10A760000501C187635BF004AA892285EFE0AFDBB6
:10A770002311A1004E85832A0400EFC0FFAE29E11A
:10A780008357440085440144F11793B71700A30091
:10A79000F1000348110003572100D6875285CE8669
:10A7A0002686CA85EFF0EFB3A167F10748003EC4E3
:10A7B0002302910022C6EFF0AF8641016F708FD95E
:10A7C000A28513061100EFF01FCF2A84894471D1AE
:10A7D0008357210011678544BA97C2071167C18367
:10A7E0001307F7EFE367F7FA97B7FF1F9387875EC3
:10A7F0009C4391C7854513052100EF40300E8355DA
:10A80000210022858144EFC09F9D41D52310050082
:10A810002285EF808048B5BFEF72AFCF83C7950028
:10A8200041112A8B93F7F707A384F50032852E8A0E
:10A830003284EFE04FCF93170501C1876359F004CD
:10A84000AA8A2285EFE02FCE2A895685832B040021
:10A85000EFC09FA121E18357440081440544F117D3
:10A8600093B71700A301F10003483100DE875A8532
:10A870004A87D6862286D285EFF0AFA6A167ED077C
:10A8800048003EC42302810026C6EFE07FF9410163
:10A890006F70AFCBA28513063100EFF0DFC1AA8441
:10A8A000094479D19167CA97C2071167C183130719
:10A8B000F7EF0544E36AF7FACA85EFC05F920144F7
:10A8C00045F58149EFD04FF263DBA9009848939793
:10A8D0001900BA9703D7070015E723902701EFD097
:10A8E000AFF01544E382A9F82685EF80003B97B7C7
:10A8F000FF1F9387274E9C430144BDD74A85EF40F5
:10A9000040769DB785097DBFEF728FC179713E8416
:10A910007C083EC82E8AB7071400A1653ECAE5052B
:10A920007C08AA89080836C4428932C6BA8AC68415
:10A930003ECCEFC09F9DCA850808EFE00FB33246BA
:10A940000808B285EFE0AFB3A246630E09029D4549
:10A950000808EFE00FAD1D468145EF700FC163871A
:10A960000A0691450808EFE0CFAB1146A685EFE057
:10A97000A027100801478146D2854E85EFC07FB9D8
:10A9800045616F702FBDB6850808EFE04FAF1C40E2
:10A990000808D8439355C701858912075183B2052A
:10A9A000D98DEFE0CFAD1C40080883C58700EFE0EC
:10A9B000CFAB1C40080883C5A700EFE00FAB1C40DD
:10A9C000080883C59700EFE04FAA51BF89450808E2
:10A9D000EFE02FA583C704002300F50083C7140010
:10A9E000A300F50079B7EF72AFB383C795004111AB
:10A9F000AA8993F7F707A384F5003285AE843284E1
:10AA0000EFE06FB293170501C1876357F0042A89FD
:10AA1000032A0400EFC05F8519E983574400054805
:10AA2000F11793B71700A307F100814621A8130679
:10AA3000F100A285EFF03FA81DC11C459DC383D640
:10AA4000470001480347F10093078500D2884A86F2
:10AA5000A6854E85EFF05FEB41016F70AFAF0948FF
:10AA6000E9B71D48D9B7EF72AFAB65715C083EC45A
:10AA7000B7077B013EC65C083EC883C795002A8A9B
:10AA8000328593F7F707A384F500AE89EFE04FA86E
:10AA90008357E100C5C389452800EFC01F87814562
:10AAA0002800EFE08F9CEFC0FF8B97B7FF1F9387C5
:10AAB000A76A9C4317B4FF1F03444413AA8433348A
:10AAC000800099C31364240097B7FF1F9387471A28
:10AAD0009C4399C31364440097B7FF1F9387872F44
:10AAE0009C4399C31364840083D504002800014962
:10AAF000EFE0EF9883D524002800EFE04F9883D54E
:10AB000044002800EFE0AF97EFD00FC9931505017F
:10AB1000C1812800EFE0AF96A2852800EFE02F96D4
:10AB20009C44636CF900014781463000CE85528514
:10AB3000EFC03F9E59616F70EFA1DC4413144900D0
:10AB400028003E94EFE06F8C834744000347540095
:10AB500089070607BA978607E36EF5FC835524003C
:10AB60002800814AEFE0AF91834544002800EFE0E0
:10AB7000CF8F834554002800EFE02F8F8347440098
:10AB800063C9FA00814A8347540063CFFA0005097C
:10AB900041BF1C4413975A002800BA9783D5070079
:10ABA000850AEFE0CF8DD9BF032BC40093975A00DD
:10ABB00028003E9B83552B00850AEFE04F8C835580
:10ABC0000B002800EFE0AF8B7DBFEF720F975C4961
:10ABD00093E717005CC9EF8020336F704F98EF72D6
:10ABE000CF952E848145EFF08F9B05C183570500DB
:10ABF000FD172310F50009C4835725002310F40026
:10AC0000EFF0BFFC01456F708F9531456DDC23106F
:10AC10000400D5BFEF72CF9083C7950041112A8AF7
:10AC200093F7F707A384F50032852E893284EFE08D
:10AC30008F8F93170501C187635EF004AA89C14510
:10AC40002285EFD0BFFA2A8B4E85832A0400EFC0FD
:10AC5000AFE121E583574400231101000544F117BA
:10AC600093B71700A300F100814403481100035774
:10AC70002100D6875285CE862286CA85EFE07FE600
:10AC8000A1679387170248003EC42302810026C6AD
:10AC9000EFE01FB941016F70EF8B13061100A28521
:10ACA000EFF07F81AA8409E523110100094475BFF3
:10ACB000930521005A85EFF09FF2835721002A84E3
:10ACC000CDD797B7FF1F9387E7109C4391C7854562
:10ACD00013052100EF408040835521002685314433
:10ACE000EFC0EFCF59D1231005002685EF70F07A21
:10ACF0000144A5BFEF726F8441112E896C00AA84B4
:10AD000002C6EFF0CF8909CD0357050005072310D0
:10AD1000E500EFF09FEB81473E8541016F702F8486
:10AD20003247954775DBCA852685EF20D008C14795
:10AD3000E34405FE3244854741462310F40083571F
:10AD40000900A685130544002311F400EFD0D06953
:10AD50002285C1B7EF62DFFC83C795004111AA8A43
:10AD600093F7F707A384F5003285AE893284EFD0DC
:10AD70009FFB93170501C187635EF0042A8AC145D2
:10AD80002285EFD0BFE6AA845285032B0400EFC0D2
:10AD9000AFCD21E583574400231101008544F1170D
:10ADA00093B71700A300F1000144034811000357B3
:10ADB0002100DA875685D2862686CE85EFE07FD2BF
:10ADC000A1679387070248003EC42302910022C670
:10ADD000EFE01FA541016F60FFF7A2851306110088
:10ADE000EFF06FED2A8409E523110100894475BF56
:10ADF000268593052100EFF0FFEFAA845DF58355CA
:10AE000021002285EFC0AFBD4DF10149EFD0CF9DAC
:10AE1000635DA900184893171900BA9703D7070074
:10AE20001DE7035721002390E700EFD0EF9B63025B
:10AE3000250397B7FF1F9387E7F99C4389C70355FD
:10AE40002100EF4000222285EF703065B9BF05096F
:10AE500075BF954499BF05C19307F00F630FF500C7
:10AE6000C547630CF5009307F5FF05453315F5005D
:10AE70004205418182800145828041657D15828045
:10AE8000B9E1EF629FEB034506033284EFF0BFFCAC
:10AE90009305803EB305B502C205C18191C9035730
:10AEA000E402854763F6E70013050401EFC02016AE
:10AEB0008357E40241677D176385E700FD17231779
:10AEC000F4026F60DFE98280EF62BFE4004283C773
:10AED0009500444D0349140093F7F707A384F50048
:10AEE00083470400220911673369F900A167B3475A
:10AEF000F90041112A8BAE8A63ECE70C83472400EA
:10AF00001307C00EB91793F7F70F6371F70E0347D6
:10AF10003400C14763ECE70C834744001307E007A4
:10AF200093C707086373F70A834984008347740053
:10AF3000A209B3E9F900856763F9F908034A6400D7
:10AF4000834754004E85220A336AFA00EF4040627C
:10AF500045C123962403834B3400137AFA00239AC5
:10AF60003403238874032399440393890401631AE7
:10AF7000090023A60402239804024E85EFC0A00A0C
:10AF80001DA0034924004A85EFF0FFEC2397A4029B
:10AF9000834744004E85A388F402E3810BFEE30F50
:10AFA00009FCEFC06005EF70907981460146D685B7
:10AFB0005A85EFE09FA5A167938797033EC42302BC
:10AFC0000100480002C6EFE0BF8541016F60FFD776
:10AFD0008544A2862686D6855A85EFE01FA3A16701
:10AFE000938797033EC423029100E1BFBD44D5B7C8
:10AFF0009144C5B7EF62DFD201111C08404D3EC23B
:10B00000B7070F003EC41C083EC62A89AE89EFC0B0
:10B010001F9D585C1C5C634CB70A6394E50063E8B1
:10B02000A70A3385A740B3B7A700B305B7401306F7
:10B03000803E81469D8DEFD0407B93140501C180F9
:10B04000A1659385C5034800EFC02FAC814548003A
:10B05000EFD0BFC1835504044800EFD05FC28355D1
:10B0600024044800EFD0BFC1814599C8C167FD17CE
:10B070009305F00F6386F4002685EF402015AA851E
:10B080004800EFD09FBE03554404814511C9C167F4
:10B09000FD179305F00F6305F500EF402013AA8517
:10B0A0004800EFD09FBC834564044800EFD0FFBB4D
:10B0B000834574044800EFD05FBB500001478146D0
:10B0C000CE854A85EFC0EFC405616F60BFC881447B
:10B0D00085BFEF629FC683C7950093F7F707A384E8
:10B0E000F500EFF03FF16F609FC7EF627FC383C74A
:10B0F00095004111404D93F7F707A384F5002A8A84
:10B100003285B284AE89EFD01FC22A8B2685EFD05C
:10B110009FC12A892685EFD0BFBF93170B0163CA51
:10B120000702E177CA97C207C183116763E3E702A9
:10B1300093070910C207C1831307B00F637BF700A1
:10B1400093170901C187AA8A6348F000C54763FACB
:10B15000570141016F601FC0EFC08F83E31B25FFC4
:10B16000F5B763060B0263040902814463870A0290
:10B17000B7077F0023106405231124057CC0568582
:10B18000EFF07FCD9304803EB304950239A0B7075A
:10B190007F00232004047CC0814403552404EFB0C5
:10B1A000101095CCEFC0BF83269593D7F441333769
:10B1B0009500AE97BA9708DC5CDCCE855285EFF03F
:10B1C0007FE399E023220404A1679387B703480033
:10B1D0003EC42302010002C6EFE08FE49DBF814719
:10B1E00001481CDC232E0403C9BFEF621FB5EFC06A
:10B1F000FFE9E1473305F5029145EF30507FE55710
:10B2000011C597B7FF1F23A1A79E81473E856F6099
:10B210001FB5854717B7FF1F230AF79C8280EF628F
:10B22000DFB197B7FF1F9387E79B80432DC08357FC
:10B230000404639EA70483572404639AB7043689E1
:10B24000B284EFC0CFF95C5C63C3B7046395B70009
:10B250001C5C63EEA7028347640463F3F400A687D3
:10B260002303F4048347740463F39700A687A303BE
:10B27000F4048357440441677D176385E70085071D
:10B280002312F4043C4481C7CA85268582976F60E7
:10B290001FAD97B7FF1F9387E7949C43014599C360
:10B2A00003C587008280EF625FA90111B70707001D
:10B2B0003EC683C79500584D0AC493F7F7070AC8DE
:10B2C000A384F5002A89AE8401CB1C4283C7070002
:10B2D0002304F700EF70D045216493055402280041
:10B2E000EFC0AF82EFF0FFFAAA852800EFD0FF97FA
:10B2F000300001478146A6854A85EFC08FA113041F
:10B300004402480822CC230A010002CEEFE04FD1CC
:10B3100005616F60DFA4EF625FA201117C003ECA8D
:10B32000B70707003ECC7C003ECE83C795002E8435
:10B33000AA8493F7F707A384F500A16593855502C6
:10B340004808EFB09FFCEFF0DFF4AA854808EFD083
:10B35000DF91500801478146A2852685EFC06F9B8B
:10B3600005616F60DF9F97B7FF1F9387A7879C4397
:10B37000094599C303C59700828097B7FF1F93873C
:10B3800067869C43094599C303C5D700828097B758
:10B39000FF1F938727859C43014599C303C5A700D9
:10B3A0008280EF62FF970111B70708003EC683C78E
:10B3B0009500404D0AC493F7F7070AC8A384F50027
:10B3C0002A89AE8429C01442854703C7060063EE6C
:10B3D000E7068347940009468149638EC700B30797
:10B3E000F740A304E400B339F00083C71600230537
:10B3F000F400EF70F03303572403058B09C763840F
:10B400000900EFA0B06B2164930584022800EFB01F
:10B41000DFEFEFF05FF5AA852800EFD01F85EFF092
:10B420001FF7AA852800EFD05F84014781463000CE
:10B43000A6854A85EFC0EF8D13047402480822CC1C
:10B44000230A010002CEEFE0AFBD05616F609F905F
:10B45000EF62BF8E01117C003ECAB70708003ECCE8
:10B460007C003ECE83C795002E84AA8493F7F7070D
:10B47000A384F500A165938585024808EFB0FFE835
:10B48000EFF07FEEAA854808EFD02FFEEFF03FF0F7
:10B49000AA854808EFD06FFD500801478146A28574
:10B4A0002685EFC00F8705616F607F8B97A7FF1F11
:10B4B000938747739C43014599C303C5B7008280B6
:10B4C000EF62BF870111B70707003EC683C795002B
:10B4D000404D0AC493F7F7070AC8A384F5002A89E8
:10B4E000AE8405C41C42054783C70700636AF7049E
:10B4F0000347B400630BF700A305F400EF7050237B
:10B500008347B400A9C3EFD00FD921649305B400D9
:10B510002800EFB09FDFEFF07FF9AA852800EFD079
:10B52000CFF4014781463000A6854A85EFB07FFE03
:10B530002904480822CC230A010002CEEFE04FAED6
:10B5400005616F60DF81EFD02FDAC1B7EF62EFFEE8
:10B5500001117C003ECAB70707003ECC7C003ECEFE
:10B5600083C795002E84AA8493F7F707A384F50078
:10B57000A165AD054808EFB05FD9EFF03FF3AA85AC
:10B580004808EFD08FEE500801478146A2852685F6
:10B59000EFB03FF805616F608FFC97A7FF1F93879F
:10B5A00067649C43094599C303C5C7008280EF6265
:10B5B000CFF801117C00AE843ECAA165B707070031
:10B5C0002A843ECCD1057C0048083ECEEFB0FFD3A4
:10B5D000EFF0BFFCAA854808EFD02FE950080147DB
:10B5E0008146A6852285EFB0DFF205616F602FF7F7
:10B5F000EF62AFF483C7950093F7F707A384F500D4
:10B60000EFF0FFFA6F60AFF5EF628FF183C795003F
:10B610000329C501411193F7F707A384F5001C42E4
:10B6200083C90700854763EC370597B7FF1F9387EA
:10B63000A7B29C432E84AA8495C7EFF01FF68947D2
:10B640006302F502630009028347C900638C370176
:10B6500023063901EF70D00D83572903898B99C3D5
:10B66000EFA0D0452685A285EFF07FF4A167CD0736
:10B6700048003EC42302010002C6EFE06F9A410178
:10B680006F604FED97A7FF1F9387C7559C431D45DC
:10B6900099C303C5E7008280EF622FEA0111B70763
:10B6A00007003EC683C79500584D0AC493F7F707B5
:10B6B0000AC8A384F5002A89AE8405C71C4283C743
:10B6C000070093968701E18663C806048546638573
:10B6D000D7048346E7006386F6002307F700EF7080
:10B6E000300521649305E4002800EFB01FC2EFF09D
:10B6F0007FF9AA852800EFD04FD701478146300057
:10B70000A6854A85EFB0FFE03504480822CC230A1D
:10B71000010002CEEFE0CF9005616F604FE4EF6271
:10B72000CFE101117C003ECAB70707003ECC7C0088
:10B730003ECE83C795002E84AA8493F7F707A3848F
:10B74000F500A165B9054808EFB03FBCEFF09FF3E5
:10B75000AA854808EFD06FD1500801478146A285DD
:10B760002685EFB01FDB05616F606FDFEF624FDB97
:10B77000AA84014417A9FF1F13090947E149EFC033
:10B78000FF906344A400014519A8330534038327BF
:10B7900009003E95835725006395970011056F605A
:10B7A0006FDB0504E9BF032E850063040E1017A3A9
:10B7B000FF1F1303236203230300631503002943C0
:10B7C000639A060E03234E01631503001D43639322
:10B7D000070EEF620FD4C689428A3E89BA8AB684C0
:10B7E000328BAE8B2A84A1E903554E0009E5014353
:10B7F0001A856F608FD5A167A98F116763F7E7007E
:10B80000EFF0DFF68145EFF08FBD0844B70700E0A9
:10B810005841F98F18455CC1B707001FF98F1CC547
:10B820005C4981C76105EFB01000E38209FC228505
:10B83000EF70606E6DBF3285EFA0E0620D434DD9B1
:10B840001C44116703D54700A167A98F63F7E70080
:10B85000EFF0DFF18145EFF08FB8032384009316FA
:10B860004B01D1828347B300035663008588FD8B6B
:10B87000A305F300FD777D8E558EFD76FD16B2048F
:10B88000F18E83274301C58E231273012313D30046
:10B890002304530123052301A3044301D9D722859F
:10B8A000EFB07FBBAA850844B5DD6105EFB0207617
:10B8B000ADBF1D431A858280EF628FC60569AA84D9
:10B8C000AE89328A0144FD5A7D19EFC0EFF063451D
:10B8D000A40001456F600FC8D84493171400BA97AD
:10B8E00003D70700631B37032390570163050A0042
:10B8F0002685EF70E0389C448DC383D76700B3F78B
:10B900002701639C3701D28801488147014781465E
:10B91000014681452685EFF01FE905047DB7EF62FA
:10B920002FC079711C103EC4B7070F003EC61C1013
:10B930003EC883C79500AA8A328593F7F707A38488
:10B94000F5002E893284EFD00FBE93170501C18711
:10B950006350F006AA892285EFD0EFBC2A8A4E8573
:10B96000032B0400EFB05F9039E583574400814416
:10B970000544F11793B71700A303F1008345710045
:10B98000DA872287D2864E862800EFE03FA401475F
:10B9900081463000CA855685EFB0BFB7A16793874F
:10B9A000F70348083ECC230A810026CEEFD05FE79C
:10B9B00045616F602FBAA28513067100EFE0BFAF3B
:10B9C000AA84094445DD5285EFE0EFB80D445DD50A
:10B9D0000546D2852685EFF03FEE2A8445B7EF6213
:10B9E000CFB5835507000346270041112A842E85D1
:10B9F00032C62EC4EFE02FB611C53246A2452285CD
:10BA0000EFF09FEB41016F608FB5EF628FB083C79E
:10BA100095004111AA8A93F7F707A384F5003285B0
:10BA2000AE893284EFD02FB093170501C1876357D9
:10BA3000F008C1452A8A2285EFD04F9B2A8D2285A6
:10BA4000EFD06FAE2A892285EFD08FAC930705F82F
:10BA500093F7F70F1307E007AA8B6371F7062285A8
:10BA6000EFD00FAB2A8C2285EFD08FAAAA8C5285FB
:10BA7000032B0400EFB04FFF29E583574400231147
:10BA800001008144F11793B71700A300F1000544AA
:10BA90000347110083562100938784005685DA8876
:10BAA00022885286CE85EFE03FE6A167E90748008D
:10BAB0003EC42302810026C6EFD09FD641016F60AD
:10BAC000CFA813061100A285EFE0FF9EAA8409E526
:10BAD0002311010009446DBF930521006A85EFF031
:10BAE0006FA12A8455F5835521009356C90013167A
:10BAF000490185486688E2875E87858A5182268566
:10BB0000EFF07FCA2A8469B7EF62AFA083C79500C0
:10BB100041112A8B93F7F707A384F5003285AE898C
:10BB20003284EFD04FA093170501C1876352F0080C
:10BB30002A8A2285EFD02F9FAA8A2285EFD0AF9E36
:10BB40002A892285EFD0CF9C930705F893F7F70F4A
:10BB50001307E0072A8C637DF7042285EFD04F9B03
:10BB6000AA8C2285EFD0CF9A2A8D5285832B040090
:10BB7000EFB08FEF29E18357440085440144F1176A
:10BB800093B71700A301F100034731009307840026
:10BB90005A85DE882688D6865286CE85EFE0DFD6A7
:10BBA0008D4748003EC42302910022C6EFD05FC7F4
:10BBB00041016F608F99A28513063100EFE0BF8FBE
:10BBC0002A84894471D19356C900131649018548C6
:10BBD0006A88E6876287858A5182D685EFF0BFBC86
:10BBE000AA845DB7EF62CF932A8981440144617AC8
:10BBF000916A17ABFF1F130BEB1DEFC0EFBE63C5C0
:10BC0000A40022856F600F95832709009399140083
:10BC1000CE9703D50700330745014207418363628E
:10BC2000570311CD03270B0009C785453E85EF302B
:10BC3000E04A832709000504CE9723900700850476
:10BC40006DBFEFF0BFB2832709000504CE972390A4
:10BC5000070075D58145EFE09FF8D5B7EF624F8CAF
:10BC600083C7950041112A8A93F7F707A384F5004B
:10BC700032852E893284EFD00F8B93170501C1874F
:10BC80006354F004AA89832A0400EFB0EFDD21E1B8
:10BC90008357440085440144F11793B71700A3016B
:10BCA000F10003483100D68752850147CE862686AB
:10BCB000CA85EFD01FE3A167F50748003EC4230201
:10BCC000910022C6EFD0DFB541016F60AF88A28539
:10BCD00013063100EFE02FFE2A84894479D197A71B
:10BCE000FF1F9387270F9C4381CB0449EFC0CFAF41
:10BCF000AA852685EF30803E13050401EFF09FEE04
:10BD00002285EF609079814469BFEF628F8083C79D
:10BD100095004111AA8A93F7F707A384F5003285AD
:10BD2000AE89328423110100EFC0FFFF9317050194
:10BD3000C187635CF0042A8AC1452285EFC01FEBEE
:10BD4000AA8B5285032B0400EFB00FD231E1835749
:10BD5000440085440144F11793B71700A300F10094
:10BD60000348110003572100DA875685D2862686BC
:10BD7000CE85EFD01FD7A1679387270248003EC426
:10BD80002302910022C6EFD0BFA941016F50FFFBF3
:10BD9000A28513061100EFE00FF22A84894469D1CD
:10BDA00097A7FF1F9387070398433E8901CB044958
:10BDB000EFC08FA3AA852685EF304032130504011A
:10BDC000EFF05FE2EFC04FA2954459D993052100EF
:10BDD0005E85EFE03FF2AA8441F51C48035721003D
:10BDE00022852390E700EF60506B83270900ADDBCD
:10BDF00003552100EF30E026A5B7EF529FF183C72E
:10BE000095004111AA8A93F7F707A384F5003285BC
:10BE1000AE893284EFC03FF193170501C1876359A2
:10BE2000F0042A8A2285EFC01FF02A895285032B4D
:10BE30000400EFB06FC321E18357440085440144FF
:10BE4000F11793B71700A301F10003483100DA8717
:10BE500056854A87D2862686CE85EFD09FC8A167B1
:10BE6000F90748003EC42302910022C6EFD05F9B31
:10BE700041016F509FEDA28513063100EFE0AFE363
:10BE80002A84894479D19167CA97C2071167C1830F
:10BE90001307F7EF8544E36AF7FA97A7FF1F938725
:10BEA00067F39843BE8B01CB0449EFC0EF93AA859B
:10BEB0002685EF30A02213050401EFF0BFD2EFC0BA
:10BEC000AF92954459D11C48228581442390270183
:10BED000EF60B05C83A70B00ADDB4A85EF306018E4
:10BEE000ADB7EF529FE52A844105B284EFF09FCFB2
:10BEF00001C52285EF60705A81460146A6852285DC
:10BF0000EF70C00B1C4C89C7DC4799C32285829710
:10BF10006F50FFE497A7FF1F9387C7CC9C43014551
:10BF200099C313850701828097A7FF1F938787CB4B
:10BF300088438280EF527FE09317C600DD8DC205F3
:10BF40004111C1812A8432C6EFC07FD33246228597
:10BF500011829375F60FEFC05FD141016F503FE042
:10BF6000EF521FDC79713C083ED2B7070C003ED47B
:10BF70003C083ED683C79500AE842A8993F7F7071D
:10BF8000A384F500A165938535044810EFB0EFB7A1
:10BF9000C165FD15014417AAFF1F130A2AE5930A7C
:10BFA000400EAE892E8B2EC6EFC00F874205931729
:10BFB00004014181C183B24563E3A702C167FD1754
:10BFC0006385F5004810EFC09FCB501001478146B4
:10BFD000A6854A85EFB0EFD345616F50BFD73307D1
:10BFE000540383270A0BBA9703D6C70163083601A7
:10BFF000638835014810EFF0FFF3DA85050465B773
:10C00000B285EDBFEF52FFD079717C083EC8B7070B
:10C0100011003ECA7C083ECC83C79500AA893285B0
:10C0200093F7F707A384F5002E89EFC0DFCF85676C
:10C03000637EF502A165AA8489050808EFB0EFAC1C
:10C040002685EF30E052133415000A04A285080853
:10C05000EFC0BFC1A6850808EFC07FC235C0014749
:10C0600081461008CA854E85EFB0AFCA45616F5052
:10C07000DFCDB30754030327CA0ABA9703D70700D3
:10C08000631A970003D62700638A65030808EFF058
:10C090007FEADE8505042EC6EFB01FF9420593172F
:10C0A00004014181C183B245E3E5A7FCC167FD17E7
:10C0B000E387F5FA0808EFC09FBC55B7B285D9BF32
:10C0C000C165FD15014417AAFF1F130A2AD2930A5E
:10C0D00080022E8BAE8BC1B7EF523FC6184183470B
:10C0E000170083460700A207D58FD207D18323907C
:10C0F000F50083472700034717008D45A207D98F16
:10C1000091832310F600EFC03FAD6F505FC5EF5233
:10C110003FC1C164014417A9FF1F130929CD930929
:10C120008002FD14EFB05FF06345A40001456F503D
:10C130007FC2330534038327C90A3E958357050020
:10C14000E38797FE0504F9BFEF529FBD2A8AAE89A7
:10C15000B284B68AEF30C04109E591473E856F5001
:10C160007FBF2A894E85EF9010502A84638A0A0483
:10C170008D476DD503570500C547E31147FF0347BA
:10C18000F9018546AD47E31BD7FC8347450091CBBA
:10C190004146A6855D05EFC0D022814761D1AD47FC
:10C1A00075BF130965012302E500CA852685EF10D6
:10C1B000202D15CDA547E3830AFA2302040079BF99
:10C1C00011CD83570500E39A47F94146A685190525
:10C1D000EFC0301F814759D1994749B74E85EFF0DD
:10C1E0001FF32A8495473DD9130955007DBF414669
:10C1F000A685231044012311340113051900EFC053
:10C20000B01E2285EF60B03C814789BFEF52FFB27C
:10C2100079717C003ECCB7070A003ECE7C003ED050
:10C2200083C79500B2842E8493F7F707A384F500A3
:10C230001306A1002A892C002685EFF0FFE9A165ED
:10C2400028088D05EFB06F8C90408355A1000355F1
:10C2500081008546EFF05FEFAA84AA852808EFC029
:10C26000DFA00356A100835581002808EFF09FCC82
:10C27000300801478146A2854A85EFB08FA98547DE
:10C2800048103ED42302910202D6EFD06FD9456107
:10C290006F50FFACEF527FAA79717C003ECCB7079C
:10C2A0000A003ECE7C003ED083C79500B2842E8427
:10C2B00093F7F707A384F5001306A1002A892C0041
:10C2C0002685EFF07FE1A16528088D05EFB0EF83AB
:10C2D00090408355A100035581008146EFF0DFE6D1
:10C2E000AA84AA852808EFC05F980356A100835549
:10C2F00081002808EFF01FC4300801478146A2855D
:10C300004A85EFB00FA148102302910202D402D651
:10C31000EFD00FD145616F509FA4EF521FA2EFF0F5
:10C32000BFE26F50DFA397A7FF1F9387E78B884378
:10C330008280EF529FA0835725004111AE842A844A
:10C340002307B10017F5FFFF1305A5696C0023163D
:10C35000F100EFB0CFD581C42285EF60B02DFD573D
:10C360002310F40013062002814513055400EF50FA
:10C37000DF9F41016F50BF9EEF529F9A79717C0001
:10C380003ECCB7070A003ECE7C003ED083C7950066
:10C39000AA89AE8493F7F7073285A384F5001306C4
:10C3A000A1002C00EFF05FD3035581001144EF3062
:10C3B000201C15C10355A1000144EF90D02A01CDE6
:10C3C000035705008357810045446316F7008545F0
:10C3D000EFF03FF601442169930539002808EFA0EA
:10C3E000DFF2A2852808EFC05F880356A1008355BD
:10C3F00081002808EFF01FB4300801478146A68568
:10C400004E85EFB00F9148104AD42302810202D624
:10C41000EFD00FC145616F50FF93EF527F90979718
:10C42000FF1F9387277C2A8488432E8915C10357D1
:10C4300045038357C401631DF70023260502231813
:10C4400005024105EFA0303E63040900EF60302F84
:10C45000814497A9FF1F93896999130A8002EFB05D
:10C46000BFBC63CCA40297A7FF1F938767809C4340
:10C4700089C70355C401EF10407663050900228582
:10C48000EF6050031306400E81452285EF50FF8D6B
:10C49000FD57231EF4006F50FF8B3385440383A7A1
:10C4A000C90A3E95035705008357C4016315F70079
:10C4B000CA85EFF01FE885045DB7EF527F8683C71A
:10C4C00095004111AA8993F7F707A384F5003285F7
:10C4D000AE84EFC05F8585676370F5042A89EF300D
:10C4E0002009014411C983D7040031446386270120
:10C4F0008545EFF09FF201444E85A2864A86A685C7
:10C50000EFD02FBFA1679387170448003EC42302D2
:10C51000810002C6EFD0CFB041016F50BF83EF5210
:10C520003F809797FF1F9387E76B80431DCC0145A2
:10C53000EFA0E05681470148C1641CDC232E0403B0
:10C540002320040417A9FF1F1309498A01449309F2
:10C55000400EFD14EFB05FAC634BA400814517059E
:10C56000000013054598EFB08FB46F50AFFE330550
:10C5700034038327090B3E958357C50163859700D4
:10C580008545EFF09FE90504F1B79357050113D7EF
:10C590008700A380F50093170501C183A183238041
:10C5A000E5002381F500A381A5008280EF52EFF81A
:10C5B0002300050083C71500A300F50083C72500ED
:10C5C0002301F50083C73500A301F50083C74500AB
:10C5D0002302F50083C75500A302F50083C7650059
:10C5E00093059500A30305002303F500230405002C
:10C5F0003285EFF09FF96F508FF6EF526FF24111D5
:10C60000E9541DC995C993F9C5FF2E842A89AA84C6
:10C61000338AA900B7EA040063149A020D8885449E
:10C6200001CCB7E704009C5F82972AC622866C0083
:10C6300033053901EFC0405B268541016F508FF112
:10C6400083A78A039104829793170501C183A1836D
:10C65000A38EF4FE93570501238FF4FEA183238E4E
:10C66000A4FEA38FF4FE4DBF63E0D502EF52EFECC2
:10C67000B28741113686BE8536C6EFC0E056B24657
:10C68000410136856F50AFED8146368582808387C4
:10C6900005001387F5003D05FD8793F7770883466E
:10C6A00007007D158606B58FA300F5006307B70068
:10C6B0007D17834717009D83DDB78280EF52EFE738
:10C6C000B7E7040083A7070932872A863A8582974D
:10C6D000133515006F50AFE801CD814799C9EF526E
:10C6E000CFE54146EFC0405085473E856F502FE76C
:10C6F00081473E8582801DC5EF522FE4414681452A
:10C700002A84EF508FE64146814513050403EF501C
:10C71000CFE50147C1672322040438C87CC805451A
:10C720006F50EFE301458280814729CDA1CDEF52C3
:10C73000CFE0B2842E891306800581452A84EF500C
:10C74000CFE2CA8524C42685EFF01FF94146814512
:10C750002285EF508FE13044A2852285EFF01FF64D
:10C7600093040401A2852685EFF07FF2A6851305C8
:10C770000402EFF0DFF12285EFF0FFF785473E85F9
:10C780006F50EFDD3E858280EF528FD94111E95421
:10C790001DC995C993F9C5FF2E842A89AA84338AB5
:10C7A000A900B7EA0400639444030D88814401CCD6
:10C7B000B7E704009C5F82972AC622866C00330587
:10C7C0003901EFC06042268541016F50AFD883A781
:10C7D0008A039104829793170501C183A183A38ED5
:10C7E000F4FE93570501238FF4FEA183238EA4FE4C
:10C7F000A38FF4FE4DBF71CDEF528FD2B28401E60C
:10C8000005456F502FD52A842E890145FDD93C4816
:10C810007848B3E6E700F5D69386F7FFB3B7F6009E
:10C820007D17032A4404BA9734C87CC8630F0A04EE
:10C83000C14913050A03B38949412295637B360137
:10C84000B2862E86A685EFF03FE27C40BE9464C09F
:10C8500045BFCE862E86CE85EFF01FE1C114D2945F
:10C860004E9923220404A2879306040103C70700FC
:10C8700003C607038507318FA38FE7FEE398F6FE13
:10C880003044A2852285EFF07FE32699C149330623
:10C89000994063EA9900ADD4A686A68513050403E2
:10C8A000EFF09FDC6DB78147B306F4003307F60065
:10C8B0000347070083C5060085072D8F2380E60008
:10C8C000E39437FF3044A2852285EFF03FDFC114A7
:10C8D0007DBF0145828019C9EF522FC6130680051E
:10C8E0008145EF508FC805456F506FC70145828065
:10C8F00081473DC9B5C9EF524FC4FC4141462E8422
:10C90000AA846393C70413860501A2878146C145A3
:10C9100003C7070003C507038507298F3305D60022
:10C92000034505008506298FA38FE7FEE392B6FE37
:10C930003044A2852685EFF07FD82285EFF0BFF93D
:10C9400085473E856F50AFC1138507031D8E814516
:10C950002295EF508FC17C40130700F813060402A4
:10C96000A2972388E70255B73E858280EF52EFBC3D
:10C970006D712E84B284AA85901028003689EFF05C
:10C98000BFDA19E9D55705A050400C402800EFF058
:10C990009FE66DD9FD142104E5F82C004A85EFF0DF
:10C9A0003FF5814765D13E8551616F504FBBEF52D6
:10C9B000CFB841112EC432C62C000546EFF01FFB44
:10C9C00041016F50CFB9EF524FB701112A842EC6E3
:10C9D00002C802CA02CC02CEEFC06049B2462A8623
:10C9E000A2850808EFF0BFFC1375F50F05616F50C5
:10C9F0000FB7EF528FB47971B2872A84214623088A
:10CA0000B10013051101BE853AC436C6EFC0C01D82
:10CA1000B246930591013685EFF03FB72285141099
:10CA200035460C08EFF0BFF82A84224711E521466D
:10CA30000C103A85EFC0401B228545616F502FB224
:10CA4000EF52AFAF7171AE84AA850A853284EFF0E0
:10CA5000BFC801C90A86A6852285EFF03FC6814777
:10CA600011E1C5473E854D616F506FAFEF52EFA9A1
:10CA70001D712A8AB289BE84354685471305110186
:10CA80002E8CB68A3A8BC28C468D2308F100EFC0FB
:10CA9000A01510100C085285231F0100EFF05FFA5B
:10CAA0002A842DE9A147631BFD069307900591E0B9
:10CAB000E5473546E2851305110113990A0123085C
:10CAC000F10013590901EFC0201213578900939701
:10CAD0008A00D98F90080C085285231FF100EFF0CF
:10CAE0003FF62A8405E9A1E09387FA009183137940
:10CAF000F9003EC6631309004149668B8144C14B6E
:10CB0000854DB2476397970C6A868C0033855C012C
:10CB1000EFC0800D228525616F50EFA2930790042E
:10CB2000C9F8A54779B7834701050947C14B2308D1
:10CB3000F10083471105A58FA308F1009387240016
:10CB4000814463EFFB02014714083386E6008C083A
:10CB5000B386E400BA95DA9683C6060083C505005D
:10CB60000507AD8E2300D600E390E7FE41476398AA
:10CB7000E70490080C085285EFF09FEC35D535A8F6
:10CB8000B3069B00BA871008B305F60090083E96DE
:10CB900003C506000346060085078506298E238007
:10CBA000C500E39277FF998F90080C085285BE94D8
:10CBB000EFF01FE98947014749D52A84A1BF9008B2
:10CBC0003E96034606001408BE962380C6008507DD
:10CBD00079BFB2478504638B971281471808B30663
:10CBE000F70098083E973386F9000347070003468D
:10CBF00006008507318F2380E600E39177FF9008D8
:10CC00000C085285EFF0DFE34DF93546E285130558
:10CC100011012308B101EFB0307D13970401418366
:10CC2000939784002183D98F10180C085285231FF5
:10CC3000F100EFF0FFE051F1814710183387F90060
:10CC40003E960347070003460600B306FB00850730
:10CC5000318F2380E600E39277FF75A01808B306B2
:10CC6000F70098083E973386F9000347070003460C
:10CC700006008507318F2380E600E3E127FFCA879E
:10CC80006398770990080C085285EFF07FDB15F563
:10CC900081479800B306F700900818103E973E961B
:10CCA00003470700034606008507318F2380E6000F
:10CCB000E39177FF3546E285130511012308B101A1
:10CCC000EFB09072139704014183939784002183FE
:10CCD000D98F10180C085285231FF100EFF05FD692
:10CCE000E31D05EC814710183387F9003E96034792
:10CCF000070003460600B306FB008507318F23803B
:10CD0000E600E3E227FFC109410BE5BB8147B5B768
:10CD10009408BE9683C6060018083E972300D700E5
:10CD20008507B9BF638E062CEF423FFE59712A84F6
:10CD3000BE89B28B85473546130511022E8B468C72
:10CD40004289BA8A368A2300F102EFB0F0691018DE
:10CD50000C10228523170102EFF09FCE631E0510F1
:10CD6000A1476319FC069307900563930900E54703
:10CD70003546DA851305110293140A012300F102E6
:10CD8000C180EFB0706693178A0013D78400D98FE3
:10CD900090080C1022852317F102EFF07FCA69ED8D
:10CDA000639009049307FA00BD88918391E0C14420
:10CDB000C207C183DE8C814A3EC6414DB24763EA59
:10CDC000FA0C6286B3854B018810EFB0905F4DC5B9
:10CDD0003D555DA093079004E39C09F8A54749BF22
:10CDE000834701050947C14C2300F1028347110520
:10CDF000B3C7F900A300F10293872900814963EFCB
:10CE0000FC02814618103306D7008C083387D900FE
:10CE1000B69556970347070083C5050085062D8FF5
:10CE20002300E600E390D7FE4147639AE7049008A9
:10CE30000C102285EFF0DFC035D53DA8B3863A014E
:10CE4000BA871010B305F60090083E9603C5060099
:10CE50000346060085078506298E2380C500E392D8
:10CE600097FF3387EC4090080C102285BA99EFF0B9
:10CE70003FBD8947014741D565616F40DFEC9008B0
:10CE80003E96034606001410BE962380C600850712
:10CE900069BFB247850A93990A01939D8A0093D985
:10CEA00009016399570D85473546DA851305110247
:10CEB0002300F10293D98900EFB01053B3ED3D0187
:10CEC00090000C1022852317B103EFF07FB74DF5CA
:10CED0008147A68963E6970626860C084A85EFB047
:10CEE000B05081471810B306F700100898083E9715
:10CEF0003E9603470700034606008507318F2380CF
:10CF0000E600E3E197FE639DA90590080C102285D9
:10CF1000EFF01FB335F181479810B306F700900882
:10CF200018183E973E9603470700034606008507FC
:10CF3000318F2380E600E391A7FF4109C10CBDBDFD
:10CF400018089000B306F7003E963387FC000347AD
:10CF50000700034606008507318F2380E60095BF52
:10CF600098084E97034707001C10CE972380E700D0
:10CF7000850951BF85473546DA851305110223001F
:10CF8000F10293D98900EFB03046B3ED3D01900036
:10CF90000C1022852317B103EFF09FAAE31E05ECC6
:10CFA000814718089000B306F7003E963387FC00CF
:10CFB00003470700034606008507318F2380E600FC
:10CFC000E391A7FF41460C084A85EFB0F041814745
:10CFD0001810B306F700100898083E973E960347CE
:10CFE0000700034606008507318F2380E600E391A2
:10CFF000A7FF90080C102285EFF09FA41DDDADBDAA
:10D000007D558280EF427FD301112A842E859305BE
:10D010005100328902C002C202C402C693047400E5
:10D02000EFF0AFD61D46A68513059100EFB0D03BBB
:10D0300010088A854A85EFF0BFA019ED9307140008
:10D04000180883C607000346070085070507B18E49
:10D05000A38FD7FEE397F4FE05616F405FD0EF42E8
:10D060003FCC2E848C414111AA89838715003289D7
:10D07000914463D30700A1449797FF1F9387C70D7F
:10D080009C43B1C3B5CE8D472310F10083C7250063
:10D090004A852301F10083C73500A301F10083C74E
:10D0A00045002302F10083C75500A302F10083C7A6
:10D0B000650093059100A30301002303F1002304FD
:10D0C0000100EFF08FCC0C404A860A85EFF00FCEBE
:10D0D0000328040083564400A6881D0881470147A1
:10D0E000E51642868A854E85EFF05F982A8909E524
:10D0F000A6852285EFB0FFB24A8541016F409FC5EA
:10D100004A860A85EFF08FCA7DBFEF427FC12E8429
:10D110008C414111AA89838715003289914463D3D8
:10D120000700A1449797FF1F938707039C43B1C350
:10D13000A5CE8D472310F10083C725004A85230122
:10D14000F10083C73500A301F10083C74500230226
:10D15000F10083C75500A302F10083C76500930562
:10D160009100A30301002303F10023040100EFF069
:10D17000CFC10C404A860A85EFF04FC38356440066
:10D18000032804008A85858EC2061D08C1822312E9
:10D19000D400A68881470147E51642864E85EFF008
:10D1A0007FB841016F401FBB4A860A85EFF00FC070
:10D1B000C9B7EF429FB8B335B000011185052A8980
:10D1C0001315F601336515012308B100930511010C
:10D1D00036843AC632C03EC442C2EFF00FBBA2470B
:10D1E0001248425593D68700230BF1009305910115
:10D1F00093578800A30AD100A30BF100230C01016F
:10D20000EFF0AFB83247024603280400B337E0001E
:10D21000835644009207914411C2A1444A85A688CE
:10D2200042860C08EFF09F842A8909E5A6852285AD
:10D23000EFB03F9F4A8505616F407FB2EF425FAE1E
:10D2400001113EC68647B335B0008505AA8913157E
:10D25000F6015D8D2308B1009305110136843A89EA
:10D26000B28442C446C2EFF04FB2224892481645FB
:10D2700093578800A30AF1009305910193D7880082
:10D28000230B0101A30BF100230C1101EFF0EFAF11
:10D290003247104083564400B337E000920703281A
:10D2A0000900914891C0A1480C084E85EFF09FA756
:10D2B000AA8411E5835544004A85EFB09F962685E0
:10D2C00005616F403FA9AA959307F00F17F700007B
:10D2D0001307478A6317B50013C5F7FF1375F50FDA
:10D2E000828005058346F5FFB58FBA9783C707008F
:10D2F000D5B70357450014419307F00F17F6000008
:10D3000013064687369742074183139506014181EC
:10D31000631BE500AD8FB29703C50700130515F336
:10D32000133515008280850603C5F6FFA98FB297D5
:10D3300083C70700D9BFEF425FA0B28736842E862D
:10D34000BA86AA853E85BA84EFF06FE6634B050086
:10D350002285EFB0D0312A86A686A2852685EFF0F9
:10D360000FE56F40DF9FEF42BF9B5D712A8BAE8A56
:10D3700017E500001305857D2C00B284368ABA8932
:10D380003E89EFF04FE42A8459E534104146DA85AE
:10D390002800EFF0CFE12A843DED8547A303F1009B
:10D3A000A6C2930771002408BEC4A68685470D4611
:10D3B0002C18281002DC02DED6C0BEC6EFF00FDB50
:10D3C0002A8431E983477102A6860D4693F7F70751
:10D3D0002300FA00C1473EDE2C188947281026DCBE
:10D3E000A303F100EFF08FD82A8415E54146A68506
:10D3F0004E85EFB0607F8D47A6860D462C1828100D
:10D40000A303F100EFF08FD62A8411E54146A685EB
:10D410004A85EFB0607D228561616F40BF93EF4226
:10D42000DF9197D700009387270C984383C7470065
:10D4300079712A89AE8417E500001305A5710C08DF
:10D440003AC42306F100EFF00FD82A8415E5141032
:10D450004146CA850808EFF08FD52A8411ED1408DB
:10D4600015462C000810EFF08FD42A8411E52146D0
:10D470002C082685EFB04077228545616F403F8EAE
:10D48000EF42BF8B97D70000938707069C477971BF
:10D49000AA842E8417E500001305456C0C083EC6CF
:10D4A000EFF06FD20DE514104146A6850808EFF0A5
:10D4B0000FD011ED140811466C000810EFF02FCFBB
:10D4C00019E58347F10193F7F7032300F400456161
:10D4D0006F40FF88EF427F863688A1488147014729
:10D4E000E546EFF0AFD86F409F87EF421F85368843
:10D4F000A14881470147E546EFF0DF826F403F8654
:10D50000EF42BF8301112A842E850C0832C6EFF04A
:10D510008FCB19E9324797E600009386A662100880
:10D52000C1452285EFF03FE105616F405F83EF4227
:10D53000DF804111C1472EC032C48A8509463EC2F0
:10D540003EC6EFF0AFC241016F407F81EF42EFFE78
:10D550004111AE8613061009AA850A8502C002C2CF
:10D5600002C402C6EFF0AFC441016F404FFFEF426B
:10D57000CFFC328797E600009386C65E2E86930521
:10D580000002EFF05FDB6F408FFDEF420FFB797120
:10D59000C1472ACC2ED032D42C080D4628003ECECE
:10D5A0003ED23ED602C402C602C802CAEFF00FBC89
:10D5B00045616F40CFFAEF424FF80111AA842E84E3
:10D5C00017E500001305855A8A85EFF0CFBF05E502
:10D5D00014084146A6850A85EFF06FBD09ED834723
:10D5E000E1010347F101A207D98FCA07C983617717
:10D5F000D98F2310F40005616F406FF605C9EF4223
:10D60000CFF39787FF1F9387A76290439785FF1FEC
:10D61000938545621785FF1F1305855DEFB080096F
:10D620001785FF1F1305C55C6F406FF31785FF1F3C
:10D630001305055C82809DC5EF422FF09787FF1F81
:10D640009387075F944301112E840A869785FF1FF5
:10D650009385455EEFB0800A0A8502940145056115
:10D660006F40EFEF7D558280EF422FEDEFB08014D9
:10D670009787FF1F23AEA75A17F5FFFF130525F85D
:10D68000EF90D0406F40AFED1787FF1F1307875C07
:10D690009317150008433E95FD572310F50082802F
:10D6A000EF42AFE92A84084019E16F404FEB1C417B
:10D6B00058401CC06313E5005CC08347550023201D
:10D6C0000500F99BA302F500EFB0EFF9E9BFEF42C7
:10D6D0002FE59787FF1F9387E75998432A8411CB3B
:10D6E0008347350093F7070289C70355050089452D
:10D6F000029713054401EF9010138355040003555E
:10D70000E400EF20701B485809C5EFB0CFF5232A7D
:10D71000040213058403EFF0BFF88144B149EFA080
:10D72000FF9A63C5A402834734002320040493F7BF
:10D7300027FCA301F4000048EFA05F9A1316150020
:10D7400081452285EF406FE26F40CFE0B38734031D
:10D750000329040385043E994A85EFF07FF42304EE
:10D76000090075BF8347350093F7070299E3014528
:10D7700082808357E500E39CB7FEC167FD176316FF
:10D78000F600054582800545B9A0EF420FDB9317EF
:10D790000601C187B2842A8401496359F002835784
:10D7A00005008DCB01456367F600034584003E9577
:10D7B0003325A6001375F50F39A81C481317190057
:10D7C000BA9783D70700E38097FC0509EFA01F9164
:10D7D000E345A9FE01456F408FD8EF426FD4AE8973
:10D7E000AA84EFA07F852A84EFD0BFAAAA8601472A
:10D7F0001306840197050000938545E91785FF1FEF
:10D8000013058545EFA0AFD52A8921CD8C4413049B
:10D81000C50022859E0593F50508EFB00FC5CC40E5
:10D8200083877400E18163D1070493E505082285AD
:10D83000EFB0AFC30D46938544002285EFB00FC112
:10D8400083D504002285EFB0EFC583D5240022855F
:10D85000EFB04FC503D6490083A509002285EFB07C
:10D86000EFBE4A856F400FCF93F5F507C9B7EF427A
:10D87000CFCC01112A84328532C6EFB06FB4EF905D
:10D880003F91835704001787FF1F1307275632461F
:10D89000231BF100930700F8A30DF1001C47184368
:10D8A000231AA1008983858BB307F740B285480806
:10D8B0003ECE231C0100230D0100EFF01FF2056195
:10D8C0006F40EFC9EF42CFC50041014529CC930419
:10D8D000C40026853289AE89EFB08FB295452A8A79
:10D8E0002685035B0401EFB02FAF2685EFB02FC66E
:10D8F0008D45AA8A2685EFB02FAE2685EFB02FC5BD
:10D900005C48420A135A0A01D2975CC42318640186
:10D91000814763983A0146054D8133062541933787
:10D92000160013F5F70F6F40EFC2EF428FBE896903
:10D930002A8BAE8B328AB68A81440144314CFD1960
:10D94000EFA0CFF863C9A400EFA04FFB018D33B562
:10D95000AA006F408FBF3389840383270B003E9951
:10D9600063170A008347890085043E94D1BF03569C
:10D970000A00DE854A8533F6C900EFF0BFF47DD199
:10D980000545C1BFEF426FBB01112A847C000355DE
:10D99000E5003ECAB70707003ECC7C003ECEEF1044
:10D9A000303D2A8985454808EFB0EFC199454808C0
:10D9B000EFB02FA7AA844A85EF10B03D2380A400C2
:10D9C0009787FF1F938787429C434166130606F0A3
:10D9D0009396870113D78701558F93D68700F18ED1
:10D9E000558FA207B706FF00F58FD98F11462C007F
:10D9F000138514003EC4EFB0201F5008A38204001A
:10DA000089452285EFF0BFE609C9AA85130584037D
:10DA1000EFB0EFBB3C4085073CC005616F402FB4C1
:10DA2000EF42AFB1EFA08FED2A840504EFA00FEC19
:10DA30003305A402F14791453305F502EF10207B31
:10DA400001E565556F40AFB19787FF1F23ACA72055
:10DA5000EFA0CFEA2A840504EFA04FE93305A40222
:10DA600089450605EF10A07869DD9787FF1F23A37E
:10DA7000A71EEFA0AFE82A840504EFA02FE7330428
:10DA8000A4029787FF1F2399871CEFA02FE72A8402
:10DA9000EFA0CFE5930714003385A7029787FF1FF8
:10DAA000239DA71A97E70000938707D01787FF1FCA
:10DAB0002328F71A014579B7EF428FA6AA842E8949
:10DAC00001449789FF1F93896932130A8006EFA0EA
:10DAD000EFE16345A40001456F40CFA73305440340
:10DAE00083A709024A86A6853E95EFF0BFC719E1D4
:10DAF0000504F1BF0545CDB7EF42AFA1AA8A2E8B31
:10DB0000B28B368C3A8A814401448149978CFF1F3D
:10DB1000938CCC2D130D8006EFA04FDD63C7A400BE
:10DB200011E085494E856F404FA23389A40383A736
:10DB30000C025E86D6853E994A85EFF0BFC219CDAC
:10DB4000EFA0CFDB0544636B4501D2866286DA85A0
:10DB500013050903EFF07FDD11C1854985046DBF11
:10DB6000EF420F9CC16441112A8901449789FF1F2C
:10DB70009389C927130A8006FD1436C632C42EC203
:10DB8000EFA0CFD692452246B2466346A400014597
:10DB900041016F402F9C3305440383A709023E9542
:10DBA00009C683473500C18B9DC791C683473500A1
:10DBB00093F707028DC3630699008357E500639CC2
:10DBC00027010357050001CB63E7E5008347850084
:10DBD000BA97E3CFF5FA05044DB7EF426F94C164ED
:10DBE0002A8901449789FF1F93894920130A8006D7
:10DBF000FD14EFA0AFCF6344A4006F40AF95330591
:10DC0000440383A709023E958357E5006388970084
:10DC10006304990063942701EFF07FAB0504D1BF43
:10DC2000EF42AF8E89692A8AAE8A328BB68B8144E5
:10DC3000178CFF1F130C8C1B930C8006314DFD19A4
:10DC4000EFA0CFCA63C4A4006F40EF8F3389940361
:10DC500083270C028355CA015A863E994A85EFF004
:10DC60007FB005CD814D05A03384AD038327090323
:10DC700003D60B00D68533F6C9003E942285EFF01B
:10DC80007FC419E5850DEFA06FC4E3CFADFC31A0D3
:10DC90002285EFF0FFA023040400850455B7EF426E
:10DCA0004F874169AA8A014A178BFF1F130B0B1478
:10DCB0007D19C14B054CEFA06FC36344AA006F40B0
:10DCC000CF8893098006B3073A0383290B02BE99D4
:10DCD00083D7E900638C270163842A016398570185
:10DCE00003A4890311E44E85EFF0DFC9050AE1B70B
:10DCF00083570401639977079304C4002685EFA036
:10DD00003FF085452A8D2685835C0401EFA0DFEC7A
:10DD10002685EFA0FFFF62056185635F05028D45E3
:10DD20002685EFA07FEB89452685EFA0FFEA894590
:10DD30002685EFA07FEA85452685EFA03FEB834748
:10DD40000500094793F7F7076398E700994526858B
:10DD5000EFA0DFE9A30285014848337D2D01231898
:10DD600094016A9548C40040B5BFEF321FFD37E407
:10DD700004008327041D82979787FF1F83C707F43A
:10DD80001755FF1F1305053DA300F5008327441C0D
:10DD900082978327841C81461306F00F8145014535
:10DDA00082976F30DFFB1787FF1F130727E11843A8
:10DDB0009785FF1F83C585F09787FF1F938787EEA1
:10DDC00083468703034697036397D5009787FF1F12
:10DDD0002386C7EE828083C587010347A7036317A5
:10DDE000B6009787FF1F238BE7EC828003C687016D
:10DDF0006317C7009787FF1F2382D7EC828083C6F3
:10DE00008701130750026319D70093076002178731
:10DE1000FF1F2305F7EA828083C68701130660028D
:10DE20006315D60093077002DDB783C7870155BF1E
:10DE30009787FF1F938707E7D44B09476385E60859
:10DE4000EF32BFEF1789FF1F130909E33E848347B1
:10DE50000900918B9DCFB7E4040083A7041D82972E
:10DE600083A7441C1785FF1F130585E1829783A7AD
:10DE7000841C81461786FF1F034686E281450145C3
:10DE8000829721C183470900ED9B1787FF1F230558
:10DE9000F7DE8347040093F7F70F85C7914717878D
:10DEA000FF1F232BF7E0EFF05FECEFF0DFEFB7E7BA
:10DEB0000400BC4F414691451785FF1F034505DF10
:10DEC00082976F30DFE98280EF323FE78D47411163
:10DED0006304F504C5476306F50285476310F50240
:10DEE0009787FF1F238EA7DCB7E70400BC4B930581
:10DEF00000101785FF1F034565DB829741016F30D6
:10DF00001FE685471787FF1F230CF7DAB7E70400E2
:10DF1000BC4B93050020F1BF9787FF1F938787D8DD
:10DF2000D44B1147638DE600B7E7040083A7071DB4
:10DF30008297B7E70400BC4B930500045DBF054919
:10DF40001787FF1F232A27D783C7070032C62E84CF
:10DF500093F7F70FC5D7B7E4040083A7041D7D141A
:10DF60001374F40F8297E37689FCB245994703C690
:10DF70001500E3F0C7FCFC4409061785FF1F1305D5
:10DF800065D48297BC48930500081785FF1F034599
:10DF9000E5D1829779BFEF325FDA1787FF1F13074A
:10DFA00067D04047184B1C409786FF1F23A2F6D02E
:10DFB0006316E4001787FF1F232EF7CE130584FE98
:10DFC000EF907FF3035564FFEF903FC6EFA0BFE9EA
:10DFD0006F30FFD8EF327FD69787FF1F938787CCAC
:10DFE000D84BDC4799C3EFF01FFB85471787FF1F0E
:10DFF0002324F7CC9787FF1F938747BC9C43930547
:10E0000000021785FF1F034565CA83C7870317876B
:10E01000FF1F2305F7CAB7E70400BC4B82976F3098
:10E020001FD49787FF1F23A1A7C88280EF325FCF3D
:10E0300037E404007C4CA1451785FF1F034505C745
:10E0400082977C48A1451785FF1F034525C6978405
:10E05000FF1F938424C58297DC4489E7EFF05FDDDE
:10E060006F305FCF03D567FFEF903FBCAA897DD5A6
:10E07000D84891476310F7027C4C91451785FF1FE4
:10E080000345C5C282977C4891451785FF1F03450C
:10E09000E5C1829703A9490103D409018947B7E97A
:10E0A00004001787FF1F2329F7C083A7091D210438
:10E0B0004204829783C784011755FF1F1305850902
:10E0C00061191757FF1FA307F70883A7491C418051
:10E0D00082979787FF1F238507BE83A7C91C8146A8
:10E0E00009469375F40F4A85829711E99787FF1FB8
:10E0F00083C747CD89C79740FF1FE7806077B7E7A1
:10E100000400BC4F2146A1451785FF1F034505BAF2
:10E110008297B9B7EF327FC293F7052001112E84A1
:10E1200081CBEFF03FEB1345042005616F303FC317
:10E1300093F70510A9CB9784FF1F9384A4B6DC48FE
:10E14000EFF07FC61787FF1F130747A7184383C742
:10E150008401034787036316F700DC4499C3EFF09B
:10E160009FE385471787FF1F2328F7B4B7E704000D
:10E17000BC4B930500021785FF1F034525B382970B
:10E18000134504105DB793F70508ADC79787FF1FC8
:10E1900083C757B3E91719469785FF1F9385A5B223
:10E1A0001305D10093F4F70F1789FF1F034989B1B5
:10E1B000EFA0902393970401C1831787FF1F1307D4
:10E1C000E7B0231DF100231CF1009787FF1F938701
:10E1D00067AD3ACE3ACAD8432306010009CBDC43E7
:10E1E0009315890154080D46E1856800829713450F
:10E1F000040825BF93F72500B1CF9787FF1F9387AA
:10E2000067AAD84B89476306F7029787FF1F83C722
:10E21000A7A613F7270011EF918B99CFB7E704005A
:10E22000BC4F1306000A89451785FF1F034505A843
:10E23000829713452400D5BD9787FF1F93870798C2
:10E240009C4383C787031787FF1F2309F7A6EFF0B7
:10E25000FFDDC5B793F7050291C7EFF03FDD13452A
:10E260000402E1B593F7850091C7EFF0BFD61345DF
:10E27000840065BD93F7150091C7EFF07FBB134590
:10E28000140065B593F7450091C7EFF07FBA1345C9
:10E29000440061BD93F7050485C39787FF1F83C7BB
:10E2A00067A081CBEFF07FAC91471787FF1F232535
:10E2B000F7A01345040495BD93F705010145E386D6
:10E2C00007E69787FF1F9387E79DD84B9147631019
:10E2D000F7049787FF1F9387279A9C4313D727003C
:10E2E0008583D98F858B91E7B7E7040083A7071D46
:10E2F0008297B7E70400FC4F91451785FF1F034540
:10E30000E59A829785471787FF1F2327F79A1345BA
:10E31000040121BD9787FF1F2386A7AA8280EF32C1
:10E32000DFA19787FF1F23A507989787FF1F23A3C8
:10E33000079885471784FF1F130444881787FF1F1A
:10E34000232CF7961C4083C787031787FF1F2307DB
:10E35000F796EF90FFDF39C19757FF1F23A0A7E083
:10E360001C4017050000130525DB83C787031787AB
:10E37000FF1F2305F7941757FF1FA30DF7DC97879F
:10E38000FF1FA3810792B7E7040083A707088297BE
:10E390009787FF1F238CA7906F307F9CB7C7898E0C
:10E3A000938767ED1757FF1F232AF7DA55BF1787A3
:10E3B000FF1F0347278F795555E39787FF1F9387E3
:10E3C000678E03C7170005079786FF1FA38CE68C8F
:10E3D00003C717008D463377D7029786FF1FA383A5
:10E3E000E68C83C617001777FF1F1307277D184396
:10E3F00093F6F60FA9EA834787031787FF1F230FBA
:10E40000F78A85471787FF1F230EF7889787FF1F17
:10E41000938787869C430145998BA9E3EF32FF914F
:10E4200037E404007C48C1451785FF1F0345058874
:10E4300082973C4885451785FF1F034525878297AE
:10E4400001456F30DF9183C7170085466395F6005D
:10E45000834797035DB78347A70345B782809787B4
:10E46000FF1F83C72784A1CBEF323F8D37E4040021
:10E470009787FF1F238807827C4885451785FF1FE4
:10E480000345C58282977C4C91451785FF1F034544
:10E49000E58182977C4891451785FF1F03450581DB
:10E4A00082973C48C1451785FF1F03452580829709
:10E4B00001456F30DF8A79558280EF321F882A84C8
:10E4C000035565FFEF906FF69777FF1F9387877D62
:10E4D000D847BE841DEBEFA05F989C482320040022
:10E4E0008DEB9777FF1F23A7877C9777FF1F23A1CB
:10E4F000877CB7E70400BC4B89451775FF1F0345B0
:10E50000E57A829701456F309F85630A870018433B
:10E51000D1B780C39777FF1F23AE8778D9BF7955CE
:10E52000DDB7EF329F819787FF1F9387E789884385
:10E5300023260500232405005105EF80D02E6F30DF
:10E540001F82EF328FFF1784FF1F1304E4871C40E4
:10E55000411189CF9C472302B5002AC61CC1EFF0A8
:10E560005FFC1C409C4B99C33245829741016F3040
:10E570000FFFEF328FFC4111444D328532842EC69D
:10E58000EFA00FF92AC42285EFA0EFF903A84400F9
:10E59000630C0800B245835744001840224683D5D7
:10E5A0004500AA862685029841016F304FFBEF3265
:10E5B000CFF8404D1DC408C0970500009385E502C3
:10E5C00013054401EF8090189777FF1F9387C77F4B
:10E5D0009C43014589E79777FF1F23A7877E6F300C
:10E5E0000FF87D55EDBFEF324FF50111680093052F
:10E5F000F00F02C602C802CA02CC02CEEFF07FF4CE
:10E6000005616F30CFF59777FF1F9387E77B9C43BA
:10E61000D847A1679D076311F702EF320FF201118E
:10E620003285EFA0EFEE230AA10081456800EFF0EC
:10E630005FF105616F30AFF282809777FF1F93879C
:10E64000A7789C43D847A167938777036311F702A4
:10E65000EF32AFEE01113285EFA08FEB230AA1005C
:10E6600081456800EFF0FFED05616F304FEF82806C
:10E670009777FF1F938747759C43D8479547631C3F
:10E68000F702EF328FEB011132853284EFA04FE8B1
:10E69000230AA1002285EFA00FE983574400231B22
:10E6A000A10081453ECC1C4068003ECEEFF07FE9E2
:10E6B00005616F30CFEA8280930785FF89CF83277A
:10E6C000C5FF91CBDC4B81CBEF322FE7032585FFD4
:10E6D00082976F30CFE88280EF322FE62A8432852E
:10E6E000EFA00FE3BD4763EBA70018449377F50055
:10E6F0000345B70041995D8DA305A7006F302FE654
:10E70000EF32AFE301117C003ECAB70707003ECCF1
:10E710007C003ECE5C4D8DCF2A8413858700AE846D
:10E72000EF807004A1652A899D054808EF80FFBD30
:10E730009305803EB345B902480893F5F50FEFA065
:10E74000CFD2014781465008A6852285EF807FDC25
:10E7500005616F30CFE0EF324FDEEFF07FFA6F30C0
:10E760000FE0EF328FDD01117C00AE843ECAA1655F
:10E77000B70707002A843ECC48087C0093857503C0
:10E780003ECEEF809FB81C44480883C5B700BD89C2
:10E79000EFA0AFCD500801478146A6852285EF80C6
:10E7A0005FD705616F30AFDBEF322FD92A84AE849B
:10E7B000EFF09FF2A6852285EFF0BFFA6F302FDAD7
:10E7C000EF32AFD7EFF0FFF96F306FD9EF32EFD6FE
:10E7D0000329C5014111630409022A843285B284E8
:10E7E000EFA00FD32AC62685EFA0EFD383274900D9
:10E7F0002A8691C7DC4781C7B245228582974101AD
:10E800006F30EFD5EF326FD3444D81CC2A843285FF
:10E81000EFA06FD1DC40AA8589C79C4799C32285A8
:10E8200082976F30CFD3EF32AFCF032AC5014111AA
:10E8300063030A062E89AA84954532853284EF80C7
:10E84000DFAC85452285EFA0CFBDAA89CA85228588
:10E85000EFA0EFC283274A009DC7DC438DC7228506
:10E86000EFA0AFBA83274A00104083564400DC4330
:10E870007115A307A100B2961307F1004E86CA8551
:10E880002685829701C52380090031A08345F100C8
:10E890002285EFA00FB941016F30CFCBEF32EFC926
:10E8A00065711C083EC2B70780013EC41C0832894E
:10E8B0003EC62A84AE84EFF07FF14A85EFA0AFC652
:10E8C0008357A10089CFAA8550002285EFF0BFF5BC
:10E8D000014781465000A6852285EF809FC359617C
:10E8E0006F30EFC7EF32CFC365711C088329C501B4
:10E8F0003EC2B70780013EC41C082A84AE84328918
:10E900003EC6EFF03FF0638409024A85EFA0AFC135
:10E910008357A100AA8581CF50002285EFF0BFF078
:10E92000014781465000A6852285EF809FBE596130
:10E930006F304FC2EF326FC065711C083EC2B7071F
:10E9400080013EC42A841C0832853EC6AE84EFA0F6
:10E950008FBD8357A10089CFAA8550002285EFF093
:10E960009FEC014781465000A6852285EF807FBA43
:10E9700059616F30CFBEEF324FBC444D91E88347B1
:10E98000450093B71700B307F0403E856F302FBDA9
:10E990001845FD577DDB97070000938707032A84FE
:10E9A0005CCB97050000938565D113858400EF80CB
:10E9B000E05980C003474400814761FB1777FF1F80
:10E9C00023269740D9B7EF32AFB58329C50141114E
:10E9D000032985008147638B0908032409019145B8
:10E9E0002A8A2285EF807F9285452285EFA06FA33A
:10E9F0008945AA8A2285EFA0CFA2AA84EF809F969C
:10EA000083A749002A8B9DC79C438DC72285EFA011
:10EA1000CF9F83A74900A306A1001040835644005E
:10EA20009C431307D100B296D6851306E1005285A8
:10EA3000829709CD83570B002380F400A183A38024
:10EA4000F40023800A00A306010029A88357E100EF
:10EA500022852380F4008345D100A183A380F400A4
:10EA6000EFA02F9C8347D100B337F0000347B900D4
:10EA7000920701453D9BD98FA305F90041016F30F5
:10EA80006FADEF328FAB41111DE99777FF1F938771
:10EA9000E733804305C80440130984009DC55C40EA
:10EAA00099C79C4B89C726852EC68297B245930786
:10EAB000803EB385F5024A85EF80605521A0404D28
:10EAC000AA8479F841016F308FA94A85EF80A0555B
:10EAD0005C40EDDBDC4BFDD726858297E5B7EF3256
:10EAE000CFA52A843285EFA0AFA2AA852285EFF0B8
:10EAF0005FF96F30CFA6EF324FA42A84AE84EFF0D7
:10EB00001FFEA6852285EFF0BFBF6F304FA50841DD
:10EB10003355B50005898280EF322FA21774FF1F8D
:10EB20001304C42C1C5C0111231701008D83858BF9
:10EB3000A303F1008327040B23180100231901000C
:10EB400003D7C7013ECA3C002314E1007D572315BB
:10EB5000E1000357C4023ECC02CE2316E100EF8051
:10EB60002FE38357E101231EA10093F707E093E70A
:10EB70001710231FF1009777FF1F83C7C72985C38D
:10EB800005470145638AE7008347840393E727002D
:10EB90001777FF1F2308F72805616F304F9C8147C7
:10EBA00017D700001307471C8546130671008545DB
:10EBB0004808EF70E04B6DF183478403F59B1777AE
:10EBC000FF1F2301F72685471777FF1F2305F7242B
:10EBD000E1B7EF328F93977DFF1F938D2D2103A611
:10EBE000CD0639712A898147814493060002335743
:10EBF000F600058B01C7850493F4F40F8507E398AD
:10EC0000D7FE83A70D0B231701022318010203D798
:10EC1000C7013EDA3C102314E1027D572315E102BF
:10EC200003D7CD023EDC231901022316E10202DEE6
:10EC3000EF800FD68357E103231EA102014593F70E
:10EC400007E093E71710231FF1029777FF1F83C791
:10EC5000871CA9EF9777FF1F83C7D71C3EC69779FC
:10EC6000FF1F9389A9180144014D9D4A054B954BFF
:10EC7000177CFF1F130CCC1E977CFF1F938CCC1DA1
:10EC800003DAC90563090A00EA8563145903668536
:10EC9000EFF0FFE71DC1050DA1478909E312FDFE55
:10ECA0002DE09777FF1F23AB071A014521616F30D5
:10ECB0008F896285EFF0BFE579DD3247B387840045
:10ECC000E3F0E7FE9C001306140006043E941317BD
:10ECD0008A0093578A00D98FC207C183A30EF4FC20
:10ECE000A183230FF4FC03A70D07B317AB01D98F42
:10ECF0001777FF1F2324F71663047601328461BF60
:10ED000015449777FF1F83C7E7101387170097767F
:10ED1000FF1F2381E61093161400230EF10017D76E
:10ED2000000013076704814785067008CA854818E4
:10ED3000EF700034E34705F68347C10105451777B7
:10ED4000FF1FA309F70C9777FF1F2386270DB9BF75
:10ED5000EF221FFD0111AA892E84EFD0EF9C2A8992
:10ED60009774FF1F938484086399090A9C5C414748
:10ED700093F707036393E70A1777FF1F0347F70922
:10ED8000894763ECE70883A7040B231701002318C6
:10ED9000010003D7C7013ECA3C002314E1007D57A0
:10EDA0002315E10003D7C4023ECC2319010023162A
:10EDB000E10002CEEF80CFBD231EA100EFC06FCDDA
:10EDC0008357C101230FA100914613D78700A207E3
:10EDD000D98F2312F1009777FF1F83D7C70413D76A
:10EDE0008700A207D98F2313F10017D7000013075C
:10EDF00027F78147500095454808EF706027058840
:10EE00009317240003C484036D985D8C9777FF1FCC
:10EE1000238A870005616F20FFF3EF70B0781775C4
:10EE2000FF1F1305A500EF80002083A7040B977533
:10EE3000FF1F83D565FE03D5C701EF10E027977745
:10EE4000FF1F83C727FE93F60702014789E617775E
:10EE5000FF1F035767FC9776FF1F2397E6FC177782
:10EE6000FF1F130767F7184309CBC18B99C7894563
:10EE70001775FF1F035545FA02979777FF1F23ADBC
:10EE800007F89777FF1F238807F89777FF1F23A5B9
:10EE900007FC9777FF1F23A307FC9777FF1F23A18A
:10EEA00007FC83D7840393F7270C93E717001777A2
:10EEB000FF1F2319F7F683572903A18B99C3EF701E
:10EEC000E03F11C49777FF1F23A407F4A1B78D4734
:10EED0001777FF1F232EF7F2EF902FA59305803EA3
:10EEE000B305B5021775FF1F130545F4EF80201217
:10EEF00015B79777FF1F938767EFD85325C791C939
:10EF00009777FF1F238907F09777FF1F23A807F440
:10EF10008280EF229FE283C7F70241112EC6850748
:10EF20001777FF1FA30BF7EE9777FF1F239FA7EE1F
:10EF30009D471777FF1F232DF7ECEF900F9E2A8434
:10EF4000EF90AF9DB24501E5EF902F9DAA85B305E7
:10EF5000B4401775FF1F130565EDEF80400B4101AD
:10EF60006F20FFDF82809777FF1F938727E8D853B2
:10EF700031C7EF229FDC03C7F70205079776FF1F13
:10EF8000A38DE6E811CD8C5F0D4701458981858908
:10EF90009776FF1F23AEE6E6EFF09FDB6F203FDCA6
:10EFA00085479305C0441775FF1F130525E817779C
:10EFB000FF1F232FF7E4EF808005CDB78280EF227B
:10EFC000DFD71777FF1F034707E58547631EF70065
:10EFD0009777FF1F938787E183C7870393C78700CE
:10EFE0001777FF1F2300F7E41775FF1F130505E4CC
:10EFF000EF806003EF807FEF99471777FF1F23298A
:10F00000F7E09777FF1FA38A07E09777FF1F238416
:10F0100007E0EF90AF8F930740063305F50297772F
:10F02000FF1F23ADA7DE6F209FD39777FF1F83C7F6
:10F0300067DFC18B99C7EF225FD0EFF0FFAD6F2084
:10F040001FD2695582809777FF1F938727DADC5399
:10F0500081CBEF229FCE8545EFF09FCF6F203FD031
:10F0600082801777FF1F130767D801468146BA854C
:10F070002148631E06019DCA2390A60083C785030D
:10F0800093E717001777FF1F230EF7D805A08357C4
:10F09000C705631DF502F8598547B397C70093C7A5
:10F0A000F7FFF98F1777FF1F232CF7DA9C5D918309
:10F0B000858B85C79777FF1F83C7E7D599EFEF2229
:10F0C000DFC71D45EFF0FFB06F207FC981E699E3F0
:10F0D0009306C7050506090769BF8280EF227FC333
:10F0E0008605AA84B309B500977AFF1F938ACAD60A
:10F0F000054B977BFF1F938B6BD6214C6394340396
:10F100009777FF1F938787CE9C5F9183858B89CBF1
:10F110009777FF1F83C727D081E72145EFF07FABAB
:10F120006F20BFC203DA0400630B0A041779FF1FC4
:10F130001309C9CB0144CA8C8357C905639D470392
:10F14000A2855685EFF0BF9C11E5A2855E85EFF0A4
:10F150001F9C05C903A74C07B3178B00D98F1777DE
:10F16000FF1F232FF7CE83C78C0393E71700177772
:10F17000FF1F2309F7CA05040909E31F84FB89045B
:10F18000B5BF231E0904C5BF1777FF1F0347A7C8D4
:10F190008547631AF700EF225FBAEFF05FE2EFF006
:10F1A000BF976F20DFBB8280814785451306000231
:10F1B00093861700B397F500E98F13F7F60F89E7E9
:10F1C000B687E397C6FE01473A858280FD478545AD
:10F1D0007D56B396F50013871700E98E1377F70F66
:10F1E00089E6FD17E397C7FE01473A85828089E9E2
:10F1F00001473A85828001473A8541016F203FB639
:10F20000EF22BFB341112AC62E852EC4EFF0DFF9DD
:10F21000A2457D158547B397A700E39EF5FC3246CE
:10F220009377360099C3719A11069777FF1F9387DA
:10F23000A7BB94433E871778FF1F130828BA89EAB3
:10F24000832708009107F19B9776FF1F23AEF6B83E
:10F25000032588001843B307A700B3F7B702B387A5
:10F26000F540FD15FD8D83274800AA95B306B6002D
:10F27000E3F3F6F8E371D5F82E979777FF1F23A3F2
:10F28000D7B63DDB3A858145EF203FAE2A87ADB743
:10F2900018419777FF1F938767B423A4070098C38B
:10F2A0005841D8C39777FF1F23A007B48280EF226D
:10F2B0003FA7AA8401441779FF1F130929B39309B3
:10F2C000400EEF807FD56345A40001456F209FA8C5
:10F2D000330534038327090B3E958357C501E38724
:10F2E00097FE0504F9BFEF22DFA29779FF1F9389EC
:10F2F000E9AF3E84BA848347060003A709004111A1
:10F300009D83058B3D8F83C74401AE8A2A89F99B73
:10F31000D98F238AF4001C44B685231204001CC034
:10F320002285328A36C6EF90DF8FB246D285368686
:10F33000EF90900BDC4883A509000840858B56862A
:10F340009D8DEFD03FCC61E918407D558347570034
:10F3500003476700A207D98FC207C1872394F4002F
:10F360006358F00A83C7440193F70703B5CBD0482D
:10F370009377160003A609001D8E9777FF1F9387CA
:10F38000A7DD9C43ADEB814641A003A70B0093177B
:10F390002A00BA9718409443834757008345670073
:10F3A00033F65601A207CD8F6311F602834737006B
:10F3B0000346470003472700A207D18F4207D98F92
:10F3C000BD82B3F76701638AF604050AEF80DFC3E5
:10F3D000420593170A014181C183E3E8A7FA41BFBF
:10F3E000A16A370B0200014A977BFF1F938BCBADBD
:10F3F000FD1A7D1BE1BF83C7440113070003854647
:10F4000093F70703E391E7F8A2854A85EFD0FFCF92
:10F4100041016F209F936155E5BF7955D5BFEF221C
:10F420003F909774FF1F9384A4849C40D9EF9777F3
:10F43000FF1F9387279A9C436399070CEF80DFBED9
:10F44000930780023305F5028945EFF05FDA41C981
:10F450009777FF1F23A2A7A4EF801FBC9307400E3E
:10F460003305F5029145EFF09FD835C99777FF1F17
:10F4700023A6A7A2EF805FB201CDEF80FFB1914537
:10F480000E05EFF0DFD621CD9777FF1F23AAA7A0A7
:10F49000EF801FCB11CDEF80BFCAD9473305F502EE
:10F4A0008945EFF0DFD405CD9777FF1F23A4A79EF2
:10F4B000EF809FB591450A05EFF07FD30DC1977797
:10F4C000FF1F23A3A7A0014521A8EF803FC29307F8
:10F4D00080063305F5029145EFF07FD101E56555D2
:10F4E0006F205F879777FF1F23A2A7920144130A1B
:10F4F00080061779FF1F1309698FB14AEF801FBF7C
:10F500006364A4029C40E38407F2EF803FBE93074C
:10F51000A0043305F5028945EFF07FCD69D19777D7
:10F52000FF1F23A7A79A19BFEF805FBB8945060578
:10F53000EFF0FFCB4DD5B3094403032709024E97E3
:10F5400008CBEF80BFB8330555039145EFF03FCAB4
:10F5500059D58327090205041374F40FCE9788DB6D
:10F5600071BF9777FF1F93876788884705898280D7
:10F57000C167FD176319F5009777FF1F938707870A
:10F5800003A5070B8280EF224FFBEFF05FD26F20C5
:10F590000FFD814709C58347E501B337F0001777B1
:10F5A000FF1F1307A78418470983058B19C393E727
:10F5B00027003E858280EF224FF82A84EFF07FFDFE
:10F5C0008347E401AA851305940899E3130504030E
:10F5D0009776FF1F938686819442130615021307C0
:10F5E000840213059504EFD0CFC06F204FF7EF22B0
:10F5F0002FF39764FF1F9384647F98442A892E8495
:10F600000983058B9C4019C76314F5006380050EC0
:10F61000014401A2E3FEA7FE1387A702E36AA7FE47
:10F62000850763FCA70883A9440BEF80FF96131698
:10F63000350081454E85EF204FF39767FF1F23A7C5
:10F64000277B9767FF1F23A5077A49CC9C4493E744
:10F6500047001767FF1F232FF7789777FF1F238334
:10F660000780630F040C9767FF1F23A127790144CC
:10F670000549EF807F926341A40AEF80FF949305D0
:10F680000006B3C5A502B7F73600938707E81765EC
:10F69000FF1F1305657D416901449309400E7D19E3
:10F6A000B385F502EF70B016EF801F97634FA40883
:10F6B0000145EF3040700544A9A86398A7029DE575
:10F6C00083A9440BEF805F8D1316350081454E856D
:10F6D000EF20AFE99767FF1F23AA27719767FF1FE6
:10F6E00023A807709C44ED9BADB785C51767FF1F26
:10F6F000034747779307F005E3FCE7F021F8EF6055
:10F70000F03C6DD19C4493E707021767FF1F23234A
:10F71000F76E22856F200FE483A7440B1315340086
:10F720003E958357050081CB8347250099C7214625
:10F730008145EF208FE305042DBF23012501E5BF9F
:10F740009767FF1F23A6076A0DBF3305340383A7FE
:10F75000040B3E958357C50163842701EFF0BFE595
:10F76000050499B7EF226FDDEF801F8613040006B2
:10F770003345A4029764FF1F9384446783C78407BB
:10F780003E951375F50F9767FF1F238DA76C9307A1
:10F79000F00563E7A7020545EF30E061EF80DF8207
:10F7A0003345A402B7F53600938505E8B305B502E5
:10F7B0001765FF1F1305456BEF7070056F202FDA7B
:10F7C0009C4405458983858B81CBEF904F88884089
:10F7D0008145EFF0DFE1DDB7EF30E05DC5B7EF2247
:10F7E0002FD4130495082A8913069005A2851305C2
:10F7F0000503EF90603F1306900581452285EF20B9
:10F80000CFD64A85EF30C0548144176AFF1F130AD0
:10F81000EA5D930A8002EF803F8163C4A4006F20F9
:10F820006FD3338454038327CA0A3E9403570400DA
:10F830008357C9016317F702834744009DC39309A7
:10F8400064014546CE8513055400EF90E0394546E6
:10F8500081454E85EF206FD1228523020400EF30D1
:10F86000005785044DBFEF224FCD9767FF1F938749
:10F8700027409C432A8491C70DC50355C501EFE07D
:10F880000FC29777FF1F9387278D9C4389CBEFB0DB
:10F89000DFD085476315F5002285EF50C05D6F20EE
:10F8A0000FCC41657D15E1BFEF222FC91764FF1F03
:10F8B0001304C4534440938714001767FF1F232980
:10F8C000F752EF30605E1C448983858B9DE758407A
:10F8D000B7E7B0009387075063F1E7020145EFF007
:10F8E0001F9D01CD0545EF809FF608408545050524
:10F8F000EFF0FFCF0145EFF01FF726856F202FC6F1
:10F90000EF220FC2A1642A8901449769FF1F9389DE
:10F91000A95BFD14338AA500EF800FEF6344A400B8
:10F920006F204FC303A7090093172400BA97984389
:10F93000658F42074183634C2701635A4701238047
:10F940000700A380070023810700A38107000504A7
:10F95000E1B7EF228FBB83594500C547411163F5DD
:10F9600037310441C1E533853401834785FF0347BF
:10F9700095FF0348B5FFA207D98F0347A5FFC2072C
:10F98000220733670701D98F0347C5FF0348D5FF17
:10F990002207336707010348E5FF0345F5FF4207E8
:10F9A00022083365A800498FB98F1767FF1F130717
:10F9B000674F1768FF1F1308E8503A858328070030
:10F9C0006384172B1107E31B07FF1767FF1F13073C
:10F9D000674F18431318270042951CC10507A1471C
:10F9E0003367F7029767FF1F23AEE74C93F73500A5
:10F9F0001397470083474601C16B368993F7F7FC9D
:10FA0000D98F32842E8A230AF600814A176CFF1F91
:10FA1000130CCC3DFD1B976CFF1F938C6C25176D51
:10FA2000FF1F130DED4AEF802FDF63C7AA00E154DB
:10FA3000268541016F202FB11308400EB3870A03BA
:10FA400003280C0BB30DF800638E0D2083D7CD0176
:10FA5000638A772183A70C00014B6397071697678A
:10FA6000FF1F938727379C436390071683C70400C3
:10FA700003C70D0493F7F707631BF71ACA8722879A
:10FA8000CE86268693859D0613851D04EFF0BF85DF
:10FA9000631F051883D7CD01032709002320B40174
:10FAA0002312F400FD572313F4008347170093F645
:10FAB000F7078347D40093F707F8D58FA306F40020
:10FAC00093F7F707B337F000B307F0402307F400CC
:10FAD000834717009D839396370083474401DD9B3E
:10FAE000D58F230AF4008347370083464700A207D7
:10FAF000D58F83462700C206D58F1CC88347770061
:10FB000003478700A207D98F2315F4000D4763042C
:10FB1000EA00BD5491DF93870710C207C183130722
:10FB2000B00FBD54E376F7F0EF800FC98144E311C5
:10FB300005F09766FF1F83C666399387160017671F
:10FB4000FF1F2305F7381767FF1F1307E737231B2E
:10FB5000D40093972600144303578400E175BE96A2
:10FB6000A1671386F7FFB377C70098426D8FD98FCF
:10FB70009CC21848F18F3E07D98F9CC2EF80CFC836
:10FB80009767FF1F83C7873433F5A7029767FF1F67
:10FB9000238EA73271BD9307A004B308FB0283270D
:10FBA0000D00BE9803D7080083D7CD01631DF70071
:10FBB00083C7040003C7880093F7F707630BF700B8
:10FBC00083C7FD019DEB050BEF804FD2E345ABFCF6
:10FBD00071BD9385980113859800CA872287CE86C8
:10FBE000268646C6EFF02FF0B24879F983474401E4
:10FBF00093E74700230AF40071BD83C7040003C7DD
:10FC0000980293F7F707E310F7FCCA872287CE869E
:10FC100026869385A8031385A802EFF0CFEC45F55F
:10FC20008347440193E72700230AF400C1B783C741
:10FC3000FD018DCB83C7040003C79D0993F7F70728
:10FC40006312F702CA872287CE86268693852D0CFB
:10FC50001385AD09EFF02FE911E58347440193E7E0
:10FC6000270049BF850AC1B3FD54D9B3EF226F8A7B
:10FC7000797183544500AA8B2E84B28AEF80CFBB62
:10FC8000590563499504B7E4040003A90407EF800C
:10FC9000AFBA59054205418102992A8905CD2AC684
:10FCA00023180100EF804FB959052319A1006146BF
:10FCB000814528089769FF1F938949134ACAEF2095
:10FCC000CF8A2302810203A48900058819E4BC5469
:10FCD0004A85829745616F204F8774003008D6852A
:10FCE0005E85EFF01FC765F56800EF807FF1176A4A
:10FCF000FF1F130A6A4683270A00AA84035B0101D7
:10FD000089CB89476397FA00835501025E85EF50DE
:10FD1000203003552102EF704FC819E50355210229
:10FD2000EF708FD43334A000931764000344C102F2
:10FD30002C0868001374F4FB5D8C23068102EF60CD
:10FD4000B056E9576314F5028356E1029767FF1F27
:10FD5000938787179C43139726006176BA97984339
:10FD6000718F98C39767FF1F2382D71683172102CD
:10FD70006345F00085476396FA00B25793F7070C86
:10FD800095E7D247C2040347C102C180BE9426C68C
:10FD90002318610113770703C147631DF7008347E9
:10FDA0005102054793F7F7076390E704B7E70400AC
:10FDB000BC5739BF92570544A18393F7F707E37700
:10FDC000F4FE15C78347C1021307000293F7070328
:10FDD0006397E700EFB06FFC8547E319F5FC8347B5
:10FDE000C10293F7070389CFEFB0AFCA21A8EFB0E4
:10FDF0008FD7E30985FCEFB04FFAE31985FAD9B73D
:10FE0000EFB0EFD8AA8501460545EF707FF82A8448
:10FE100051DD8347C102414793F707036384E7023B
:10FE200032478347170093F707F8A300F7003247DC
:10FE3000925783461700A18393F7F707FD17D58FD5
:10FE4000A300F70003560101B245130BC4005A8505
:10FE5000EF80DFDFE24A130690058347C10283C4C7
:10FE6000EA01918BB384C40213851404569595C39B
:10FE70005444B3879A0083C7070403C70600137767
:10FE800007F82380E600584483460700D58F2300F7
:10FE9000F700B25703A609008146858B1D8EDA85CF
:10FEA000EFD0EF9B15E9B25783A5090048441386AC
:10FEB0009406858B56969D8DEFD0CF9411ED8327B8
:10FEC0000A0099EFB257054791838D8B6387E7044A
:10FED0009DCF09476389E7042285EF80DFF8F9B5F4
:10FEE000EFB0AFEB85476309F5008347C102414797
:10FEF00093F70703E398E7FC835521025A85EF4007
:10FF0000907C69D183172102E35EF0FAF1B7EFB07C
:10FF10008FC57D151335150061D1014681452285B8
:10FF2000EF70FFEF55BFEFB04FE7E5B7EF12FFE01F
:10FF30009764FF1F938404ED2685EF809FEB2A844E
:10FF400019E16F10DFE11305C40005468145EFF0AC
:10FF5000FFD12285EF803FF1C5B7EF121FDE4111BF
:10FF6000AE842A8493079503130715019306F100C5
:10FF700005466C00268523060100EFD0CFBE1DED9F
:10FF8000A68541462285EF8030468347F1009305E0
:10FF9000140226852308F400EFD06FC805E19767A7
:10FFA000FF1F9387671B9C4389EF1306940497C533
:10FFB00000009385E5DB2685EFD08FD441016F10DB
:10FFC0001FDA1306940297C500009385E5DA2685AB
:10FFD000EFD00FD379D9DDB7EF129FD49767FF1F0A
:10FFE000938787EE8043AE84B289368AAA8AEF80EF
:10FFF000AF811316250081452285EF101FD7976723
:020000040001F9
:10000000FF1F238507EC9767FF1F938727DE03A455
:10001000070B13F714003E89230FE400CE8525C794
:1000200013059408EFF07FF301C555556F109FD26B
:100030008947A30FF4009767FF1F9387E7119C433D
:1000400003278900858093B7170086072300F402F1
:10005000231E54019767FF1F23AA47D985889377EA
:10006000B7FF99C0936747001767FF1F2324F7D88E
:100070002285930700061767FF1F2305F7DEEFF0C1
:100080008FD3014565B713050403EFF01FED45D588
:1000900069BFEF129FCAFD572310F5002311050019
:1000A00023120500231305001306200481452105B2
:1000B000EF10BFCB6F10BFCAEF129FC64111AA84C9
:1000C00001441769FF1F1309A9E09309A0042EC674
:1000D000EF80CF81B2456344A40061550DA0330584
:1000E0003403832709003E9583572500639CB7009E
:1000F0008357050063989700EFF0BFF90145410170
:100100006F105FC50504E1B7EF129FC19767FF1F2E
:10011000938747CC9C434111AA842E84B28903590A
:100120002500C1C39767FF1F83D707CF639B2707AE
:10013000EF700F862A8903D5240093051002B305BA
:10014000B40285472302F10093578900A302F1000E
:1001500093578500A303F10083D744002304A10033
:10016000254613D787002305F10083D76400A30435
:10017000E1004E8513D78700A305E1002306F100B7
:100180001387950093879501A105B386B400A697C0
:100190004C00269723032101EFD0EF9C41016F1003
:1001A0007FBBEF60FFFE51BFEF129FB74111AA84E2
:1001B00001441769FF1F1309A9D19309A0043AC686
:1001C00036C432C22EC0EF707FF282451246A2467C
:1001D00032476344A400615599A0B3073403032553
:1001E0000900AA9703D8070003D5C4016310A80427
:1001F00095E91DEE91CA03C6E4019305100233068A
:10020000B60225063E9690C2014511CB83C6E40195
:1002100013061002B386C602E506B6971CC3410159
:100220006F105FB303D52700E305B5FC050441BF9C
:1002300083C5E40113051002B385A502BE9583C5ED
:1002400085002300B6007DB7EF129FAD5C414111E0
:100250002A8403DA2700C167FD17AE843289630C54
:10026000FA002685EF807F9A8D4763EDA7007D55C4
:1002700041016F103FAE2E85EF803F999D47E3E22D
:10028000A7FEF5B75C40268583D54700EF809F9099
:10029000835584002685EF80FF8F8D452685EF806E
:1002A0003F8EAA89EFF04FE0935705012380F900B4
:1002B00093578500A380F9002381A9005840C167A6
:1002C000FD178345A7006314FA0093E5050826850A
:1002D000EF801F8F9767FF1F9387C7AF9C4308402E
:1002E000D9CF8347B400858BD9CB7800340013066F
:1002F00071008145EFF05FEB1DC98347B4001840E2
:1003000093069005F99BA305F4008347E701B387A3
:10031000D702B306F70083C60604A303D100938671
:10032000170493879706BA96BA9736C43EC61764E1
:10033000FF1F1304A4AB1C440C4026858983858BC6
:100340009D8D834771009E05DD8D93F5F50FEF8040
:100350003F871C44104022458983858BCA861D8EA9
:10036000A685EFC0DFCFE31505F01C440C403246F4
:1003700089838840858B9D8DEFC0DFC8D5BD8347BD
:10038000B40013079005F99BA305F4008347E5012A
:10039000B387E7023307F50003470704A303E1002F
:1003A00013871704938797062A973E953AC42AC65F
:1003B000BDBFEF12FF96032A45009307F00FAA84F2
:1003C0000347AA00AE89328436896316F700EFB07E
:1003D0006FAB2305AA00938AC9000146D6852685FE
:1003E000EFF09FE62A8A21E51767FF1F1307C7D69C
:1003F0001843DC4039C383C6A7000547638FE60274
:1004000083D547005685EF40102C05C9DC40839703
:1004100047006354F00201CC1C4089C74A868145DD
:10042000014582975C4081C7CA85014582974E8508
:10043000EF807FA352856F10FF91DC4003D547000A
:10044000EF60BFD501E9DC4003D54700EF60DFE195
:1004500081471DCD19C41C4089C74A868145014585
:1004600082974E85EF807F9FAA851765FF1F130532
:100470006599EF80DF9511C45C4081C7CA8501454D
:1004800082971765FF1F13052597EF60F0368547A4
:10049000D84085460346A700E30BD6F8031747006C
:1004A0006353E000C9F74A86A2854E85EF703F97F7
:1004B000BDBFEF12FF86AA8401441769FF1F13090D
:1004C00029A19309A004130A9508EF703FC2634461
:1004D000A400014535A033053403832709003E9568
:1004E0008357250099E30504CDB70357050083D74B
:1004F000C401E31AF7FE52868545EFF0FFC065D5CB
:100500006F105F85EF12DF81AA8401441769FF1F16
:100510001309099C9309A004EF705FBD6344A40014
:100520006F105F8333053403832709003E9583579B
:10053000250081CF835705006399970093059502A5
:10054000130610022105EF80206A0504F1B7EF12AF
:10055000CFFE0347E5012A848347F5016307B7000F
:1005600089E781452E856F108FFF230FB400054763
:1005700081C9E398E7FE8947A30FF4008545DDB7FD
:10058000638BE7020947E39FE7FC2285EFF02FA585
:100590009767FF1F938707849C4399E79757FF1F2F
:1005A0009387076D9C4389C70355C401EFF09FF5FE
:1005B000A30F0400E1B755D6C9BFEF126FF6EFA045
:1005C000FFEE85476312F508EF80EFCC1764FF1F3D
:1005D000130484B81C4081CBEFA03FFC894763041F
:1005E000F5001C4082979757FF1F9387A77E9C4377
:1005F000B9CF82979757FF1F938787679C4391C313
:1006000082971754FF1F1304647E8327040B83D43F
:10061000C701EF60FFB78327040BAA85144003C608
:10062000E7011C448983858B99C3136626002685C0
:100630004169EF40C03D8144D9497D19EF705FB0F9
:1006400063CAA4006F100FF1EF800FCA41B7EF70BB
:100650005F884DB7B38734030327840ABA9703D55D
:1006600027006308250103C6470183D50700EF4033
:10067000A03B8504E1B7EF12AFEA01449754FF1F96
:100680009384C4761309400EFD59EF70FF98634FB1
:10069000A40401449754FF1F9384447513098002F6
:1006A000FD59EF707F98634CA40401449754FF1FD9
:1006B0009384C4735949FD59EF709FA8634AA404F9
:1006C00097F5FFFF9385450A1755FF1F1305C57959
:1006D000EF60D00797050000938585851755FF1FAC
:1006E00013058571EF6050056F10CFE633072403C3
:1006F00083A7040B0504BA97239E370179B7330704
:10070000240383A7C40A0504BA972390370151BF75
:100710003307240383A7840A0504BA97239137017A
:1007200061BFD4410387350085473356F5026377AF
:10073000E600A54899E7238006008280B387E70298
:10074000EDB73358F502038735003375F502B3D79B
:10075000E7021307000363DA080103C60500130765
:100760007003118A19E21307700585064297A38F5B
:10077000E6FEC9B718451C416376F7005C41BA979D
:100780002380B7001C4585071CC58280EF12EFDA75
:100790004111AA872E85B285368636C68297634870
:1007A0000500B246158D3335A0003305A040410148
:1007B0006F10EFDAEF12CFD6056941112A8A232094
:1007C000060001448149975AFF1F938AEA72056B1C
:1007D0007D1932C62EC4EF703F85AA84EF70DF8387
:1007E0002695A24532466346A4004E8541016F100E
:1007F0006FD603A70A0093171400BA9703D7070010
:100800003377670101E71CC20504E1B703D707008E
:100810009356D700858AE39946FF33772701E3157E
:10082000B7FEBE89D5B7EF124FD101112EC6B284E3
:100830003689EFB02FEE2A84615501C8B24589E9A7
:10084000232E040023200402014505616F102FD1DF
:10085000A1463008CA852685EFF05FF37DF5835702
:1008600081010357A101231EF4008357C101231006
:10087000E4022311F4028357E101D207D18323124A
:10088000F4028357E1011397370163560700FD57C0
:10089000231FF4005DBF231F040045BFEF124FC8A4
:1008A0001754FF1F130484548327040B03D7C70175
:1008B000C167FD17630EF7109767FF1F9387078ABD
:1008C0009C4381C70545EF406077C1690149930AA0
:1008D000400EFD19176BFF1F130B0B88EF70CFF342
:1008E000634BA90E1757FF1F0347C7579307F00520
:1008F00063E4E702EF704FED93050006B3C5A50270
:10090000B7F73600938707E81755FF1F1305C5553E
:10091000B385F502EF60A06F814517050000130550
:100920008520EF60DFF8EFB0EFDE01CD0357C501A2
:1009300009CB0357E50111C78347050299C3EF604F
:10094000A06BEFB06FDE31C51757FF1F0347475E3F
:100950009757FF1F9387C75D0DCF03C71700230469
:10096000E50003C72700A304E50003C737002305FC
:10097000E50003C74700A305E50003C757002306AA
:10098000E50003C7670083C77700A306E5002307D8
:10099000F5001C4493E717001757FF1F232CF7445B
:1009A0005C4085E7EF708FEF0DC1EF702FEF444093
:1009B0002A89EF70AFEE33F5A4025C40FD17CA97A9
:1009C000898F1757FF1F2325F7420145EF70DF9FDF
:1009D00001456F102FB8B30459038327040BBE944D
:1009E00083D7C40163883703138A0403D2855285F1
:1009F000EFF0AFD605E183C7F40199CF9385940852
:100A00002E85EFF08FD509C91306900581455285D3
:100A1000EF10AFB50509D9B583270B00268593B72D
:100A2000170086072380F402EFE0FFB8E5B785479B
:100A300063F8A7009307F5FFBE953305A040E98D45
:100A40002E8582809841C167BA9713D70701630446
:100A5000A7009CC182804207998FE5BFEF12EFADDE
:100A600041112EC63284B684EFB00FCCE15701C9D4
:100A7000B24591E99757FF1F238C074A81473E856E
:100A800041016F10CFAD9D461756FF1F1306564A02
:100A9000A6852285EFF09FCFAA8775F10547975667
:100AA000FF1F2387E648E1BFEF128FA7411191E9AD
:100AB0009757FF1F23AE07320144228541016F1073
:100AC0006FA9B68532858D467000EFF03FCC2A8441
:100AD0006DF58347D1000347E1001759FF1F130944
:100AE000E930A2074207D98F0347C100D98F1757B2
:100AF000FF1F232FF72EEF706FDA61D1EF700FDA3F
:100B000083244900AA89EF706FD933F5A4028327A3
:100B10004900FD17CE97898F1757FF1F232AF72CFF
:100B200069BFEF128FA11C45AA8491CFD84B01CF8A
:100B300083D7470089CBEF601F92AA8509C58844F7
:100B40006105EF60C04C9757FF1F9387A7289C4310
:100B5000014489EF6F10AFA09C4813171400BA9797
:100B600003D5070019C1EFE0CFCF0504EF70CFC761
:100B7000E344A4FEC5B7EF124F9C011185E9EF6075
:100B80005FDA01449757FF1F23AE072E9757FF1FC9
:100B900023AC072E9757FF1F23AA072E9757FF1F37
:100BA00023A8072E228505616F106F9BB6873285BB
:100BB000C9467000BE85EFF07FBD2A8465F54146C9
:100BC0009305E1001755FF1F1305C52BEF80C001EA
:100BD0000355C100EF608FD7F1B78DE19757FF1F25
:100BE00023A607209757FF1F938747209C4701455F
:100BF000ED9B1757FF1F232FF71E8280EF12EF93F5
:100C00004111B685328595463000EFF03FB815EDBD
:100C1000A2471757FF1F232BF71C9757FF1F9387D8
:100C2000E71C9447B24713F7B6FF13F6170019C233
:100C300013E74600858393F7F7079756FF1F23AB0B
:100C4000E61A1757FF1F230FF72041016F102F914E
:100C5000EF120F8D03841500DC412A89AE848507CD
:100C60000387F7FF19C36340800C8387240091C773
:100C7000635580007D14620461849C40370700FF47
:100C80000907F98F3707001009076392E70A6355D0
:100C9000800079146204618483C70400858B95E326
:100CA0009379F40F4E8A93178A01E187634AF0081B
:100CB000A2876353040081473384F9407D146204A2
:100CC00061848385240081C54A85EFF0BFAA9C40DA
:100CD000370700FF0907F98F370700100907639AE4
:100CE000E706930500034A85EFF0DFA883C70400F9
:100CF00093058005918B99E3930580074A85EFF072
:100D00007FA783C70400858B81CB1374F40F9317DF
:100D10008401E1876347F004C04005048305F4FFC4
:100D2000A1E96F102F837D14620461840DBF370722
:100D300000080907E392E7F6E35080F67D1499BFB7
:100D4000930500024A857D1AEFF0DFA2137AFA0FAD
:100D500099BF370700080907E395E7FA93050003F1
:100D600071BF930500034A85EFF0DFA07D1471BFCA
:100D70004A85EFF03FA055B7EF023FFCEF70CFAAD6
:100D80002A84EF706FA9229589450605EFE02FC6EA
:100D9000E55711C59757FF1F23A0A71681473E852A
:100DA0006F00FFFB930700026306F5005D15133526
:100DB0005500828005458280EF029FF64111AA8985
:100DC0002A89130419008304F4FF32C62EC4268531
:100DD000EFF05FFDA245324659E19307D0026392DE
:100DE000F408830404000548130429009377F6FEF1
:100DF000C9E793070003639FF40E830704001307FA
:100E0000800593F7F7FD6399E706830414004146D4
:100E10000904B70600806314080093C6F6FFB3FE0A
:100E2000C6028147254F654EFD5F33D3C602138747
:100E300004FD6368EF06BA8463D5C408630DF50149
:100E40007D55636AF3006394670063C69E000545A1
:100E5000B307F602A69705048304F4FFC9BF2289ED
:100E60008DB79307B0020148E392F4F883040400BD
:100E70002A88130429009DBF01CA8947E31BF6F89D
:100E800093070003E397F4F8830704001307200493
:100E900093F7F7FD639BE7048304140009460904F4
:100EA0008DBF13E704021307F7F9636CEE00938814
:100EB000F4FB1307700363741E0113077005998C0C
:100EC000A5BF7D576300E50263040800B307F04047
:100ED00091C519C19309F4FF23A035013E85410155
:100EE0006F005FE7B687FDF5D5BF9304000315F2E9
:100EF000214605B719FE294629BFEF027FE20111FD
:100F000061540DC53284AE89414681453689EFF082
:100F1000BFEA93140501C180639E09002685EF3066
:100F2000102B014401C58145EF2050162285056133
:100F30006F005FE22285CD467000CA85EFF01F8505
:100F40002A846DF52685EF30902809E90356C10003
:100F50008345E1012685EF20500B01C941469305E9
:100F6000E1001105EF705048D1B75D54C1B7EF02F1
:100F70003FDB0111E15401CDB284AE894146814588
:100F80003689EFF07FE32A84639709008144268540
:100F900005616F003FDC2685D1467000CA85EFF001
:100FA000EFFEAA846DF58357C100EDD3EF700F8E6D
:100FB0004205931704014181C18363F9A702EFB091
:100FC0008FB64204E14741803304F40241460C08E5
:100FD0002A9413054400EF7030418357E100231138
:100FE000F4008357C1002310F40055B7E55445B70A
:100FF000EF021FD37971E15415C53284AE894146A1
:101000008145B684EFF05FDB13190501135909011F
:10101000639E09004A85EF401065814401C5814502
:10102000EFB02FB1268545616F00DFD2A68593060C
:10103000300270002285EFF06FF5AA8465F54A85CD
:10104000EF4070622A8411E54A85EFB04F8C2A8404
:1010500031C58357C1002311240193096400231073
:10106000F4008347E1009305F10041462302F400B8
:101070004E85EF7070371309740141469305F101F5
:101080004A85EF707036930554004E85EFC04FBF10
:10109000930564014A85EFC0AFBE69B7DD5459B707
:1010A000EF021FC8797111E5E154268545616F0093
:1010B0007FCAB284AE89414681453689EFF0DFCFE1
:1010C000131A0501135A0A015285EFE06FCA2A84E8
:1010D0006398090071D98145EFB02FB48144F1B70D
:1010E0002685930610027000CA85EFF02FEAAA84C5
:1010F0004DFD31C8B2479305D1004146858B230F82
:10110000F400B24713050403858393F7F707A30F91
:10111000F400EF70702D41469305D101130594083A
:10112000EF70902C59B73304690383A70A0B3E94E0
:101130008357C401638337030509EF60FFEDE34480
:10114000A9FEDD549DB7C1690149975AFF1F938AD3
:10115000EAC9130B400EFD19CDB7231E440159BF38
:1011600049CDEF02FFBB4111B289AE8441468145B2
:10117000368AEFF07FC4931A050193DA0A01014918
:10118000175BFF1F130B8BC6EF601FE1634AA900BB
:101190000145ADCC81441759FF1F130929C581A80A
:1011A00083274B0B131439003E9483570400638844
:1011B00057050509D1BF8327490B139434003E948A
:1011C0008357040085E72310540191467000D285AF
:1011D0004E85EFF0AFDB1DE9B24713978700E1833F
:1011E0002183858B58C02301F4000DA08504EF6096
:1011F000BFDAE3C2A4FC5D5511A861558280F1F409
:10120000214681452285EF005FB6014541016F000F
:101210007FB41971D2C4130AC10686CEA2CCA6CA65
:10122000CAC8CEC6D6C2B6D6BAD8BEDAC2DCC6DE08
:1012300052C463810524FD151C102ACC2ECA02CE8F
:101240003EC89304B0021549A9498305060013045A
:1012500016009DE1F2465247E24763FBE620B6974F
:10126000238007007245F6406644D6444649B64995
:10127000264A964A09618280930750026386F500E8
:101280004808EFF02FCFF5A88357C10023070100CE
:10129000014593F7C70F2316F10081450148014727
:1012A000014681469308D00213030003130E300257
:1012B00005048307F4FF99C7638C970463C3F404A0
:1012C000638BC70501CA0346C100858A799AD18E0E
:1012D0002306D100630908008346C100098BF59AF3
:1012E000558F2306E10019C12307B100138707FDBD
:1012F0001377F70FA54663E2E6068146A545294523
:1013000035A0E38717FBE39F67FA0546FD564DB707
:101310000545854571BF05487D5759BFB386A6026F
:1013200005048307F4FFBA96E206E18613F7F70F88
:10133000130607FD1376F60F63E5C500138707FD57
:10134000F1BF1306F7F91376F60F636EC902138720
:1013500097FAE30537FDA306D100130790066385CE
:10136000E704634BF706130780056384E70A6345C8
:10137000F702E38107EE1307500293055002E38161
:10138000E7F02286D9B51307F7FB1377F70FE3646D
:10139000E9FC138797FC75BF130730066386E70ADD
:1013A00013074006E39FE7FC03250A00A947A307AC
:1013B000F100930A4A00635805009307D0023305F1
:1013C000A0402307F1006C00EFF0AFB56C004808B7
:1013D000EFF01F88568A75B713073007638EE7064C
:1013E0006341F7021307F006638EE7041307000753
:1013F000E399E7F80347C100136727002306E100DC
:1014000009A813075007638BE70213078007E39AC5
:10141000E7F6938787FA414793B71700A307E100E0
:10142000139727008347C100ED9BD98F2306F10056
:10143000930A4A006C0003250A0079B7A947A3075D
:10144000F100FDB7A147E5BF83050A004808930AEC
:101450004A00EFF02FB2BDBF83270A006C00480896
:101460003EC8EFF0EFFE1C10930A4A003EC89DB73D
:10147000BA97FDB30145C5BBEF023F8C2A8836857C
:1014800083464800BA8703475800A206D98E3287A0
:1014900017B600001306869089E517B600001306FC
:1014A000A690BE85EFF0FFD66F007F8B9757FF1F8A
:1014B000938787A79C4381CFEF023F88D843B286AA
:1014C0002E861847AA853E8502976F005F89615571
:1014D0008280EF029F868357050039712A84231E7C
:1014E000F100834745009305650041461305F1016E
:1014F000230FF100EF70406F93057401414613050F
:10150000F102EF70606E8356240017B600001306D8
:10151000E691E5450A85EFF0DFCF6C08130630024F
:101520000A85EFF0BFF821616F007F83EF02FF8033
:1015300039712A849305050341461305D101EF70E3
:10154000A06A9305940841461305D102EF70C06963
:101550008347E4010347F4018356C401858B0607E2
:10156000D98F17B600001306268DE5450A85230E90
:10157000F100EFF01FCA6C08130610020A85EFF0A5
:10158000FFF221616F00AFFDEF028FF93704000118
:10159000B70400FF0111814A1759FF1F130909857C
:1015A0007D149389F4FF17BA0000130A6A8DEF6067
:1015B000BF9E63C5AA0005616F00CFF98327490B61
:1015C00013973A003E978347370095CF5C43A301BA
:1015D00007005286B3F687008247E5454800E58F4D
:1015E000D58F3EC083462700B3F73701858AE206D0
:1015F000D58F835607003EC0EFF0BFC111468A85E4
:101600004800EFF0BFEA850A5DB7EF020FF301462D
:101610008145EFF0BFE96F008FF483576500638E5B
:10162000071A1D71A2CCA6CACAC886CECEC6D2C41D
:10163000D6C2DAC05EDE801013F717003289AA84A2
:1016400031CBF99B2313F500EF601F9906053D058B
:1016500041990A8BC16A3301A1408A8B8149014AB1
:10166000FD1AEF607F97634CAA0C7947930604FB41
:1016700017A600001306C67FCA852685EFF0DFDFB8
:10168000638F090C13961900DE85130504FBEFF038
:10169000FFE15A8183D7640013F7270021CBF59B24
:1016A0002393F400EF605F9406053D0541998A8A13
:1016B0003301A1400A8B8149014AEF60FF926345E3
:1016C000AA0A6547930604FB17A600001306C67A0C
:1016D000CA852685EFF05FDA6387090A1396190039
:1016E000DA85130504FBEFF07FDC568183D76400B5
:1016F00013F7470005CBED9B2393F4006547930652
:1017000004FB17A6000013066677CA852685EFF04E
:10171000BFD69C4481C703D747003DEB130504FBAC
:10172000EFF0BFEE130104FAF6406644D644464992
:10173000B649264A964A064BF25B25618280DC4414
:1017400013171A00BA9703D7070063085701939736
:101750001900DE972390E7008509050A19B71305DC
:1017600004FBEFF09FEA35B79C4813171A00BA97AD
:1017700003D7070019C793971900DA972390E7005A
:101780008509050A1DBF130504FBEFF01FE8B1BF73
:101790002314E4FA03D767008326C4FA21465207CC
:1017A00051832315E4FA370700F0758F94479305AA
:1017B00084FA130504FB92069182558F2326E4FADE
:1017C00083C7770013F707018347F4FABD9BD98FCE
:1017D000A307F4FAEFF09FCDB1B78280EF026FD389
:1017E0001744FF1F130484600444797193F7F4FBDA
:1017F0001747FF1F2320F76093F70404A1C78588CC
:10180000A1E097A900009389A967EF60EFF863DB77
:10181000A4028327440B139934003E998356090090
:1018200091CE4E86E5454808EFF0BF9E4808EFF0A0
:10183000DFDD214681454A85EF002FD38504F1B7CE
:10184000EFF09FD41C4413F7F7F79746FF1F23A32D
:10185000E65A93F707086397071E1C4413F7F7EF40
:101860009746FF1F23A8E65813F707106318071EB3
:1018700018449377F7DF9746FF1F23ADF65693760C
:10188000072095C6058B630A072018408983858B3E
:101890003ACA0347840715464C080607D98F17A58F
:1018A00000001305A55A230CF100EFF03FC01C44C3
:1018B00013F7F7BF9746FF1F23AEE65293F7074093
:1018C0008DC3835744000D464C08231AF1008357FB
:1018D000640017A500001305A557230BF100EFF0D6
:1018E000FFBC1844FD749387F47FF98F9746FF1F60
:1018F00023A2F6509317470163DF0700EFA08FE1A3
:1019000019C98356C5016391061A17A5000013056E
:10191000A554EFF09FCF1C447D777D177D8F9746B0
:10192000FF1F23A9E64C13973701635A0702858BE3
:101930006388071CEFA04FDF1DC118458347E500F2
:101940001D463ACA0357C5004C0817A500001305E9
:101950002551231CE100230DF100EFF03FB51844A1
:10196000F977FD17F98F9746FF1F23A5F6489317C0
:10197000270163D90700814517050000130525CA13
:10198000EF50FFF21844E177FD17F98F9746FF1FDC
:1019900023A2F6469317070163D30702EFA0BF986F
:1019A0002A84814417A900001309094CEF600FEE47
:1019B000939704014205C183418163EAA7144561FD
:1019C0006F00AFB883A70A0093141900BE9483D7A1
:1019D000040033F767011DCF1396170133F7770122
:1019E000B3F637016352060417A600001306064437
:1019F00009E717A6000013062644E5454808EFF05E
:101A00005F814808EFF07FC083D70400B3F7470138
:101A10002390F4000509EF602FE1AA84EF60CFDF87
:101A20002695E341A9FA15BD368519C7EF40A043B5
:101A300061DDEFF01FAAC9BFEFD09FB371D5EFF002
:101A4000FFAED9B785697D7A0149974AFF1F938A0E
:101A5000AA4A056B896BFD197D1A75BF858B9DC7D9
:101A6000EF500FF3231AA10041469745FF1F9385BE
:101A7000654113056101EF70201749464C0817A511
:101A800000001305253CEFF07FA2DDB317A5000091
:101A90001305453BEFF07FB7E1BB17A50000130529
:101AA000E53AEFF09FB621B50357E501C177850709
:101AB0003E978357A101FD14133717003207E58FB6
:101AC000D98F231DF100231AD10083560502035735
:101AD00025022146231BD100231CE10003574502A8
:101AE0008566FD16758FFD76F58FD98F4C0817A585
:101AF000000013056536231DF100EFF03F9B21BD6B
:101B000017A500001305C535EFF03FB089BD5C484F
:101B100013F7E7FF58C8858B89CFA6864A86C94543
:101B20000A85EFF00FEF8357040099E70A85EFF07D
:101B3000DFAD850461049DBD231AF10083572400A5
:101B40009305440041462808231BF100EF70C009AB
:101B500051464C080A85EFF07F95E1BFEF02EF9DFB
:101B600085473395A7009747FF1F938727289C47F2
:101B7000411181455D8D9747FF1F23ADA7269377C0
:101B8000057085E393576500858BA1CBC16793876B
:101B900007887D8D05EDEF606FD19305803EB3051D
:101BA000B5021745FF1F130565352EC6EF50A03B44
:101BB000B24519C16349B50085C51745FF1F130517
:101BC000E533EF50C04441016F006F99EF600FCED5
:101BD0002A84EF60AFCEE360A4FCEF602FCE75BF28
:101BE0000145EFF0BFBFC5B7EF022F957971AA8607
:101BF00001441749FF1F1309691F36C6EF60CFB9AB
:101C0000B246635CA4028327490B93143400BE944C
:101C100083D704006396D70285C617A60000130673
:101C20002626E5454808EFF0CFDE4808EFF0FF9D97
:101C3000214681452685EF004F9345616F002F9225
:101C4000050465BF19C223200600814701C593061C
:101C5000D00389E53E8582808505050583870500DB
:101C60000307050099CF6394E700E397D7FE814708
:101C7000D5B79306D0038547E30ED7FC93371700FB
:101C8000D1BF9307F002E316F7FE854761D605053D
:101C900008C2C9B799C123A0050081470DC1130827
:101CA000D0031306F0023307F5008306070081CA4C
:101CB000638706016397C60099C1050798C13E85F1
:101CC00082808507CDB731C9EF02AF8441112E8ADA
:101CD0006C002A89368BB28A97A400009384040E84
:101CE000EFF05FFB2A8C0144A689B14B88406286E5
:101CF000CA85EF70E01801ED0E044E945C40324549
:101D0000DA865686D285829741016F000F840504DA
:101D1000A104E31D74FD6155C5BF7D55828099E521
:101D200061558280615505616F00CF82EFF25EFFE1
:101D30002E8A2A8401118145B28452854146BA898E
:101D40003689EFF06F8793150501C1811376F50F82
:101D5000A1812285EF507FB12A8469D552854C0834
:101D6000EFF05FF3524A2A8BE30E0AFA2A8697A510
:101D700000009385E50F5285EF708010AA8A0DED63
:101D80007D5AEF606FA563C5AA0099E8014561BF60
:101D90005C4413971A00850ABA9723904701D5B778
:101DA0004C442EC6EF604FA3B245131615004E8566
:101DB0000299E34DA0FC85BF5A8697A50000938544
:101DC000A50B5285EF70C00B0DE1032A0401EF60F3
:101DD000AFA11316150081455285EFF01EF9DDD431
:101DE0000C482EC6EF604FA0C1B75A8697A50000D9
:101DF0009385C5085285EF70A00841E11C44A5CF2A
:101E000081ECD443370700E0758F9447D8C3370778
:101E1000001F758F98C701BFA1463008CE854A853F
:101E2000EFE0DF96E31105F01844835781017D76DA
:101E30002312F7008357A101939647018357670048
:101E4000D182F18FD58FF2467D767D16F182858A1B
:101E5000B206F18FD58F2313F7008347E101835634
:101E6000C1012305F7008347B7002314D700FD8B7A
:101E7000A305F7004DBD7D557DB55A8697A5000099
:101E8000938545F35285EF60B07FE31D05E81C4C58
:101E9000E38A07E89C43E38707E8CE864A86A6855F
:101EA0002285829749B5EFF25EE93687B2862E86A3
:101EB000AA850545EFF0BFE66FF07EEAEFF2FEE798
:101EC0003687B2862E86AA850145EFF05FE56FF072
:101ED0001EE9EFF2FEE4411199C123A005009747E6
:101EE000FF1F93876703804381441DC82E89AA89F9
:101EF00031141DC40C4070004E85EFF0BFD419CDD5
:101F000081E8A284630C0900B2472320F90039A0BC
:101F10008C4008400146EFF0FFD265F5404869F873
:101F2000268541016FF01EE3184111CBEFF2FEE070
:101F3000AE873E85B285368602976FF05EE23555F4
:101F40008280EFF29EDF8357C50013D70501C205DB
:101F5000B387E7021841C1814849BA95BE95EFF0B1
:101F6000BFFC6FF0DEDF584111CBEFF21EDDAE8714
:101F70003E85B285368602976FF07EDE35558280CB
:101F8000184509CBEFF27EDBAE873E85B28502971E
:101F90006FF0FEDC355582805C4599C7EFF2FED9C3
:101FA0002E8582976FF0BEDB35558280EFF25ED7CB
:101FB00083290500035AC5002A844849AE84814517
:101FC000EFF09FFD2A890DE193D50401B385450308
:101FD0000356C4004848CE95EFF09FFA2A8909E5D8
:101FE00048488545EFF05FFB4A856FF0BED6EFF2BB
:101FF0003ED32A890441035BC500484979712E8488
:102000008145B28A368AEFF03FF941E193590401E4
:10201000B3896903420441802694A29903440901CB
:10202000330480403374440111CC03254901A28656
:102030005686CE85EFF03FF3AA8431E1330A8A4019
:10204000A299A29A8144630C0A025286D685080896
:1020500003244901EF605039834609011C089305A8
:10206000F00F338646413385470136C6EFF0FECF89
:10207000B2461008CE852285EFF0FFEEAA84032534
:1020800049018545EFF05FF1268545616FF09ECCF3
:10209000EFF2BECA2E864C41A1462A84EFF03FF5EE
:1020A000AA8403450401A145EFE07F985C40338595
:1020B000A74048C026856FF09ECA814797A60000BA
:1020C0009386C6CC6393C70082803387F5000347AD
:1020D00007008507398D13574500369703470700DA
:1020E0001205398D1375F50F1357450036970347C1
:1020F00007001205398D1375F50FE9B7EFF2FEC32E
:102100002A84AA851D461305F00FEFF01FFB8347B5
:1021100074003385A7403335A0006FF05EC4EFF242
:10212000DEC14111A1463000EFF0BFE109ED0357D8
:102130008100C167FD1705456317F7002800EFF020
:10214000FFFB3335A00041016FF07EC1EFF25EBDB1
:10215000AE848C414111A1462A8903440501EFF068
:102160005FDEAA8939E9A1452285EFE05F8C9C40BA
:102170000357C9002A8AAA97939607019CC0C18277
:10218000098F639CE602C16513D70701B385B74089
:1021900011E78355E900FD15C205BE958CC0A14627
:1021A0000A864A85EFF0FFD9AA8901E90A85EFF08E
:1021B000FFF401C9832749009CC04E8541016FF09F
:1021C0007EB90357C9008357210080403307474138
:1021D00063DBE70033FA470363170A004177798C22
:1021E0003E9480C0D9BF03450901A145417AEFE083
:1021F0001F84098CAA8A80C0337A4401417B6364BE
:102200008A0081495DBFA1463000A2854A85EFF072
:102210005FD3AA895DF12800EFF05FEE11E98357E3
:10222000A1000357C100337A6A0180C0BA973E9A71
:1022300033045441E9B7EFF25EB02A84AA851D4603
:102240001305F00FEFF07FE7A303A4006FF03EB19A
:10225000EFF23EAC2A84034505015D71A145EFE034
:102260000FFD5C402A8B0355E4004179B3F7270149
:102270006C003EC6EFE00FFD8355C400B247A14697
:102280003008BE95B385654122852EC8EFF07FCB1F
:10229000AA84634B05002808EFF05FE611C9B24538
:1022A0002285EFF0BFD0AA84268561616FF0FEA978
:1022B000C2470357A101417C338B6741B3F7270124
:1022C000BA973EC810100C082285C24BEFF01FE8E9
:1022D000AA8479F90810EFF07FE22DE95C403ECA4C
:1022E00030104C0822855249EFF05FE6AA844DFD7C
:1022F00003578102835701026316F7002810EFF09D
:10230000FFDF09C55840D247E31CF7FC63902B055B
:102310008357410285CF83572102B3FA8B010810FE
:10232000BE9A1C442311F102EFF0FFF0834904012F
:10233000035A4102B309304193F90902631B0A00B1
:102340000C102285EFF0DFD4AA8439FDE31C7BF763
:10235000B9B74E8963733A015289CA861018D68577
:102360002285EFF01FBEAA8421F1630909000C4405
:10237000CA8610182285EFF09FC7AA84034504017E
:10238000CA85EFE0CFEA1C443E9508C4E39E04F002
:10239000330A2A41CA9A5DB7EFF29E98411191E53E
:1023A000FD54268541016FF0FE9AC44983D725016B
:1023B0004CC904C12316F50003C705012A8423175D
:1023C000E50003C515019316070113070002230852
:1023D000A400C182E366A7FCE1D7B3E4F402E9F00C
:1023E0008547E3FFD7FAA145EFE06FE4AA89014AE8
:1023F00001498357C400931509012285BE95B38511
:1024000035412EC2EFF0BFD119ED0355E4004C0069
:10241000050AEFE02FE39245420A2285135A0A018A
:10242000EFF0FFCF09E905098357E400420913598A
:102430000901E360F9FC8357E40063944701D15438
:102440008DB7639427039245A1463000B38535418B
:102450002285EFF01FAF35E12800EFF03FCA11C52C
:102460000355E4004C00EFE0EFDD9247C17A33877B
:10247000374158C04177F98F1CC44C401C4463EE6F
:10248000F500A14630002285EFF0BFAB1DE5280026
:10249000EFF0DFC6032A44001DC15C400355E40091
:1024A0004179B3F727014C003EC2EFE0AFD9924526
:1024B0002285EFF0DFC6635C0502AA84DDB5124514
:1024C0000359A100035BC10033F5AA002A99034513
:1024D0000401DA85EFE0AFD54A9508C463144501DD
:1024E00063130B04330A3A412322440179B709C527
:1024F0008547A308F40075B54C402285EFF01FAB6B
:102500004DFD48408357C40086093375A9003E95A8
:102510003305354148C03375250108C42285EFF0E5
:102520003FD379D559BF4D5549BF83471501C9CF11
:10253000EFF22EFE2A840345050141112E8AA145A2
:10254000BA893689328BEFE08FCE8357C4000605F7
:10255000898F7D5563E727075C4081443EC2300088
:102560004C002285924AEFF07FBE21ED835B810013
:1025700063994B012800EFF07FB801E58504C204A0
:10258000C18058409247630BF702E3FA99FC8356E7
:10259000C10061559DC663E63403C175B3FABA0044
:1025A0006373D900CA868355A1005A862285D695C1
:1025B000EFF03F9919E50355C10021A06155E3886B
:1025C0004BFD41016FF06EF849558280EFF2EEF657
:1025D0000147EFF09FF56FF08EF8EFF20EF63284C0
:1025E000B2862E86835545000841EFF03FFE6353C7
:1025F00085002A8422856FF08EF6EFF20EF1834774
:1026000015013971C954BDC7034B05012EC62A8473
:10261000A1455A853689328AEFE06FC10D473307ED
:10262000E5028357C400AA8DFD54998F63E4270502
:102630006304090063000A045C403ECA30084C0889
:102640002285524DEFF09FB0AA8945ED8357810155
:1026500032476397E7002808EFF05FAA630605108A
:102660005840D247E31CF7FC8144631B090019A0C2
:10267000814499E7268521616FF0EEECE35CA0FED2
:102680005A85CA85EFE0AFBA014B11C5330BB501CE
:10269000420B135B0B01014D7D5CC17B930C44002D
:1026A0008357E4006380A70D1C4444403307FB00BC
:1026B00063EBE40432472311F1020810FD572310A5
:1026C000E102231221032303F102EFF0DFB66309D5
:1026D00009000C44CA8652862285EFF05F91AA89D0
:1026E00003450401CA85EFE08FB41C443E9508C43D
:1026F000639909000C102285EFF09F99AA89CA847A
:1027000035D9CE8485BF03450401A145EFE02FB242
:10271000B387A4002311F1028357C400B3F47401FA
:1027200023108103BE94898C44C008102312010237
:10273000EFF07FB00C102285EFF09F95AA8403552F
:10274000E400E685EFE00FB05C40B3F777011CC40E
:10275000E39204F22285EFF0BFAFAA84E31C05F0F8
:10276000050D3DBFC15439B78357C101E30209F0DC
:10277000E39827F1C177034C0401B377FD00035DB3
:10278000A101330C8041137C0C023E9DD28ACA8C7D
:10279000E28B63F38C01E68BDE861010EA852285DE
:1027A000EFF02FFAAA84E31B05EC5E860C10568529
:1027B000EF602041AA84E31505ECB38C7C415E9D5B
:1027C000DE9AE3970CFC7DB5EFF22ED781460146E9
:1027D000EFF0BFE26FF0AED8638C050EEFF26ED370
:1027E0005D71054D19C213BD160003590502B68B64
:1027F000328B05094209135909012E8A2A84CA8994
:10280000216C930A8500E15C9304F9FFC204C18046
:10281000638F84059306A0045000A6855685EFF0CB
:10282000FFDA6357050063139501A6892689E9BF7E
:102830009C083E95230A05FA4C005285EFF06EDDA8
:1028400075F563040D088357040263959708938711
:10285000F4FF2310F402894613060402A16556858D
:10286000EFF0BFD96358050661616FF00ECE0145E8
:10287000E31C0DFE0549B1675D55E387F9FE9165DF
:10288000CE9593048400C205DE865A86C1812685D2
:10289000EFF0BFD6630D09005285EF60405DAA8658
:1028A0005286CE852685EFF05FD5E34F05FA835734
:1028B000040263FF3703231034038946130604021E
:1028C000A1652685EFF07FD325A0A689014965B7CC
:1028D0007D558280A6855685EFF01FEFE34605F80B
:1028E0009165FD15CA95C205C1815685EFF0DFEDF2
:1028F000E35CA0F601458DBFEFF2AEC103540502C3
:10290000916A1D71050442042A89AE894180A16B38
:10291000130A8500FD1A130B05029304F4FFC20489
:10292000C180639D7405916B2164130A8900850B36
:10293000170C0000130CACCA83570902930414004F
:10294000C204C18085076383F40E5E949306A004DD
:102950005008A68552854204EFF05FC74180AA8ADD
:10296000854613067100A2855285EFF03FC62A8B7B
:10297000634750076347A00626847DBF569493069D
:10298000A0045008A68552854204EFF03FC4418060
:102990002A8C854613067100A2855285EFF01FC36D
:1029A000634C8003E351A0F883570902E39D97F637
:1029B0009387F4FF2310F90289465A86A165528550
:1029C000EFF0BFC3A6855285EFF01FE0A2855285C8
:1029D000EFF09FDF268491B7E358A0FCA9B7634BC3
:1029E000A000A6855285EFF03FDEA2855285EFF06C
:1029F000BFDD59B79C10BE9A238A0AFA6391090277
:102A00002C004808EFF0EFCC25D91C45224552C6D2
:102A10002318810074006286DA858297B1BF01466F
:102A2000CE854808EFF00FA261FDB9B701452561D9
:102A30006FF0AEB1EFF26EB09737FF1F9387C74DBF
:102A40008043814409C42A893114814401E42685E4
:102A50006FF0EEB0631809005C4481EF404865D820
:102A60003114EDB708400146CA85EFF0AF9D6DF512
:102A7000F5B78297E5F4AA84D5B7EFF20EAC973795
:102A8000FF1F9387E7498043AA8409EC2685EFF06E
:102A90007FFAAA840144EF502FD0636CA4002685EE
:102AA0006FF0EEAB5C402285A6859C438297004088
:102AB000E9BF05041374F40FF9BFEFF20EA8014546
:102AC000EFF0BFFB6FF0AEA99737FF1F9387474525
:102AD00023A0070023A207008280EFF20EA69737FB
:102AE000FF1F9387674323A0070023A20700EFF08F
:102AF000BFFD6FF0CEA6EFF24EA441111309850081
:102B00002A84EF50CFE5AA854A85EFF0FF88AA8492
:102B100019ED89461306E100A1654A85EFF01FAB68
:102B2000E177634405008357E1002310F402268512
:102B300041016FF0CEA29737FF1F9387673E904306
:102B40000147B28691EE05E3DC4310C11737FF1F42
:102B50002328A73C85EF9737FF1F23A5A73C82803A
:102B600036879442C5B7144385E2DC432320050031
:102B700091EB9737FF1F23A7A73A9737FF1F23A192
:102B8000A73A828088C3C1BF14C108C38280EFF214
:102B9000CE9A1734FF1F1304E4332285EFF0BFF5FC
:102BA000AA8405E51799000013094927228597375C
:102BB000FF1F23A32733EFF01FF89737FF1F23AD25
:102BC00027319737FF1F23A1873626856FF02E996F
:102BD0009737FF1F83C78735795599EFEFF2EE9549
:102BE000EFF0BFEFEFF0BFFA11E585471737FF1F92
:102BF000230EF7326FF0AE968280EFF20E94973785
